:020000040000fa
:080000000001040000000000f3
:020000040000fa
:100200008f19210000792200000188000000000001
:100210000c000700e0f72600010020001100070095
:10022000000020000000e000020032000000020098
:100230000000000006390200000000000040da0063
:100240000000fe004440a90040dc20000000e00067
:100250000300320000002000a00188004440a800f4
:100260000000060091018800800078000000eb008b
:1002700015003700e280400032a0b4009101ba00be
:10028000e280400032a0b4009102ba00e280400057
:1002900032a0b4000002eb00472bde00f507b200ed
:1002a000602ce10004003a000059eb008301e900f2
:1002b000fdff3e00040037006128e100010032002c
:1002c0000082eb00040007001101ba000200e00008
:1002d000e8ff3a00000006003159ba008301e90046
:1002e0000c0032002159ba008301e90008003200f5
:1002f0000400e00003003a00e280400032a0b400b5
:10030000f5ff370011d9ba008301e900faff3a007e
:100310008100e800e180400032a0b4000000060047
:10032000a001040000000000ce0104000000000055
:100330001c0b04000000000000000400000000008e
:10034000881f7800020478007e0007000800400043
:100350004f047800000006000000fa00881f7800b3
:10036000000478003fb99700ea81570080007800c8
:10037000001a20007a000700800078000000e000ea
:10038000020035000040eb0000f478000100780026
:100390004f0478000080fa0000000600889fbe002d
:1003a0008004780001007800020478008901780058
:1003b000110020000e000700880f500001003200dd
:1003c0008004eb00090078004f04be000000060026
:1003d0000000fa004fb99700e881570081c920005a
:1003e000e01c20005e0007000080fa00000006000c
:1003f000889fbe008a9fbe008c9fbe008e1f780023
:100400008106780083047800000678000288b9002d
:10041000000778000000e00002003a0000017800c8
:10042000420037000d00e000400032000005780077
:10043000c900900069009000808f500004003900ce
:1004400009007800ff0007000000e00029003500e7
:10045000004020001900600003003a000a04780000
:10046000800578000b0037000a017800a100200009
:100470000c00780036010700800578000000e000dd
:1004800002003a000a047800020037000c00500015
:100490000004e800c90190006900900003005000ca
:1004a000880f500002003100000478008005eb0046
:1004b000080178008c007800030078002100070014
:1004c0000806460008055500490090000000440059
:1004d000c00498000b00e00004003200090078001e
:1004e000250107000000e00002003a000a00e000d9
:1004f000cfff3a00008020001900600002003200a7
:10050000090078001c01070000c0200019006000ed
:100510000200320049009000e00498000a005700f1
:10052000110009000d80d800000178000200780059
:100530004f0778004f06be004f05be004f04be00b7
:10054000000006008001eb000200370061f0790036
:100550008301e800828f5100fcff3a000000060092
:100560006200fa00889fbe008a9fbe000004be00a1
:10057000020578008300780060f92f000f0040002a
:100580003a01070088979f0099979f000000eb00b1
:10059000a09f9f009a4578000b80fb000000ea00b6
:1005a000cf04de0050c2b30080cf550002003200fd
:1005b00009047800010037000904e9000800e000a0
:1005c0000b0034001f909700080178008a00780023
:1005d0008f9197000300010090979f000000e000ba
:1005e000930032002f98970000004400a09f9f00c6
:1005f0000905450050c2b30080cf55000400320009
:100600000b04e000e3ff3a002f98970089003700c1
:100610000000eb00809f9f00f0979f00e0979f00f5
:10062000d0979f00c0979f00b0979f00c09f9f00ea
:100630000900370000d92000008050000000400071
:1006400041d82000e10078004f9897000100700029
:10065000c09f9f000a05e8001a4478008800fb004c
:1006600000d9200006010700800078000000e000ab
:10067000f0ff3a00a0c2b300804f54000e003a00d1
:10068000bf8897000180e900b08f9f0010007800bc
:10069000b09f9f000000e00005003d000000ea0060
:1006a000b09f9f004f9897000020a000c09f9f0020
:1006b0000a05e80010003700b19f9f0009003700cd
:1006c000bf989700f0ff2700808f50000400320091
:1006d0006a08b9000000410003004000b09f9f007d
:1006e0000a05e8001a01fb0003fd2f00030041008a
:1006f000e90f5000f2ff3600e0c2b3009a4f10003d
:10070000040032000080eb00909f9f008a04780074
:100710001c0037008a04e800a0c2b300994f100003
:1007200007003a00bf8897000180e900b08f9f0062
:1007300010007800909f9f008a84e8001100370025
:100740000000eb00909f9f00090037009f989700e2
:10075000f0ff2700808f5000040032006a08b900c3
:100760000000410003004000909f9f008904e800c2
:100770001901fb0003fd2f0003004100e90f5000a9
:10078000f2ff3600194478008800fb0060d9200091
:10079000bb0007000000e00002003a0000447800bf
:1007a000010037008904e800a87f9f0080c6b300dd
:1007b000804f540004003a00994f14000a003a0098
:1007c0006640500006003700c0c6b300804f54009a
:1007d00005003a00994f140003003a0065404000bc
:1007e000a07f9f008904e8000905e800c8fb2f00ee
:1007f0000f04440060f92f000f0040008085e800de
:100800008801780019417800800078000b0078009a
:100810006e0107000000e00005003a008800780043
:100820000b0078009f0007000000e00059ff3d002a
:100830000080eb004f05be004f04be000080fa00b0
:1008400000000600889fbe0000047800c0019000f0
:10085000600090008000eb00808f5100390039006b
:10086000180178002000290000006100e20f50000c
:1008700007003200002020000200e00001003500e7
:1008800000202400000c71008080eb002d00370058
:100890000100260001006100810f500008003a00ad
:1008a00038009000808f5100050039000800780062
:1008b000310007008080eb000000e00021003a00da
:1008c00000c020001800600017003a00a804900043
:1008d0006002200008004000808f540012003a009f
:1008e00000202000b6020700800078002004980055
:1008f0000000e00005003a0029049800490498002f
:100900000900e80030049800060037001860a000d5
:10091000400498000020b00030049800410c98007a
:10092000510c9800f802070028009000500498002d
:10093000380090006004980000002600180c700039
:100940008000eb00010078004f04be0000000600ac
:100950008001eb00040037008301e80090cf100015
:10096000040032000000e800828f5100faff3a00d4
:100970000000eb0000000600889fbe000004780025
:100980000000e0000e003a008004780008c6200055
:10099000180078000000e00004003200f6ff0700b5
:1009a0000000e00001003d008084eb000884e800c6
:1009b00000c72000800f540029003200f4ff3700e8
:1009c000000022001800600024003200a8049000fb
:1009d0000800370009015000384090000000fb007b
:1009e00089007800720907000000e000130034005d
:1009f0008084440048009000808f5400f5ff390047
:100a000028009000400498001801780000c02000e1
:100a10000000610002003200a800900001003700d1
:100a2000b800900000002400000061000a003200bd
:100a3000610498008004eb00090037002800900052
:100a40004004980060049800500c98001890a00092
:100a50008084eb0002003700510c9800800478007d
:100a6000090078004f04be00000006000200fa00f2
:100a7000f1bf9f00010878000080fa000000060026
:100a8000040037000204e00001003a000000050005
:100a90000000e80010417800814f5100f9ff3a0052
:100aa000000006000400fa00889fbe008a9fbe0076
:100ab0008c1f780000047800010678007008900010
:100ac000f8009000010050008808900001005000dc
:100ad0009808900001005000a80890000100500004
:100ae000b808900001005000c8089000810550002f
:100af0000002220090bf9f0000032300a0bf9f00c0
:100b0000081090000028a30018003a000b00e00035
:100b1000160034008b04780009057800e28f540039
:100b2000020036002a002000020037000900e00021
:100b30000b00340058009000c80190000a017800b2
:100b4000ee80570003000100500498000000e00010
:100b5000960032006808900000004500600c980084
:100b60008a8454004240a900ebff3c0078019000c9
:100b70000200e0000b00340058009000c801900013
:100b80008c00780003000100500498000000e00091
:100b90008600320068089000f800900001004000d4
:100ba000600c9800880c90000900e00015003400eb
:100bb00009057800e28f5400020036002a00200068
:100bc000020037000900e0000b00340058009000dc
:100bd000c80190000a017800ec8057000300010072
:100be000500498000000e000700032006808900097
:100bf00000004500600c98008a8454004240a9001f
:100c0000ebff3c00180990000200e0000b003400ec
:100c1000e800900058009000c80190000300010017
:100c2000500498000000e000600032006808900066
:100c30009808900001004000600c9800a80c9000fb
:100c40000900e0001500340009057800e28f540027
:100c5000020036002a002000020037000900e000f0
:100c60000b00340058009000c80190000a01780081
:100c7000ec80570003000100500498000000e000e1
:100c80004a0032006808900000004500600c98009f
:100c90008a8454004240a900ebff3c0038099000d0
:100ca0000200e0000d003400e800900018089000f9
:100cb0008080400058009000c801900003000100af
:100cc000500498000000e0003800320068089000ee
:100cd000b808900001004000600c9800c80c90001b
:100ce0000900e0001500340009057800e28f540087
:100cf000020036002a002000020037000900e00050
:100d00000b00340058009000c80190000a017800e0
:100d1000ec80570003000100500498000000e00040
:100d2000220032006808900000004500600c980026
:100d30008a8454004240a900ebff3c000810900058
:100d40000028a3001b0032000b00e0001900340053
:100d50008b04780009057800e28f54000200360009
:100d60002a002000020037000900e0000b003400d8
:100d700058009000c80190000a017800ee805700ea
:100d800003000100500498000000e000070032005a
:100d90006808900000004500600c98008a845400a8
:100da0004240a90003003400eaff37000080eb0056
:100db000010037000000eb004f0678004f05be0031
:100dc0004f04be000080fa0000000600889fbe00ad
:100dd0008a1f7800000478000102780082447800bd
:100de0000305780070c6b300804f510021003c001d
:100df00000c0e900804f5100de003d00724050000d
:100e0000804f51004b0132000d003c006c405000ff
:100e1000804f51005e013c0000c0e900804f51004e
:100e2000d4003d0050c2b300804f51005501320044
:100e30007c404000804f510055013a00cd00370002
:100e400010c6b300804f5100ca00320004003c00bd
:100e500069405000804f51004d013a007200370048
:100e600030c6b300804f5100180032000040e80047
:100e70000900370000c7b300804f51001e01320047
:100e800008003c0000c0e900804f5100e40032003f
:100e900065003c006540500080cf54003c013a00a2
:100ea0000f00370050c7b300804f51005e00320082
:100eb00063404000804f51005b00320065405000ad
:100ec000804f510032013a001a0137009180e90049
:100ed000010a7800780090009171780032013700a3
:100ee000a8609000c0c6b30080cf50000a003a004e
:100ef0009400780064805000000a78001000be0062
:100f00004f89de00cf91de000002be0002037800b0
:100f1000820378001300370010c7b30080cf500061
:100f200003003200a0c6b30080cf500006003a0094
:100f30009400780068805000000a78003002be00fb
:100f40002003be00070037001480e900000a780083
:100f50001000780000027800cfa2de0005037800c0
:100f600086037800049cbe000694be00a860900032
:100f700080c6b30080cf50000e00320020c6b30000
:100f800080cf500005003a000400fb00cf80de0057
:100f900001017800820178000a00370040c7b300e1
:100fa00080cf5000030032006640400080cf5000e8
:100fb00006003a0004007800cf80de0001017800ce
:100fc00082017800009cbe000294be003800be0082
:100fd0002801be00e00f5000e08f5800e00f5900dc
:100fe000e08f590003003d0078009000d1c2b300ab
:100ff0000a003700081090000018a3000300320018
:1010000078009000b1c2b300040037000008a300cc
:10101000530032007800900001c2b30001757800df
:101020000000e8004d003700a8609000c0c6b30083
:1010300080cf500006003a00940078006480500091
:10104000000a78001002be006033b80013003700b9
:1010500010c7b30080cf500003003200a0c6b30019
:1010600080cf500006003a0094007800688050005d
:10107000000a78003002be002003be0007003700df
:101080001480e900000a780010007800000278005f
:10109000050020000600200007002000049cbe0080
:1010a0000694be00a860900080c6b30080cf5000b8
:1010b0000e00320020c6b30080cf500005003a0079
:1010c0000480fb000100200002002000030020003b
:1010d0000a00370040c7b30080cf50000300320041
:1010e0006640400080cf500006003a0004007800bf
:1010f000010020000200200003002000009cbe0030
:101100000294be00081090000038a30014003200c2
:101110003800be002801be00e00f5000e08f5800ec
:10112000e00f5900e08f59000d00320080c7b30076
:1011300080cf54000300320080c5b30080cf54003c
:1011400007003a007800900001c3b30001757800f1
:101150008000e80009f578000080e800700498003d
:1011600078009000000045006004980089407800f5
:101170006d003700a8609000c0c4b30080cf50005d
:1011800006003a009400780068805000000a780059
:101190005001be004000be000500370094007800fa
:1011a00064805000000a78001000be00d6090700d5
:1011b000009cbe000294be00380090000000e000d9
:1011c00003003d0078009000d1c2b3000a00370050
:1011d000081090000018a30003003200780090006f
:1011e000b1c2b300040037000008a30005003200bc
:1011f0007800900001c2b300017578000000e8009b
:101200007004980078009000000045006004980089
:101210008940780008007800a702070064003700c2
:10122000a8609000c0c6b30080cf500025003200f7
:101230000a003c006440500080cf5000280032007b
:1012400000c0e80080cf5000140032006840500019
:1012500080cf500022003a000a00370040c7b30098
:1012600080cf50001e0032006640400080cf50000a
:101270001b0032006940500080cf500018003a0037
:10128000060037001480e900000a7800100078009a
:10129000485c900008487800450037001480e90059
:1012a000000a78001002780068089000cf80de0005
:1012b0000101780082017800009abe000292be000f
:1012c0003b0037001480e900000a78001001780024
:1012d00068089000cf80de000089be00340037002f
:1012e0001480e900000a780010007800680c900073
:1012f000080878002e0037001180e9008008780087
:1013000010007800cf80de000101780082017800b3
:10131000009cbe000294be007800900000004500d2
:101320006004980081c7b30008007800ce00070071
:101330001f0037001480e900000a780010007800d0
:1013400060049800580990000200e00002003d008f
:1013500052020700090037008000eb007cfd070007
:10136000800078000000e000030032006800900078
:10137000008050000100370058089000100c9800c1
:101380000b003700780090000275780006003700e7
:1013900078009000800045000904e00001003a0058
:1013a00059c2b300894878000000e8007004980032
:1013b0000000eb004f0578004f04be00000006005f
:1013c000889fbe00e30440000900a100808f540004
:1013d0004a003600e38f540001003e00490020001f
:1013e000026d80000200e0000200320082007800fe
:1013f0000c00370021da200003003700908f5400e2
:10140000230036008080e800110078000000e00032
:10141000faff3a000f003700908f54001c0036008e
:101420008080e800110078000000e000faff3a0038
:101430001201780021da200003003700908f540059
:10144000130036008080e80011007800820f500001
:10145000faff3a00f86c8000890f54000100310057
:1014600009047800080078003c0407000000e00050
:1014700004003a00890f5400200032000804d10013
:10148000f5ff3700081878003b040700d4ff370049
:10149000110178009201780064805100890f50009a
:1014a0000300310012009000800878000700370028
:1014b0000900410080087800920190001300980014
:1014c0001100780012881400090978009100780052
:1014d0000100e00005003200110090000000e00073
:1014e000020032000180e800010037000000eb003c
:1014f000006d88000280e800010037000000eb006a
:101500004f04be0000000600881f780048da200063
:101510001804e00004003a00c0b120004a040700ab
:1015200020c0b300004c78004f0478000000060093
:10153000889fbe00000478000ffd0700800478003b
:101540000004200018006000020032002800900013
:10155000090407000000eb002004980038409000c8
:101560000004e000050035000000fb00c406070091
:101570000000e000010032008084eb0018109000b1
:101580000000e00008003200c60607000000e0008e
:10159000010032008084eb0018109000f603070071
:1015a0000000eb00101498000008200018006000f4
:1015b000100032000000eb0001c62000910f140063
:1015c000070032000000e8008180e800e80f5000ca
:1015d000faff3a0008007800e7030700130037001d
:1015e000000140008000eb0000c6200001307900bf
:1015f000f8ff3700000c780000c0eb003044980082
:101600006002200008004000200498004004980078
:1016100050049800400c980060049800500c98000a
:101620007004980076004400000c980009007800cf
:101630004f04be0000000600881f7800e8c62000a6
:10164000180078000000e00001003200b8ff070039
:101650000884e900e0c52000800f5400f8ff3a003c
:101660004f047800000006002f03b000889fbe00e2
:101670008a9fbe008c9fbe008e1f780000077800f6
:1016800030d72000c0b79f0080c5b30080cf500086
:101690000800320022d62000c2b79f0077404000e9
:1016a00080cf500003003a0083002000b3b79f00b2
:1016b0000a00370080c7b30080cf50000500320019
:1016c000a4002000b4b79f0080c5b30080cf5000b5
:1016d00002003a0005012000b5b79f003e04be009d
:1016e0002e05be0040c6b30080cf5000030032007c
:1016f0006540400080cf50000b003a00e00f5400de
:10170000e08f5c00e00f5d00e08f5d0006003d00b3
:101710006000b8006011b8000804500089845800c7
:101720000a0559008b8559003fb19700e80f510019
:1017300003003200f00f510045003a00020037006c
:101740003c002000010037004c002000e00f540056
:10175000e08f5c00e00f5d00e08f5d0005003a0067
:101760005e08900083012000a3b79f000000e00006
:10177000080032003fb297000400e9000800600052
:10178000cfb297006540780090df9f007001200085
:10179000a0b79f008c0078008100e90005003300ad
:1017a0008b05d1000a85d3008984d3000884d30037
:1017b000f9ff3700089fbe000a97be002fb19700bf
:1017c0000200e90023fc2f008f81410000844100ca
:1017d000140037002fb097000000e900a0b79f0069
:1017e0003fb197000200e90004006000cfb197000c
:1017f000635478003e00be002e01be000c0278004b
:101800000402e900050033008381d1000281d30086
:101810008180d3000080d300f9ff3700009fbe0015
:101820000297be003e02be002e03be00e00f520033
:10183000e08f5a00e00f5b00e08f5b00da003400bd
:101840002fb097000000e000e2ff3c00d600370018
:10185000ae60900080c6b30080cf50000b00320015
:1018600006003c000104e000080032006640500021
:1018700080cf500073003a0004003700c0c6b300a8
:1018800080cf50006f003a00310037000801780027
:101890000800e00005003a005e0890008101200089
:1018a000a1b79f000000e00009003200bfb197001f
:1018b000110009000381d8008000fd004fb297009d
:1018c0006440780090df9f0075012000a5b79f005d
:1018d0003fb29700110009000481d8008001780010
:1018e000afb297000500e90021fc2f008f80400077
:1018f000008240000c003700bfb2970011000900c1
:101900008501d800000178002fb097000000e900a1
:10191000a0b79f000590b90000805100cfb097009c
:1019200061527800820178000300e0000300340077
:101930002fb197000200e000efff3c0003007800a9
:10194000cf80de0001017800820178003a00370084
:101950000806be00e00f5400e08f5c0005003a006e
:101960005e08900083012000a3b79f000000e00004
:10197000090032003fb297006121b9000c00be009f
:1019800049060700cfb297006540780090df9f00be
:1019900070012000a0b79f003fb297006121b900fd
:1019a0000c00be00300607000006be00afb2970074
:1019b0000500e90021fc2f008f804000808040005e
:1019c00091b79f00110037003fb197006114b90033
:1019d0000801be000c00be00e60507000005be00c1
:1019e000afb197008301e900a3b79f000801be00d3
:1019f000da050700000056001fb29700cfb297002b
:101a00006552780094b79f000a06be00e00f5600aa
:101a1000e08f5e00030034002fb097000000e0006c
:101a2000e9ff3c004feade00cfa2de000c00be0062
:101a30000401780084017800009fbe000297be0078
:101a400059003700e00f5400e08f5c00e00f5d00ac
:101a5000e08f5d0005003a005e08900081012000e3
:101a6000a1b79f000000e0000d0032003fb19700d9
:101a700002027800cfa2de0005037800860378001a
:101a80000800be000a01be003f0807004fb29700e1
:101a90006440780090df9f0075012000a5b79f008b
:101aa0003fb1970002027800cfa2de000503780064
:101ab000860378000800be000a01be002b0807005c
:101ac000009fbe000297be00afb197000300e9007f
:101ad00024fc2f000f0242000006420024003700c1
:101ae000bfb2970005047800cfc4de000905780076
:101af0008a0578000802be000a03be005fa89700ae
:101b0000efa897007fa997008fb1970022080700e0
:101b1000d0b79f00e1b79f00f2b79f0083bf9f003f
:101b20002fb097000000e900a0b79f000802be0098
:101b30000a03be005fb09700efb097007fb1970037
:101b40008fb997009a0507005faa9700000052001e
:101b5000cfb29700655678005fb09700efb097005e
:101b60007fb197008fb99700009fbe000297be001b
:101b70003e00be002e01be00d0af9f00e1af9f002f
:101b8000f2af9f0083b79f00e00f5000e08f580036
:101b9000e00f5900e08f590003003400afb0970008
:101ba0000100e000ceff3c003fb19700e80f51007c
:101bb00013003a000e1090000038a300100032000d
:101bc000afb19700f78f510006003e0024fc2f00b4
:101bd0000f0242008300420000c3b300914f100087
:101be00007003200afb297008502e900a5b79f0059
:101bf00000c3b30021fc2f008f80400080f07a00ea
:101c0000afb1970078811100120f98006e0090001c
:101c100024fc2f000f0242008300420049fa070013
:101c20001e0990005e089000800f510006003d00e4
:101c300002005000000f98000e1090000040a1001c
:101c4000001798000f0037000000e0000d003d0075
:101c50000e10900074006000f00f500009003a0070
:101c60007e089000fe009000010050008e08900059
:101c700001005000020050004240a9000100340061
:101c8000000f98004f0778004f06be004f05be00ba
:101c90004f04be002f03b100000006008000780052
:101ca000010037000000e8001004e000fdff3a00ea
:101cb00001005000000006008f04b000889fbe00a5
:101cc0008a9fbe008c9fbe008e1f7800f0b79f00d9
:101cd00081f79f005001be004000be00f0979f00ba
:101ce000819f9f00929f9f00a39f9f0010c6b300fb
:101cf0000ff19700804f51001600320010c4b3005e
:101d0000804f510013003200ffb19700530890003c
:101d10000000e00003003d0060002000d0099800b2
:101d20000c0037000000e0000a003a0070c6b30063
:101d30000ff29700804f52000300320070c4b300ce
:101d4000804f520003003a0010002000ffb29700bd
:101d5000d00a9800ffb09700c0fa2f000f00400093
:101d60004602070080017800e20f500015003a009b
:101d700030002000ffb097009008980010c6b30014
:101d80000ff19700804f51000a003200644040007c
:101d9000804f5100070032000040e800804f5100a2
:101da0000400320001d320000040e800804f5100c1
:101db00001003a0041d32000ffb19700630090007a
:101dc000160037000000e00018003400300020004a
:101dd0007fb29700100a980010c6b3008ff29700e8
:101de00080cf52000a0032006440400080cf520091
:101df000070032000040e80080cf520004003200ab
:101e000081d320000040e80080cf520001003a005a
:101e1000c1d320007fb19700620090003158780054
:101e20003158780011487800c601370014c6b30055
:101e30008ff2970084cf52000300320010c4b30029
:101e400080cf520013003a007fb0970060019000ed
:101e50008200780000c3b30080587800ffb297007a
:101e6000e102980080c7b3008ff2970084cf520040
:101e70000100320080c5b300804878000280e8008d
:101e8000ffb09700e0009800710090000080e8002b
:101e9000f00098000300e00005003a00e3979f007f
:101ea00064fb2f000f01420003077800a0013700f8
:101eb00005d42000e5b79f0010c6b3008ff097004f
:101ec00080cf50000500320010c4b30080cf500016
:101ed000a7003a0012d52000e2b79f00ffb197009b
:101ee000530890001e0220000000e00001003500b1
:101ef0000007e8000e02e800d4b79f006022b80097
:101f00006033b8007f9097008f9897001f999700d3
:101f1000af999700a6070700ffb097003102be00f7
:101f20002103be000000e00004003d000400be00ec
:101f30000601be0003f0a200020037000400be004c
:101f40000601be00f0979f00819f9f00929f9f0017
:101f5000a39f9f006f91970064015100e2979f003b
:101f6000c3fa2f008f8141006a8041000048eb00d6
:101f70006b824100c4b79f0031003700c2012000ce
:101f800003002000e5fa2f000f804200e701070060
:101f90007f9497008f9c97001f9d9700af9d97009f
:101fa0000800be000a01be00860707000006be004a
:101fb0005fb1970067015100d2b79f004240a9006e
:101fc0000a003400ab0707000002be000203be0097
:101fd0000800be000a01be00a9070700f0979f0095
:101fe000819f9f00929f9f00a39f9f00cfb197006a
:101ff0006780410071002000050037006f606600b7
:102000004c6add004466de000c067200c4eede00a1
:10201000e00f5600e08f5e00050034008100e9000b
:10202000e18f4000f5ff3a00010037000060eb004f
:102030008100e900fdff3b0067004000c0b79f0042
:10204000dfb297000500e000090034006022b8000c
:102050006033b8007f9097008f9897001f99970082
:10206000af999700880707000000e000c3ff3c001d
:1020700060fb2f008f0040004fb19700010051001e
:102080000000e9008e0f500001003d0000077800bd
:102090000e00e00003003d0073fb2f000f814100a4
:1020a0002c003700800f570005003d000e804000d7
:1020b00010409000f3c0b300e74f500001003c0017
:1020c0008041eb00c4fa2f000f0242000e004200d4
:1020d0006a0040008e007800010037000000e9002f
:1020e0008100e90010417800834f5100fbff32006e
:1020f0000107e800efcf510001003a000248e80074
:102100000100e0000300350075fb2f000f81420045
:10211000060037000e07e8006f909700640040004b
:10212000e0979f0061fb2f000f8140008e0041006f
:102130008e017800030037001100fb006fb297009a
:10214000e44878008301e9008100e9000300e00031
:10215000f9ff3d00ffb29700550890000000e00035
:10216000f3003d000e00e900d00a9800f0003700af
:102170007f9497008f9c97001f9d9700af9d9700bd
:102180006022b8006033b8000800be000a01be003b
:10219000070707000000e00005003d000bf0a2006b
:1021a000f8979f00899f9f009a9f9f00ab9f9f0079
:1021b0006f909700725927000280b900026a2800c8
:1021c00013002000eb030700e4005000e1979f009c
:1021d00015003b00e3801000c0ff2f00008460006a
:1021e0000800ea00e0979f007f9097008f98970083
:1021f0001f999700af99970089ce200007003700fc
:102200000808a300030032003902be002903be0003
:10221000220707000884d100e88444000800e00099
:10222000f7ff3c001b0037000100e0001d003400f8
:10223000c0ff2f0000806000e0979f00000478003e
:102240006000b8000200200003ff230089ce2000b8
:10225000070037000808a300030032003902be005f
:102260002903be000d0707000884d100e88444005c
:102270000800e000f7ff3c000002be000203be00c1
:102280007f9097008f9897001f999700af999700bc
:1022900077070700f0979f00819f9f00929f9f0004
:1022a000a39f9f00ffb097005109900060c6b30044
:1022b0008ff1970080cf51000400320061002000b0
:1022c00060c4b30080cf510002003a006f929700c3
:1022d000ea00420001074100f30f570001003400fb
:1022e0003e01200000c3b300e0779f0075fb2f0084
:1022f0008f824200b5b79f00330037000800be0050
:102300000a01be00af0607000006be0068075700be
:102310004240a9000e003400d60607000002be00ad
:102320000203be000800be000a01be00d40607007a
:102330006022b80046782d0077192400d7060700e0
:10234000f0979f00819f9f00929f9f00a39f9f00f7
:102350003fb0970068044000890020000d0037005e
:10236000a4002000050020000c01be00e0fd2f00ad
:102370000f004000660107007fa897008fb097000c
:102380001fb19700afb1970004c3b30004644100cc
:102390000006be00e00f5600e08f5e00060034002d
:1023a0008904e900e18f4400edff3a0002003700a4
:1023b00000c3b300006478008904e900fcff3b001f
:1023c00068044400b8b79f000e00e0000b00340022
:1023d0007f9497008f9c97001f9d9700af9d97005b
:1023e0006022b8006033b8000800be000a01be00d9
:1023f000a50607000000e000c0ff3c00c5fa2f0062
:102400008f8242006a804200bfb097000080500077
:102410008001e9006f919700e70041006b81420065
:10242000010037000201e80000c3b300924f100022
:10243000fcff320074fb2f000f0042008080400040
:10244000828050000080410002025000e1979f000e
:10245000ffb29700d509900060c6b3008ff29700d5
:1024600080cf52000300320060c4b30080cf52001e
:1024700002003a008100e8000a00370050c6b300ad
:102480008ff0970080cf5000050032008000eb00f5
:1024900050c4b3008ff2970080cf520001003a0081
:1024a00011002000018741008e0f520001003d0005
:1024b000040778000e00e0001d003500840f57006f
:1024c00005003d00e2407f0095c3b30040c3b30068
:1024d00080cf500001003c0005c3b3000e00410056
:1024e0008000e9008e017800010037008100e900da
:1024f0008301e90011427800854f5200fbff320052
:102500000307e80090c3b30080cf520001003a00f7
:102510008448e8000300e00005003d000201e900f6
:102520000e07e8006f9097000000e800e0979f001a
:102530006f9297008e0178008ff097007fb0970020
:10254000100107004f0778004f06be004f05be0080
:102550004f04be008f04b100000006000000e00040
:1025600003003400d8020700e10f400001003a00e8
:102570000000eb00000006000000e0003100320027
:102580008080e90091027800e38f52002d00360030
:102590000508a3002b003a00126d80000200e00045
:1025a00002003200828f50000400310002087800df
:1025b000116d880016003700030178009201900029
:1025c0000300e00002003200818f5100faff390061
:1025d0001202780004004100808f50001900390079
:1025e000810f500003003a00050942008200780084
:1025f000070037000300e0000300320005804000c0
:10260000808f51000f00390093009800110198004d
:10261000110190000200e0000a0032001180400029
:10262000820f500007003a0000da20000008eb009b
:1026300011009000110178009008410010009000f6
:1026400090009800000006000001780000002000c3
:102650000000e00008003200000080000000e00000
:10266000050032000000e900000088000000400082
:102670000100800002b0780000000600889fbe00c4
:10268000800478006684400000ff27001800600086
:102690004401de00f07f2000800f51000e003a0060
:1026a000800ceb00180478006f0064001c003a00f6
:1026b000210090000000e00019003a001100900095
:1026c0000000e00016003a00100020001100e000b9
:1026d00014003200120037000200e00005003c0048
:1026e00001007800db010700000178000000e00035
:1026f00008003c00f00028001800600001fe2300e4
:10270000010c700020c02f00800c41000080eb0005
:1027100004003700800ceb000000eb0001003700e4
:10272000200020004f04be0000000600889fbe006d
:102730008a1f78008c9fbe00000478000206be004d
:10274000e6044000190178000200d0004505de00d3
:102750008a007800f07f2000800f55000c003a00be
:102760006f00610065003a00280090000000e00062
:1027700062003a00180090000000e0005f003a009c
:10278000100020001800e0005d0032005b00370000
:102790000a00e00007003a0008007800ad010700d9
:1027a000800078000000e000020034000a00780099
:1027b000530037006108b9000c0140008d814800ca
:1027c000e07f2000800f5100e08f59000d003400a1
:1027d0001900e00004003d006000b8000200200085
:1027e00003ff2f00030037006000b8000200200044
:1027f00003ff2700009cbe000294be0010002000d2
:102800003f003700e00f5100e08f59000500340011
:10281000f000280019006000c410dd00810c700079
:10282000340037001900780001002800010360001f
:102830006f0060000040a000800c78006101510032
:10284000e0815900c0fc2f00f1ff2f00800f5100e4
:10285000818f59000d003d00860c78000000eb00d0
:102860002004980010049800000c78002400370021
:102870008880e800110c780064004400900878001b
:1028800019087800800ceb0070014100f00f410046
:10289000f7ff34008202ea00150032008881e80068
:1028a00070821200980078008508de00130078001e
:1028b0000400dd00008c7000640144009300780087
:1028c0008508de00120078000400dd0080897000b9
:1028d000920078008508de00190078000400dd0011
:1028e00000897000190078000500de00800c780077
:1028f000990c73000080eb000100370020002000dd
:102900004f06be004f0578004f04be0000000600d1
:102910000400fa00889fbe008a9fbe008c1f7800ca
:102920000006780092bf9f00a3bf9f000404be0072
:102930000401be001fb89700afb897000d02070052
:102940000005be000001be000800be000302070033
:102950001fb99700afb9970000005100818059005e
:1029600020069800310698000a8ebe000c00780000
:102970004f0678004f05be004f04be000080fa00ed
:10298000000006000e00fa00889fbe008a9fbe006d
:102990008c9fbe0000047800014578000206780094
:1029a00083047800840678000300e00002003c0005
:1029b000190020008cda200060c6b300804f55005b
:1029c0000e00320060c4b300804f55000b0032008f
:1029d00070c6b300804f55000300320070c4b300ce
:1029e000804f55009c003a00e48f4600800035007f
:1029f00058089000808f56007d003d008d05e8004e
:102a000060c6b300804f55001000320060c4b300b0
:102a1000804f55000d003200081090000038a300d0
:102a200004003a0058089000808f540001003d00d7
:102a3000590c9800580890000b005000500c98005a
:102a400002003b000000eb00500c98000b00e0007f
:102a500027003c00180990006800900001c3b300f3
:102a6000017079008201e800130c9800580890006a
:102a70000000e00003003c00081090000038a300b4
:102a80000500320068009000e1c2b30001f0790057
:102a90000280e800100c9800d80890000b00ea00b3
:102aa000808f500001003d008105ea000b00ea0024
:102ab000200c980001804500500c9800890f5000b0
:102ac00001003d0080047800390c980068009000f7
:102ad0009808900001004000090178008c007800ff
:102ae00098f6070058089000090050001a003700b7
:102af00098089000680090008b8f540018003d00eb
:102b000001004000090178008c0078008df6070074
:102b10001808900000814400120c980009805500ac
:102b2000200c9800580890000000e00003003c00d2
:102b3000081090000038a30006003200e800900062
:102b4000e0c2b30080707900380890000000e8000f
:102b5000300c980058089000400c9800a6003700f0
:102b6000010040000b0178008c00780075f607002a
:102b70001808900000814500120c98008b845400c6
:102b8000580890000000e00003003c00081090008e
:102b90000038a3000500320068009000e1c2b300d5
:102ba000017079000200e800100c980058089000ad
:102bb000890f500001003d008004780068009000fb
:102bc00098089000010040008b0046000901780041
:102bd0005cf607001808900000804400100c980074
:102be0005808900009005000200c9800820037001f
:102bf00070c6b300804f55000300320070c4b300ac
:102c0000804f550014003a0058089000808f5400ff
:102c100004003d00081090000038a30001003a00b5
:102c2000590c9800580890000000e900500c9800da
:102c300002003b000000eb00500c980070c6b3008f
:102c4000804f550002003a005ac6b3000b0037000f
:102c50005ac4b3000900370010c6b300804f5500b6
:102c600002003a000ac7b3000400370010c4b300e2
:102c7000804f550001003a000ac5b30018099000c2
:102c8000680090003c7079008201e800130c980005
:102c90000c027800580890000000e00003003c009f
:102ca000081090000038a30017003200e8009000e0
:102cb000e0c2b30080f079008280e800110c980037
:102cc000580890000000e0000f0034008904e9007b
:102cd000890f500001003d008004780068009000da
:102ce00000804000090178008400780015f6070094
:102cf0001808900000804400100c980058089000bc
:102d000009005000200c980068009000980890007e
:102d1000010040000086e8000a5878008000780032
:102d20000d00e00004003500b0c2b3008048780018
:102d30008c04780004003700d0c2b30080487800cb
:102d40008c0478008d06ea008005eb000a0037004d
:102d5000a20020008d0078007080570089000700d5
:102d60000fb897009fb897007a81550001f17f0056
:102d70008b05e800800678000d00e000f4ff3c00c1
:102d8000e18f550009003c0050c6b300804f55004c
:102d90000300320050c4b300804f550003003a00d6
:102da00000c3b300005e78008c0478000b00e000e4
:102db000040032000b00e900fa8057000080400058
:102dc0000600370000c3b300805c780005003700c0
:102dd0008b05e90002c3b300a05c41000b00e000da
:102de000fbff3c0068009000980890000100400044
:102df00000805400300c98000810900074006000af
:102e0000f00f50000e003a007800900098089000f3
:102e100001004000a808900001004000b8089000a0
:102e200001004000c8089000810040007808900030
:102e3000808f500002003d0001005000000c9800ff
:102e40004f06be004f05be004f04be000080fa00d2
:102e50000000060000027800e6024000150078003d
:102e600001002800810360006f006000800a780084
:102e700012003a00240090000000e0000f003a0029
:102e8000140090000000e0000c003a001600200042
:102e90001400e0003800320008003700e40042006f
:102ea000910a78000480e8009008780014087800ff
:102eb000000aeb00700353000100370016002000e9
:102ec0001500e000f5ff32001300370064014200f6
:102ed00080004000120078004f00de00808a700001
:102ee0008481e8009200780081804000130078001f
:102ef0004f00de0000897000930078008180400060
:102f0000140078004f00de00808970001400780003
:102f1000000a40000603e90015007800ef0f50009a
:102f2000eaff3600100037000481e8009400d10069
:102f3000120078004f00dd00008a7000e4004200bb
:102f40009201d100110078004f00dd00008971006e
:102f50001101d100150078004f00dd0080087100dc
:102f6000950ad1000603e80015007800ff0f500015
:102f7000edff3e00ef0a6000958a730006007800be
:102f80000000060002027800809fbe0011000900c8
:102f90008200d800000178004f00be0002a2b900f4
:102fa000848050001100980002087800000006009c
:102fb0000a00fa0080017800e20f500025003e0070
:102fc000606d8000e10f500008003200e021200019
:102fd0000000e0000500320064212000852120006f
:102fe000a62120008001780004003700c4202000c2
:102ff000e5202000062120004321200014409000fd
:103000000004e000030035008009eb000000280008
:10301000140a7000154090000028a30001003a0037
:1030200015a0a0008001eb000700370015409000bc
:103030000008a300fdff320063c078000000fb0021
:10304000000b78008301e800828f5100f7ff3a00ff
:103050000800370030002000b0bf9f00c3bf9f00b2
:10306000d1bf9f00e2bf9f006a80570000c0da0016
:103070006fb99700020078000080fa000000060097
:103080000a00fa0011002000b1bf9f00c0bf9f00de
:103090006a80570000c0da004fb897000080fa003d
:1030a000000006000a00fa0051002000b1bf9f0096
:1030b000c0bf9f006a80570000c0da005fb8970069
:1030c0000080fa0000000600889fbe00800478009f
:1030d000706d80000000e00003003a00100007005f
:1030e0000000e0000a003500706d80000900e0007b
:1030f00002003a000004780006003700000478005f
:1031000009004000060007000000e00001003d004b
:103110000084eb00080078004f04be0000000600a9
:10312000800078000000e00004003a0000db20008e
:10313000706d880001017800060037000081eb0007
:1031400080192100808f500002003e00716d8800c0
:103150000001eb000200780000000600020ab9003e
:10316000001bb9000200b80081004200810043004a
:1031700000000600839f68000100e00002003d009f
:1031800060001000e08018000300e00002003d0035
:1031900060011100e0811900330007004f00e000da
:1031a00002003b0060001000e080180000000600f4
:1031b000889fbe008a9fbe008c1f78000205be005b
:1031c0000004be000006eb00e00f5000e08f580046
:1031d000e00f5900e08f590007003d006000b80083
:1031e0006011b80008045000898458000a0559008d
:1031f0008b8559001c002000e00f5200e08f5a0020
:10320000e00f5b00e08f5b0002003d000f00070055
:103210000c00a2000800be000a01be004501070024
:103220000203be000002be000c00e00001003200fc
:10323000060007000400be000601be004f0678002d
:103240004f05be004f04be00000006006000b8003d
:103250006011b8000402500085825800060359002e
:1032600087835900000006006022b8000602200093
:103270000000d0008180d2000482d2008582d2007a
:103280000000a0000202520083825a0003003100b5
:103290000202420083824a000000a1000603e90006
:1032a000f3ff3a0000000600efff07000400be0035
:1032b00000000600889fbe008a9fbe0001057800be
:1032c0000100e0000400350008003c000000e000c0
:1032d000200032000500370060001000e080180078
:1032e00002003b0001f02c001a0037000004be0071
:1032f0006011b8006b0920000982cf00020039007c
:103300000882cf000441b000694252000e00320032
:1033100008003b0082817100610164008904d100d2
:103320000884d3008b05e8000442e800f9ff3a0066
:10333000050037000804440089844c008b05e9002f
:103340000442e900fbff3a001c0107000af0a70055
:1033500001f0a0004f05be004f04be0000000600b3
:10336000889fbe008a9fbe008c1f7800390107002d
:103370004001330003866c006450e1002e003200ef
:103380006420e100330032006150e1002f00320080
:103390006120e1003100320085855500eb07b00067
:1033a000090020000804200005003700080444003c
:1033b00089844c000a0031000603430087834b00d8
:1033c0000001530081815b00f8ff33000203be005f
:1033d0000800a0000804440089844c00f6ff39006e
:1033e000c639dd00830173000100320013002000a4
:1033f0008904d1000884d3000998a3000500320095
:103400000800a7000300a0008904d1000884d300ad
:103410008b05e8008904d1000884d3000001eb008b
:103420000281d200e500070001f0a1000cf0a70026
:1034300001f0a000180137006420e1001a013200f9
:103440000801be000200be00f7ff37006120e10066
:10345000150132006000b800f3ff370000002000c3
:1034600001f82700f0ff370003f0a200889fbe009c
:103470008a9fbe008c1f7800f6000700fd00330015
:103480006450e1004f0032006420e100520032003d
:1034900003826c0007003b000905d0000306d00042
:1034a000820f54000c065d00020039000200320059
:1034b00089017800030678008582550004003d00ec
:1034c0000003fd008103fd008502ea008b854200b8
:1034d000840f720002003b0060001000e0801800c2
:1034e0006011b8000005eb007a28e1000a003900fd
:1034f00006007800c75ddd00f707b2008780750021
:103500002d003700828171000a017800610560009a
:103510008180d1000080d3008502e900f9ff3b00e3
:10352000060440008784480002003b006004140049
:10353000e0841c000988a300070032008a81710022
:1035400082817100610164008904d1000884d30084
:103550008b05e800170037000978a30013003a0034
:103560000b00e000130034008b05e9000804440060
:1035700089844c000a4474000978a3000d003a00c5
:103580000b00e000070034008b05e900080444004c
:1035900089844c0001003a000b0020000978a30048
:1035a000f7ff32000001eb0002003700828171005a
:1035b0000a017800810007000cf0a70001f0a000cc
:1035c000b50037006420e10002003a00838f6c00f0
:1035d000b50033000801be000200be00ae00370097
:1035e000889fbe008a9fbe008c1f7800990007004c
:1035f000a000330003866c006450e1002400320018
:103600006420e100270032006150e1002200320016
:103610006120e100210032008b854200eb07b10000
:103620000134b800003ab8000804420089844a0016
:10363000013ab8000030b8008880400009014a0013
:10364000040033000000400081804800020149006e
:103650008b05e900c909dd0083017000010032001b
:1036600013002000c814de004814dd004709de0006
:103670001200b200c808de00088470004f00070086
:1036800001f0a1000cf0a70001f0a00082003700bb
:103690006120e100840032000801be000200be008b
:1036a000f7ff37006150e100fcff3a007e00370071
:1036b0000001be007f0007000470a70003f0a10016
:1036c0006509b100160032000d0035006828e100e0
:1036d00006003500f0ff2f00f1ff27000300e00097
:1036e00013003b000100280000000500000040001e
:1036f000818048008502e900fcff3a00080037009d
:10370000f88f420002003c008000eb000000050042
:103710008100d1000080d3008502e800fcff3a0060
:103720000300e00002003b0060001000e080180091
:1037300000000600889fbe008a9fbe008c9fbe00ce
:103740000404b8000506b8008904460060854e00f0
:103750000606b8000a054600e0854e000706b800d8
:103760008b054600040eb800890446000a854e0009
:10377000e0854d00050eb8000a0546008b854e0019
:10378000060eb8008b0546000416b8000a05460070
:103790008b854e000516b8008b054600041eb80048
:1037a0008b0546000800be000a01be004f06be00a1
:1037b0004f05be004f04be0000000600810020003f
:1037c000618055000b003d000b00200061fe2f00c2
:1037d0000100e1001d00340082817100610164007c
:1037e0008904d1000884d3000000e800faff3a0001
:1037f000710020006100640003007000020060009e
:103800000900320061044400e0844c000988a500ee
:10381000050032008b05e8006808e10002003a006c
:103820008904d1000884d300f20f20000258e1007f
:1038300005003d00c75ddd00f907b2008980750015
:1038400008007800000006000bf827008b007800c5
:10385000000005000004be00160007000003be00c3
:103860000405be000200be0012000700844f750070
:10387000000006000200be006450e10005003600b2
:103880006420e100020036000968a30001003a004c
:103890000800be000160a0004f0678004f05be0082
:1038a0004f04be0000000600f0ff2f00f1ff2700cc
:1038b000f9ff3700c70ade00f107b200f50fb200ca
:1038c00008003200e1cf4200020032000170a00087
:1038d00024000500810f700001003200040805007b
:1038e00044000500810f700002003a00140005003a
:1038f0008502e9000000400081c04800fcff3b0059
:103900000170a0002400050081037800e9ff070092
:103910000001be006000b8000478a30013003a0064
:103920006220e10015003e000d0039008301d10046
:103930000281d3008180d3008301d1000281d300b2
:103940008180d3008301d1000281d3008180d30024
:103950000538b000c42add00f300b2008381720094
:1039600007f0a70003f0a00000000600f3ff270007
:10397000f2ff2f006110b900fbff370003ff2700a3
:10398000f7ff3700881f7800000478005001be0060
:103990004000be0004004000858048000601490048
:1039a00087814900009cbe000294be000400e10033
:1039b0000588e1000690e1000798e100020031006f
:1039c000680044001008e8004f047800000006007a
:1039d000f4874700889fbe008a9fbe008c9fbe0070
:1039e0008e1f78000205be000004be00d4b79f0001
:1039f000e5b79f00f6b79f0087bf9f000000eb0070
:103a0000c0b79f00b0b79f00a0b79f0090b79f00be
:103a100080b79f000d042000bfb097004fb0970003
:103a2000000140000000e0000f003d004f08de00f4
:103a300000007100c0b79f009e00070001003d001c
:103a400012002000a100070001003d00120020002c
:103a5000a6000700b1000700b60007000f004000f5
:103a6000c8ff0700220037004f08de000006710083
:103a7000ccb79f008f00070001003d00120020001e
:103a80009200070001003d0012002000970007008f
:103a9000a20007000fb297009fb297002fb39700c4
:103aa000bfb39700a90007000000520081805a00b0
:103ab00002015b0083815b0080b79f0091b79f008c
:103ac000a2b79f00b3b79f000007eb009f0007005d
:103ad0000020e10001a8e10002b0e10003b8e1002c
:103ae000010031001e0020000e005600c0b79f00ec
:103af0004fb297000400e0000700350010002000de
:103b0000010020006011b800080470008984700072
:103b10000a0571008b8571008d06e900beff3a0031
:103b20000400e00003003d00820007000f00400099
:103b300094ff07004fa897000000e00004003a003f
:103b40000fb497009fb497002fb59700bfb59700ab
:103b5000940007004f0778004f06be004f05be00d7
:103b60004f04be004f01b10000000600881f78001e
:103b700018002000881f780095ff07008f87e90054
:103b80004f04780000000600801feb0090ff070044
:103b90008f87e90000000600889fbe008a9fbe0054
:103ba0008c1f78006e00070007003d0073000700bf
:103bb000e00f5b00e08f5b0007003d003200070074
:103bc0000006eb00040037003400070002003d004f
:103bd0002a0007001c00200072000700e3ff070016
:103be0000203be000002be000c00e0000100320033
:103bf000220007000400be000601be004f06780048
:103c00004f05be004f04be0000000600889fbe00a6
:103c10008a9fbe008c1f78005100070005003d0000
:103c200056000700e00f5b00e08f5b0006003d00e0
:103c3000040037001900070003003d006000b800d1
:103c40006011b8001000070056000700ceff070003
:103c50000203be000002be000c00e00001003200c2
:103c6000060007000400be000601be004f067800f3
:103c70004f05be004f04be00000006006000b80003
:103c80006011b8000000370004025000858258001f
:103c90000603590087835900000006000006eb0068
:103ca000e00f5200e08f5a00e00f5b00e08f5b00f6
:103cb000000006000180400090b79f000001eb006b
:103cc0008fb097000100e0000000060002007000c5
:103cd00090b79f000180400080b79f000001eb007b
:103ce000ffa897000100e00000000600020070003d
:103cf00080b79f00018040006faa9700cf20de00b0
:103d000001007000f0af9f00040242002500070090
:103d10004f18de000002720000000600e4af9f00b2
:103d20000804440089844c000a054d008b854d0031
:103d3000000006003fb29700cfb297005fb3970034
:103d4000efb3970000fe2f00000006003fb0970081
:103d5000cfb097005fb19700efb197000000060069
:103d60000205be000004be00e00f5000e08f5800c6
:103d7000e00f5900e08f5900000006006000b80015
:103d80006011b80008045000898458000a055900e1
:103d90008b8559001c002000e00f5200e08f5a0074
:103da000000006000800be000a01be000000060078
:103db0008f1fd100080107008f87e9000000e00095
:103dc000000006001400fa00889fbe008a9fbe0013
:103dd0008c9fbe000004be000205be0068004700c4
:103de0000a90be000890be00240107000070a700e2
:103df0000bf0a100304320009e0290008082520010
:103e0000b0fe2f000028e10011003d00b0fc2f00a3
:103e10000028e100150034001e0990008e08900073
:103e20007e0090000501b0000201d1008180d30026
:103e30000080d3008502e800fbff3a000b00e000a1
:103e400049013b0060001000e08018004601370087
:103e5000f0ff2f00f1ff27000b00e00042013b00c4
:103e600001002800000020003f0137006000b8007a
:103e70003d0137004f89de00820178003f013700a5
:103e800007f0a20074013700809feb00d20007000a
:103e90008f87e9000000e000000006002800fa001b
:103ea000889fbe008a9fbe008c9fbe0003866b0069
:103eb000190107000028a30064003a000128a300ac
:103ec00067003a000008a30062003a000108a3005e
:103ed00065003a001e009000be0890008106400078
:103ee000ed3fb100f4805700ee019000111ab800c8
:103ef0008e099000311bb8009e099000311cb8005b
:103f0000511db800f485570046000700fe019000df
:103f10003a0007008b85e8003e0007008e099000fc
:103f200040000700ee019000340007008b85e80098
:103f3000380007008e099000400007009e0990009d
:103f40001b18b800890440000a854800fe01900053
:103f5000340007008b85e80038000700ee01900070
:103f6000300007008e0990001b18b800890440003b
:103f70000a8548000a98a30008003a00040242009b
:103f800085824a0006034b0087834b0008044c00df
:103f900089844c000a054d008d06e9008482720078
:103fa000850273004c3add00850272000100320088
:103fb00015002000443ade001400b2004538de004f
:103fc000cb45dd000b007000c540de00cb4ddd00b1
:103fd0008b8070004549de00cb55dd000b01710080
:103fe000c551de000d0378009801070003f0a10021
:103ff0000cf0a70003f0a000db0037001b18b8008e
:104000008502400006834800e0834b0060044c00ba
:10401000070037001b18b8000603400087834800dc
:10402000faff37001b18b8008703400008844800d7
:10403000e0844c0060054d00000006001b18b8002d
:104040000804400089844800faff37000108a300f3
:10405000c2003a005800be005801be00e3ff37001e
:104060000008a300bd003a0009047800f9ff3700fa
:104070002800fa00889fbe008a9fbe008c9fbe0069
:1040800003866b00a40007006400e10044003200d6
:104090006408e1004a0032006100e100460032009d
:1040a0006108e10049003200ec0647006000b800fa
:1040b0003d02be003d03be00f48657006011b8000b
:1040c0003d04be003d05be007d0320000b0037000f
:1040d0000000a0008d06e900130032000402420037
:1040e00085824a0006034b0087834b000000400096
:1040f0008180480002014900838149000802520082
:1041000089825a000a035b008b835b00f0ff3b004f
:104110000802420089824a000a034b008b834b004d
:104120008d06e900edff3a008482720086827200fb
:10413000f707b200878272000100320015002000ec
:104140001e0490003e0b900006035400e63fb000b2
:104150000368a300070032000000a7000500a000cc
:104160008301d1000281d3008180d3000080d3007d
:104170000603e8008301d1000281d3008180d300cf
:104180000080d3000002eb000482d2002f01070060
:1041900003f0a1000cf0a70003f0a00072003700ac
:1041a000640247006408e1006c0032003400be0085
:1041b0003401be00f6ff37006108e10067003200fd
:1041c0006011b8006000b800f1ff370003ff27005e
:1041d00002002000fbff3700889fbe008a9fbe00c0
:1041e0008c9fbe000404be000605be00809fbe007a
:1041f000829fbe0041010700040678000800be004f
:104200000a01be003d010700840678004f03be008e
:104210004f02be008d4f76007fb097001300330031
:10422000f0ff2f008b8f6b0006003b000d06660031
:104230000c00a7000a00370007f0a60010002000bd
:104240000a003700880f5200898f5a008a0f5b00de
:104250008b8f5b00030039001000200001003e003e
:104260000000200007f0a7000000ea004f06be0093
:104270004f05be004f04be0000000600800078001d
:104280005002be005003be004439de00f700b20009
:10429000f37f200003016100090032000218e100f1
:1042a00016003a0085017200830173008381730058
:1042b0000008200015003a004000200013003700dd
:1042c00085017200830173008381730005003a0049
:1042d00004a8be0006a8be00100020000b00370096
:1042e0000201e9000402420085824a0006034b00f5
:1042f00087834b000748a300f9ff32000740a00066
:1043000004a8be0006a8be0020002000800098007f
:104310009200980000000600680447000294be0066
:104320000094be00fc0447008694be008494be0046
:1043300009007800d1ff070008007800cfff0700d0
:1043400099007800814f70000b003b000800be0010
:10435000fc0007004f00b10003003700f3ff270007
:10436000f2ff2f006110b9004f06be004f05be00de
:104370004f04be000080fa0000000600889fbe00c7
:10438000830478000300e0002c00350003003c00ab
:1043900000827000040271002600320036432000c3
:1043a000c50020008383cf000a0039000541b10019
:1043b0008283cf00070039000541b1008183cf001f
:1043c000040039000541b1008083cf0001003900ad
:1043d0000541b10085c353006022b80012003200cd
:1043e0000a003b0084827200610260008301d100f8
:1043f0000281d3008180d3000080d3000603e8004f
:104400008743e800f7ff3a0007003700000040004c
:104410008180480002014900838149000603e900c8
:104420008743e900f9ff3a008800070009f0a70078
:1044300003f0a0004f04be00000006006000100062
:10444000e080180060011900e0811900d3ff3b00f3
:10445000033e2c00f7ff37002800fa00889fbe00bb
:104460008a9fbe008c9fbe00070678008786690081
:104470000c003b00030478008704780008f0a100da
:1044800009f0a100840f5000858f5800860f590055
:10449000890f5c00030033000cf0a20001003a0019
:1044a0000cf0a1009cff07006400e1005f003200f7
:1044b000780147006408e100610032006c014700a8
:1044c000748557003200be001201be003a04be00df
:1044d0001a05be001e039000be0a9000850353001b
:1044e00006003d000004fd008104fd000205fd0002
:1044f0008305fd008703ea00050378000df8a3009b
:104500000400320060041400e0841c0060051d00fb
:10451000e0851d006022b8007d0320000d38e10019
:104520008006eb000b0039004433dd00f300b200dd
:104530008301730039003700848272000d02780015
:10454000e10664008b85d1000a85d3008984d300fd
:104550000884d3008703e900f7ff3b000800400010
:10456000898048000a0149008b81490004003b0012
:1045700060001000e080180060011900e08119005f
:104580000358a300090032008d82720084827200f9
:10459000610260008301d1000281d3008180d300d9
:1045a0000080d3000603e8001b0037000348a30087
:1045b00017003a000600e000170034000603e90087
:1045c0000d00a3000000480081804800020149005e
:1045d000838149000348a3000f003a000600e00071
:1045e000090034000603e900000040008180480013
:1045f000020149008381490001003a000003eb00f9
:104600000348a300f5ff32006022b8000200370023
:1046100084827200618266000c00070003f0a10032
:104620000cf0a70003f0a0004fff37006401470023
:104630006408e10002003a000df8a30047ff3a00c9
:104640003200be001201be0047ff370018002000f4
:1046500057002000080453000d003d000600200014
:1046600097fc2f000740e1001e0034008482720096
:10467000610260008301d1000281d3008180d300f8
:104680000080d3000804e800f8ff3a00470020004b
:104690006104600005047400040464000d0032002d
:1046a00061004000e080480060014900e08149006d
:1046b00003b8a500070032000603e8006538e100f2
:1046c00004003a008301d1000281d3008180d3002d
:1046d0000080d300f87f20000830e100030035009f
:1046e000080378006000b8006011b8004433dd00b2
:1046f000f300b200830173000000060005ff2700ed
:1047000005826100070032000428e1000100320048
:10471000240005000600070001003a0044000500df
:104720000408050002000700f9ff3a001400050024
:104730006f82610081027000850271008502720043
:1047400000000600e48240001078a3000700320059
:10475000640240001178a3003400be001401be00c2
:10476000040032000330a700000006003500be0040
:0c4770001501be000330a0000000060090
:020000040000fa
:0200000401f009
:04000000ebfb000016
:020000040000fa
:0200000401f009
:04000400ff7f00007a
:020000040000fa
:0200000401f009
:04000800efff000006
:020000040000fa
:0200000401f009
:04000c00ffff0000f2
:020000040000fa
:0200000401f009
:04001000ffff0000ee
:020000040000fa
:0200000401f009
:04001400ffff0000ea
:020000040000fa
:10000800466f0000be6d0000fc6d0000fa6e000037
:10001800286f0000466f0000466f0000466f000022
:10002800466f0000466f0000466f0000046600003f
:10003800466f0000466f0000466f000050670000e2
:1000480026770000d46b0000466f0000466f000062
:10005800466f0000466f0000466f0000466f0000c4
:10006800466f0000466f0000466f0000466f0000b4
:10007800466f0000466f0000466f0000466f0000a4
:10008800da740000466f0000466f0000466f0000fb
:10009800466f0000466f0000466f0000466f000084
:1000a800466f0000466f0000466f0000466f000074
:1000b800fa72000080720000466f0000466f000070
:1000c800466f0000466f0000466f0000466f000054
:1000d800466f0000466f0000466f0000466f000044
:1000e800466f0000466f0000466f0000466f000034
:0800f800466f0000466f000096
:020000040000fa
:10010800466f0000be6d0000fc6d0000fa6e000036
:10011800286f0000466f0000466f0000466f000021
:10012800466f0000466f0000466f0000046600003e
:10013800466f0000466f0000466f000050670000e1
:1001480026770000d46b0000466f0000466f000061
:10015800466f0000466f0000466f0000466f0000c3
:10016800466f0000466f0000466f0000466f0000b3
:10017800466f0000466f0000466f0000466f0000a3
:10018800da740000466f0000466f0000466f0000fa
:10019800466f0000466f0000466f0000466f000083
:1001a800466f0000466f0000466f0000466f000073
:1001b800fa72000080720000466f0000466f00006f
:1001c800466f0000466f0000466f0000466f000053
:1001d800466f0000466f0000466f0000466f000043
:1001e800466f0000466f0000466f0000466f000033
:0801f800466f0000466f000095
:020000040000fa
:10477c0020760000312e000030380000003100009f
:10478c00372e0000303300002e3200003031000094
:10479c003500000001000000000000006400000073
:1047ac0000000000e80300000000000010270000db
:1047bc0000000000a0860000010000004042000044
:1047cc000f0000003000000000000000dd010000c0
:1047dc0000000000a4120000000000006aba0000f3
:1047ec000000000023480000070000005ad1000020
:1047fc00480000000e740000da0000001be8000006
:10480c00b4010000832d0000d8020000065b0000fc
:10481c00b00500000bb60000600b0000176c000028
:10482c00c1160000abaa0000aa2a00000e740000fa
:10483c00da0000001be80000b4010000832d00002a
:10484c00d8020000065b0000b00500000bb60000ab
:10485c00600b0000176c0000c11600002222000043
:10486c0022220000abaa0000aa2a0000b6600000b9
:10487c000b360000c11600006c4100004a9f00007e
:10488c00f4490000000000000001000000020000dc
:10489c0000030000000400000005000000060000fa
:1048ac0000060000000700000007000000070000e1
:1048bc0000070000313200003030000020200000e2
:1048cc0000000000323400003030000020200000d6
:1048dc0000000000343800003030000020200000c0
:1048ec0000000000393600003030000020200000ad
:1048fc000000000031390000323000003020000090
:10490c00000000003338000034300000302000007c
:10491c000000000035370000363000003020000069
:10492c000000000031310000353200003030000052
:10493c00200000003a0000002100000012000000de
:10494c00960000003a000000210000000a0d000053
:10495c00576f000072640000732000003d200000bf
:10496c00256400002c2000005375000063650000d6
:10497c0073730000203d000020250000642c000013
:10498c002043000068650000636b00007375000035
:10499c006d2000003d20000025580000000a00009a
:1049ac000d5700006f72000064730000203d000082
:1049bc0020250000642c00002053000075630000cb
:1049cc006365000073730000203d0000202500008b
:1049dc00642c00002043000068650000636b00003d
:1049ec00737500006d2000003d200000255800006c
:1049fc0000500000575200000050000057520000b9
:104a0c00202d00002e2d000057000000494400000e
:104a1c000041000000490000442000002d2e000041
:104a2c002d2d0000410000005246000020500000d7
:104a3c006f77000065720000203d00002000000030
:104a4c00206400004200000050770000722000003b
:104a5c004f460000462000006166000074650000af
:104a6c007220000025690000202000000056000084
:104a7c00464f0000206c00006f6300006b200000ac
:104a8c002020000020200000204f00004e000000dd
:104a9c00564600004f2000006c6f0000636b000056
:104aac002020000020200000204f0000464600007f
:104abc00000a00000d550000736500007220000014
:104acc007365000074740000696e00006773000069
:104adc002073000061760000656400002074000003
:104aec006f20000045450000505200004f4d000063
:104afc002c200000506f0000776500007220000031
:104b0c006f660000660a00000d00000052530000a2
:104b1c003233000032200000546500007374000032
:104b2c002020000020200000202000000057000062
:104b3c0061690000746900006e6700002064000069
:104b4c0061740000612e00002e2e00002e0000006b
:104b5c0052580000206400006174000061200000c5
:104b6c00200000002020000030780000004a0000e7
:104b7c00554d0000412000005452000058320000f6
:104b8c0020000000202000004f480000324e0000a2
:104b9c004c540000204f00004837000053560000d2
:104bac0020200000000a00000d0a00000d4a000041
:104bbc00554d0000412000005452000058320000b6
:104bcc0020460000697200006d77000061720000e1
:104bdc0065200000002c00002042000075690000d8
:104bec006c640000200000000a0d0000436f000000
:104bfc007079000072690000676800007420000082
:104c0c004a75000068610000204e000069690000d0
:104c1c006e6900006b6f0000736b0000692c000064
:104c2c00204f0000483200004e4c0000540a000097
:104c3c000d0a00000d000000537900007374000091
:104c4c00656d0000204300006c6f0000636b00007a
:104c5c00203d000020250000692000006b4800006a
:104c6c007a0a00000d0000004a5500004d4100007a
:104c7c002054000052580000322000005541000022
:104c8c005254000032200000666900007865000074
:104c9c006420000039360000303000002062000033
:104cac00640a00000d000000506f000077650000e2
:104cbc00722000004f4e000000530000657200008f
:104ccc007669000063650000204d00006f640000f1
:104cdc00652000002020000020000000507500001e
:104cec00736800002044000049530000504c000041
:104cfc0041590000206e0000787400000050000044
:104d0c0075730000682000004641000053540000f9
:104d1c00203d00002053000061760000650000007b
:104d2c000a0d000045450000505200004f4d000098
:104d3c002063000068650000636b00007375000061
:104d4c006d7300002c200000436100006c200000fb
:104d5c003d200000255800002c2000004465000078
:104d6c006620000043730000203d00002025000059
:104d7c00582c00002046000061630000746f000096
:104d8c007279000020640000656600006175000007
:104d9c006c740000207200006573000065740000e4
:104dac00732000003d20000025640000000a000074
:104dbc000d45000045500000524f00004d200000f2
:104dcc0063680000656300006b730000756d000084
:104ddc0020650000727200006f7200002c20000031
:104dec00726500006c6f00006164000020660000ba
:104dfc0061630000746f0000727900002064000091
:104e0c0065660000617500006c74000073000000a2
:104e1c0050750000736800002053000045540000da
:104e2c00206600006f72000020200000202000008f
:104e3c000066000061630000746f0000727900006e
:104e4c002064000065660000617500006c74000051
:104e5c00730000000a0d0000536500007420000070
:104e6c0055410000525400003120000075730000c1
:104e7c006572000020620000617500006420000073
:104e8c007261000074650000207400006f20000047
:104e9c0023250000692c0000202000002573000051
:104eac00626400000a0d0000000a00000d530000af
:104ebc006574000020550000415200005420000091
:104ecc0075730000657200002062000061750000bf
:104edc006420000072610000746500002074000002
:104eec006f20000023250000692c0000202000000a
:104efc0025730000626400000a0d000000560000db
:104f0c00464f0000412000003d3e000020560000ae
:104f1c00464f0000422000006f6b00002000000094
:104f2c00564600004f420000203d00003e2000008d
:104f3c00564600004f410000206f00006b2000001f
:104f4c0000200000564600004f000000202000000a
:104f5c00004c00005342000000550000534200007a
:104f6c00002000004357000000540000756e000044
:104f7c0065000000202000005458000000200000b4
:104f8c004e41000052000000204d0000494400003a
:104f9c000020000057490000440000005357000057
:104fac0052000000204e00002f41000020000000a5
:104fbc0053570000522000002d2e00002d2d000014
:104fcc00002000000056000000230000256c0000ab
:104fdc005800000020520000002000005800000083
:104fec0020530000706c000074000000205300007f
:104ffc0000200000460000002056000000200000a9
:10500c00202000004c6f0000636b000000200000ab
:10501c00416400006a7500007374000000410000d8
:10502c0047430000203d0000204600006173000053
:10503c007420000020200000202000002000000030
:10504c0041470000432000003d200000536c00004d
:10505c006f7700002020000020200000202000009e
:10506c00004e000041520000004d00004944000079
:10507c000057000049440000002000004c50000084
:10508c004620000020000000256c00006920000074
:10509c00487a0000202000000053000070650000da
:1050ac006563000068500000726f00006320000010
:1050bc003d2000004f4e0000200000005370000007
:1050cc006565000063680000507200006f630000ab
:1050dc00203d0000204f000046460000004100002b
:1050ec0046200000696e0000203d0000204c0000ae
:1050fc00696e0000652000002020000020000000e8
:10510c0041460000206900006e2000003d20000098
:10511c004d690000632000002020000020200000ca
:10512c00004b00006579000065720000203d000016
:10513c0020000000446f000074200000707200001a
:10514c00692e000000490000616d000062690000da
:10515c006320000041000000496100006d62000006
:10516c0069630000204200000053000074720000cc
:10517c00616900006768000074000000435700007c
:10518c002070000069740000636800002025000096
:10519c0069200000487a0000202000000043000035
:1051ac0057200000706f0000742000003d200000ac
:1051bc0053710000756500006c630000680000000e
:1051cc0043570000207000006f740000203d000069
:1051dc0020430000577300007065000065640000f8
:1051ec00004c000043440000204200004c20000012
:1051fc003d20000025690000202000002020000038
:10520c0020200000004300006f6e0000747200004c
:10521c0061730000742000003d200000256900002f
:10522c0020200000004c00004344000020540000eb
:10523c00696d000065720000204f000046460000ba
:10524c0020200000200000004c43000044200000ff
:10525c00546900006d650000722000002569000093
:10526c00207300002020000020000000525300009a
:10527c0032330000322000003d200000004a0000c4
:10528c00554d0000415400005258000032000000ff
:10529c005961000065730000754300004154000023
:1052ac00005600006f690000636500004d6500004a
:1052bc006d00000054650000737400002020000095
:1052cc0020200000004200006175000064200000f6
:1052dc0052610000746500003d2500007300000061
:1052ec00564600004f2000003d200000412f0000da
:1052fc00422000002b200000537000006c74000052
:10530c0000560000464f0000203d00002025000004
:10531c00692000004d6500006d2000002020000079
:10532c00202000000046000020250000692000001d
:10533c0025690000205700002000000052200000ca
:10534c00256900002025000069200000572000007e
:10535c0000000000447500006d7000002045000046
:10536c0045500000524f00004d200000636f0000bc
:10537c006e740000656e0000747300000a0d00006e
:10538c00000a00000d250000352e000034580000e6
:10539c000020000025340000580000000a0d000019
:1053ac004c610000737400002073000075630000f2
:1053bc006365000073730000206300006f640000dd
:1053cc00652000003d200000255800002000000052
:1053dc000a0d00004a5500004d4100002d540000fc
:1053ec005258000032200000636f000070790000fa
:1053fc007269000067680000742000004f480000cc
:10540c003753000056200000262000004f480000b3
:10541c00324e00004c5400000a0d0000000a00003f
:10542c000d5300006f66000074770000617200007d
:10543c00652000007665000072730000696f000043
:10544c006e200000002c0000206300006f70000034
:10545c00797200006967000068740000204a00003f
:10546c0075680000612000004e690000696e000044
:10547c00696b00006f7300006b690000204f000027
:10548c00483200004e4c0000540a00000d00000091
:10549c000a0d000041440000432000002569000073
:1054ac00203d00002025000069000000454500005b
:1054bc00505200004f4d0000207200006573000038
:1054cc0065740000206300006f7500006e740000ae
:1054dc0065720000206300006c65000061720000c2
:1054ec00656400000a0d0000004c000043440000fd
:1054fc002077000072690000746500000a0d00003e
:10550c000063000068610000722000003d20000074
:10551c00257800000a0d0000004c000043440000f8
:10552c0020620000617200002067000072610000c0
:10553c0070680000202600002063000068610000f5
:10554c00726100006374000065720000207400003a
:10555c0065730000740a00000d0000002563000054
:10556c00203d00002030000078250000582000006d
:10557c00200000000a0d00004d750000746500004d
:10558c00000a00000d41000075640000696f000006
:10559c00206f00006e0000000a0d0000535f000039
:1055ac006d65000074650000722000003d20000055
:1055bc00253100002c5000004f540000203d00000d
:1055cc0020250000690a00000d0000000a0d0000f3
:1055dc002065000065700000726f00006d2e0000e9
:1055ec006465000066760000616c00002e76000099
:1055fc00666f00005f730000656c0000203d0000ca
:10560c0020250000690000000a0d00002076000033
:10561c00666f00005f69000064780000203d0000a8
:10562c0020250000690000000a0d00002065000024
:10563c0065700000726f00006d2e00006465000044
:10564c0066760000616c00002e6d00006f64000037
:10565c00655b0000766600006f5f00006964000007
:10566c00785d0000203d000020250000690000004e
:10567c000a0d00002065000065700000726f0000cc
:10568c006d2e00006465000066760000616c000001
:10569c002e6d00006f640000655b0000325d000041
:1056ac00203d000020250000690000000a0d0000cc
:1056bc0020630000775f00006163000074690000e4
:1056cc0076650000203d00002025000069000000e8
:1056dc000a0d000020740000756e0000655f00006c
:1056ec006f6e0000203d00002025000069000000c6
:1056fc000a0d000020500000545400005f490000c7
:10570c004e2000003d20000025690000000a00002a
:10571c000d530000657400003a2000006565000020
:10572c00707200006f6d00002e6400006566000052
:10573c00766100006c2e00006d6f00006465000047
:10574c005b3200005d2000003d200000000a0000dc
:10575c000d52000065660000204f000073630000ce
:10576c00203d0000202500006c690000204d000049
:10577c00487a00000a0d0000000a00000d6d0000c0
:10578c0073200000636f0000756e000074650000ec
:10579c00722000003d200000256900000a0d000069
:1057ac00000a00000d530000504900002054000076
:1057bc00780000000a0d0000535000004920000042
:1057cc0054780000206300006f6e0000740000002d
:1057dc000a0d0000504100002041000074740000cc
:1057ec00656e000075610000746f0000722000008f
:1057fc003d2000003078000025580000000a000011
:10580c000d5200004620000041740000746e000030
:10581c0020730000656c00006563000074200000bc
:10582c0069640000782000003d200000256900001c
:10583c002c200000484300003539000035200000c2
:10584c006269000074730000203d000020300000ed
:10585c0078250000580000000a0d000044440000a8
:10586c0053200000747500006e6500002074000069
:10587c0065730000742000004f4e0000000a000009
:10588c000d4400004453000020740000756e0000ad
:10589c00652000007465000073740000204f000048
:1058ac0066660000000a00000d440000445300002e
:1058bc0020740000756e0000696e00006720000007
:1058cc00776f0000726400002064000069730000b0
:1058dc00706c000061790000000a00000d4e0000a1
:1058ec006f7200006d6100006c20000046720000b9
:1058fc0065710000756500006e6300007920000082
:10590c0064690000737000006c6100007900000095
:10591c000a0d000044440000532000007475000080
:10592c006e6900006e670000207300007465000053
:10593c00702000002320000025690000203d00009d
:10594c00202500006c690000000a00000d440000d6
:10595c006976000020620000792000005a65000082
:10596c00726f0000004b0000657900002069000098
:10597c00733a000020250000640a00000d000000ae
:10598c0054720000793a000020560000616c00004f
:10599c0069640000206300006f6d00006d61000001
:1059ac006e640000730a00000d0000000a0d000078
:1059bc0053650000727600006963000065200000ea
:1059cc0026200000636100006c6900006272000018
:1059dc0061740000696f00006e2000006d6f0000a4
:1059ec00646500002c200000636100006c20000046
:1059fc006672000065710000203d0000202500004b
:105a0c006c6900002c20000044440000532000006e
:105a1c003d200000256c0000690000000a0d00000c
:105a2c0044490000535000004c4100005920000034
:105a3c003d20000070610000726100006d65000087
:105a4c007465000072200000736500006c65000036
:105a5c00637400002c2000004641000053540000e9
:105a6c002f5600004641000053540000203d00001a
:105a7c0020730000617600006520000026200000e5
:105a8c006578000069740000005300006574000024
:105a9c002052000065660000204f00007363000078
:105aac002046000072650000710000004f7300007a
:105abc0063200000256c000069200000487a00007b
:105acc000053000075700000706c0000792000001d
:105adc002000000056200000200000004361000060
:105aec006c2000006d7500006c740000203d0000ff
:105afc00202500006c690000202000002020000000
:105b0c000042000065650000702000006c6500001c
:105b1c006e2c0000203000003d4f00004646000077
:105b2c00200000004265000065700000203d000070
:105b3c0020250000692000006d730000202000006b
:105b4c0020200000005300002d6d00006574000043
:105b5c006572000000430000616c0000206d0000c5
:105b6c00756c0000742000003d200000256c0000c6
:105b7c006920000020000000466f000072770000d2
:105b8c0061720000642000000052000046200000fa
:105b9c00416d0000702e00002000000050750000c8
:105bac0073680000204600004153000054200000a0
:105bbc006c6f00006e670000203d00000066000066
:105bcc0061630000746f00007279000020640000b3
:105bdc0065660000617500006c74000073000000c5
:105bec0046610000637400006f72000079200000b1
:105bfc007365000074750000702000006f6b00006e
:105c0c00000a00000d46000061630000746f000084
:105c1c007279000020640000656600006175000068
:105c2c006c74000073200000726500007374000037
:105c3c006f7200006564000000430000616c00009e
:105c4c0069620000722e0000205300006176000093
:105c5c0065640000000a00000d430000616c000048
:105c6c006962000072610000746900006f6e0000d0
:105c7c002073000065740000746900006e670000fa
:105c8c007320000073610000766500006420000042
:105c9c00746f00002045000045500000524f00007a
:105cac004d0000000a0d000054520000415000004d
:105cbc003a2000004f730000636900006c61000023
:105ccc00746f00007220000045720000726f0000bb
:105cdc00720a00000d0000004f5300004343000007
:105cec004f4e00002030000078250000580a0000bc
:105cfc000d0000000a0d000054520000415000003d
:105d0c003a200000416400006472000065730000da
:105d1c007320000045720000726f0000720a0000d0
:105d2c000d000000573000002030000078250000e6
:105d3c00580a00000d000000573100002030000010
:105d4c0078250000580a00000d00000057320000b2
:105d5c002030000078250000580a00000d000000db
:105d6c00573300002030000078250000580a00004e
:105d7c000d00000057340000203000007825000092
:105d8c00580a00000d0000005735000020300000bc
:105d9c0078250000580a00000d000000573600005e
:105dac002030000078250000580a00000d0000008b
:105dbc00573700002030000078250000580a0000fa
:105dcc000d0000005738000020300000782500003e
:105ddc00580a00000d000000573900002030000068
:105dec0078250000580a00000d0000005731000013
:105dfc003020000030780000255800000a0d00000b
:105e0c0000570000313100002030000078250000e0
:105e1c00580a00000d00000057310000322000002d
:105e2c0030780000255800000a0d000000570000d3
:105e3c00313300002030000078250000580a0000a3
:105e4c000d000000573100003420000030780000b5
:105e5c00255800000a0d00000057000031350000e5
:105e6c002030000078250000580a00000d000000ca
:105e7c000a0d000054520000415000003a2000006e
:105e8c0053740000616300006b2000004572000039
:105e9c00726f0000720a00000d0000000a0d000075
:105eac0054520000415000003a2000004d610000a7
:105ebc007468000020450000727200006f720000d0
:105ecc000a0d0000000a00000d5300007075000060
:105edc00726900006f75000073200000496e0000ad
:105eec007465000072720000757000007420000070
:105efc0045720000726f0000720a00000d00000075
:105f0c00202000002020000045720000726f00006d
:105f1c007220000021200000202000002020000022
:105f2c00000000000a0d0000566f000069630000bd
:105f3c00652000004d6500006d200000636d0000c1
:105f4c00642000003d200000000a00000d560000f7
:105f5c006f69000063650000204d0000656d000056
:105f6c0020530000746f0000702000006f70000060
:105f7c006572000061740000696f00006e00000023
:105f8c000a0d0000566f00006963000065200000d8
:105f9c004d6500006d6f00007279000020650000f7
:105fac007261000073650000206100006c6c0000e1
:105fbc00000a00000d4d0000656d0000203d000042
:105fcc0020250000690000000a0d0000564d00005d
:105fdc002c200000706c000061790000206d000026
:105fec00656d00006f720000790000000a0d000062
:105ffc00564d00002c20000054580000000a0000f0
:10600c000d5600004d20000052580000000a000000
:10601c000d5600004d2c000020520000656300005e
:10602c006f72000064200000667200006f6d00004b
:10603c00204d000069630000000a00000d560000ae
:10604c006f69000063650000204d0000656d000065
:10605c006f720000792000006f70000074690000fe
:10606c006f6e0000206e00006f740000206900004d
:10607c006e730000746100006c6c000065640000bd
:10608c00003f00000000000010000000ff030000b3
:10609c0000040000af040000b0040000070500007d
:1060ac00080500005f05000060050000b705000052
:1060bc00b80500000f06000010060000670600007f
:1060cc0068060000bf060000c006000017070000ad
:1060dc00180700008f0700000a0d00005452000042
:1060ec00582d000032200000766f0000696300001c
:1060fc00652000006d6500006d6f00007279000076
:10610c00206f000070740000696f00006e200000aa
:10611c00666f0000756e00006420000028490000c6
:10612c0053440000313700003234000030200000ae
:10613c006368000069700000290a00000d0000006f
:10614c00504c000041590000204d0000656d0000ce
:10615c002023000020250000692000002000000002
:10616c0054580000204d000020250000692000003c
:10617c0020000000546900006d650000202500001f
:10618c006920000073200000202000002020000067
:10619c002000000052450000432000004d69000023
:1061ac0063200000204d0000656d000020230000de
:1061bc00202500006920000000520000582000003b
:1061cc004d20000025690000202000000000000088
:1061dc003d420000256900000a0d0000003d000052
:1061ec0053250000690a00000d0000003d4d000021
:1061fc00256900000a0d0000003d00005625000036
:10620c00690a00000d0000003d460000000a000075
:10621c000d0000003d410000256900000a0d000042
:10622c00003d0000572500006c6900000a0d0000bd
:10623c00003d000052250000690a00000d0000001e
:10624c003d540000310a00000d0000003d540000d8
:10625c00300a00000d00000086010000c2000000a2
:10626c006100000030000000170000000b0000006f
:10627c0007000000030000000a0d00004f7500002d
:10628c00745f00006978000064200000256900003c
:10629c002c200000496e00005f690000647800004b
:1062ac002025000069200000200a00000d000000dd
:1062bc00200000000001000001020000200300008b
:1062cc00030400000402000006060000060600009d
:1062dc00050700000707000086010000c20000004f
:1062ec006100000030000000170000000b000000ef
:0862fc00070000000300000090
:020000040000fa
:106304000200fa000000eb00000f780010003700d4
:106314001e007800000040004108200080804000fa
:10632400008b2000808040000000eb008008780093
:106334001e007800c200dd00008b200000814000b8
:106344004079280051a820000089be001e0fe800f3
:10635400d00120009e0f1000edff3400100020003b
:10636400704988000000eb008049880090002000fc
:1063740090498800c0902d00b153200080458800ca
:10638400914588000000eb00a0498800d022240039
:1063940061a82000a0458800b14588000000eb00fa
:1063a400b049880010772a00d1402100c0458800f8
:1063b400d14588000000eb00c0498800b08e22005f
:1063c40091cc2100e0458800f145880020002000a0
:1063d400d0498800b000220041862200004688008f
:1063e4001146880010002000e0498800d04b2000ae
:1063f400c137230020468800314688001000200061
:10640400f0498800f0e92500d1c423004046880003
:106414005146880010002000004a8800d0092a0054
:10642400316d240060468800714688001000200009
:10643400104a88001014210011112500804688009c
:106444009146880010002000204a88000000eb00dc
:10645400804b88000000eb00904b88000000eb00ac
:10646400b04b88000000eb00a04b88002000200007
:10647400c04b8800007d2000d04b880040062000df
:10648400e04b88000000eb00f04b8800b0042000d3
:10649400004c880020022000104c8800e0012000fd
:1064a400204c8800d0012000304c8800e0272800d0
:1064b400010020004049880051498800d04e210045
:1064c4006049880020002000404c88000000eb0058
:1064d400504c880010002000604c88000000eb0045
:1064e400704c880030002000804c88000050290047
:1064f400a1ab2000a04c8800b14c8800509d210025
:1065040001002000c04c8800d14c880040082000c5
:1065140001002000e04c8800f14c880080892000b4
:1065240001002000004d8800114d880070012000fa
:1065340001002000204d8800314d880070012000aa
:1065440001002000404d8800514d880020032000a8
:10655400604d880030c0b300aee9b70030c0b3006e
:10656400afe9b70010c0b300b0e9b70010c0b30082
:10657400b1e9b70010c0b300b2e9b70010c0b3006e
:10658400b3e9b70010c0b300b4e9b70010c0b3005a
:10659400b5e9b70010c0b300b6e9b70010c0b30046
:1065a400b7e9b70010c0b300b8e9b70010c0b30032
:1065b400b9e9b70013002000e28a2000e11f2f0090
:1065c400f007200078210700704580000000e800f3
:1065d4007045880012002000e11f2f00f007200002
:1065e4007e21070013002000e21f2f00f107200086
:1065f400e08a20009a2107000080fa0000000600cb
:106604000400fa000000eb00904c88000000eb004e
:10661400100798002c0037009e009000000720000f
:10662400808f500009003e00924c80001e009000b4
:1066340080004000008b20000080400010007800a3
:1066440000004100904c880003003700904c80000b
:106654000000ea00904c88001e00900000004000fa
:106664008000780000002f00008040008000780047
:1066740012002000f007200058210700000f7800c6
:106684001e009000000040008000780000002f00f1
:1066940000804000000178001e00900000004000cf
:1066a40080007800008b2000008040001300200050
:1066b400f10720006a210700000f78001e009000f7
:1066c4000000e800100798009e00900010072000ca
:1066d400808f5000d0ff3600904c8000801f7800df
:1066e4001e007800801f78001e009000801f780034
:1066f400c04a2a00801f780034e70700e887570063
:106704000080fa00000006000600fa000000eb001a
:10671400000f78000000eb002007980018003700f5
:106724002e0090000000400080007800008b2000c4
:10673400008140002e00900000004000800078009e
:1067440000002f000080400080007800130020002b
:10675400f007200014210700100798002e00900075
:1067640080004000008b2000008040001000780072
:106774001e0f40002e0090000000e8002007980043
:10678400ae00900010072000808f5000e4ff360018
:1067940013002000e28a2000e11f2f00f0072000f0
:1067a400012107001e0078000080fa0000000600a6
:1067b4000400fa000000eb00f04d88000000eb003c
:1067c400100798002b0037001e009000f40f5000b3
:1067d40009003e00f24d80001e0090008000400041
:1067e4004099200000804000100078000000410023
:1067f400f04d880003003700f04d80000000ea00ef
:10680400f04d88001e0090000000400080007800d9
:1068140000102f000080400080007800120020004b
:10682400f0072000ed200700000f78001e00900004
:10683400000040008000780000102f00008040001d
:10684400000178001e0090000000400080007800e5
:10685400409920000080400013002000f107200030
:10686400ff200700000f78001e0090000000e800e1
:10687400100798001e009000f50f5000d2ff36005c
:10688400f04d8000801f78001e007800801f780083
:106894001e009000801f7800504d2a00801f780051
:1068a400cae60700e88757000080fa0000000600e7
:1068b4000600fa000000eb00000f78000000eb0077
:1068c40020079800180037002e00900000004000b8
:1068d4008000780040992000008140002e00900044
:1068e400000040008000780000102f00008040006d
:1068f4008000780013002000f0072000aa20070081
:10690400100798002e00900080004000409920005d
:1069140000804000100078001e0f40002e00900000
:106924000000e800200798002e009000f50f5000aa
:10693400e5ff36001e0078000080fa000000060023
:106944000e00fa0050079800610798006e0090004e
:106954006101b900400620000013b8006010b900be
:106964000702780000024200400620000098b900a7
:1069740000024200840378005e0090006101b900c7
:106984000600be00faf107002007980031079800be
:1069940042062000030020002e009000be0090005c
:1069a400001f5100019759001e00be00e00f500067
:1069b400e08f580003003c0010002000010020007c
:1069c400008fbe00de00900010032000808f500076
:1069d40014003400ae00900040062000000ab80005
:1069e4002e0090006000b90005017800000141000c
:1069f400be009000400620000088b900000141005c
:106a0400820278000071220001002000040040008e
:106a1400858048001e01be00d5f10700400798009c
:106a2400020037000000eb00400798004e00900081
:106a34000080fa00000006000400fa00889fbe00ef
:106a4400b0002000442107006104b900004d80001b
:106a5400114d80000001be000243b80003c0b9001c
:106a640007027800000242000990b90000024200c7
:106a740084037800068fbe001e00be004008de00be
:106a840001002000d0438800d0438000530b07004e
:106a94004f04be000080fa00000006000200fa0065
:106aa400e04380006101b900207520000012b800a5
:106ab4006010b9000503780000034300207520002e
:106ac4000098b90000034300860278004028de00e5
:106ad4000100200010458800104580003f0b07008e
:106ae4000080fa00000006000000fa00c0418000a7
:106af4000000e00002003a00e8ff07000100370050
:106b0400cdff07000080fa00000006000200fa0032
:106b1400889fbe00c04180000000e00025003a00cc
:106b2400f04f2a00370c0700464d8000574d800077
:106b340052448000634480000234b80003b0b900ba
:106b440009027800000242000790b90000024200e6
:106b54008404780040c8de00cf80de00000f780097
:106b6400704480009e0f1000040034001e00780062
:106b740070448800600420008044880080448000c1
:106b84000000e90080448800804480000000e000a8
:106b940004003a0060042000804488001e0078004d
:106ba400704488007044800071072000520d070073
:106bb4000600370030502a00120c07000000eb00da
:106bc4007044880060042000804488004f04be00a4
:106bd4000080fa00000006000000fa00889fbe0052
:106be400c04180000000e00017003a00900020003f
:106bf400d92007006103b900c24c8000d34c800047
:106c04000234b80003b0b90009027800000242005f
:106c14000790b900000242008404780040c8de00f6
:106c2400cf80de0000448800c0502a00f50b070026
:106c340000448000210020002f0d0700f0502a009e
:106c4400f00b07000200370010512a00ed0b07007b
:106c54004f04be000080fa00000006000200fa00a3
:106c64000000eb00000f78000b0037001e007800d6
:106c7400c200dd00c0412a00008040001001be00b7
:106c8400d0408000e1408000800f5100818f590086
:106c940004003c001e0fe800a00020009e0f10001e
:106ca400f2ff34001e007800804188000080fa0062
:106cb400000006000000fa00e8ff070080418000a1
:106cc400fa00400040992000008040001040780005
:106cd4000080fb004e00dd00704188008041800090
:106ce4008000400080442a000080400010007800aa
:106cf400004e8800014e80007041800000807000ca
:106d0400004e8800d2408000e3408000b0602b0039
:106d140001b62000800f5100818f59000400340017
:106d2400004e80000108200001007000004e880021
:106d3400604c80000000e00004003200004e80003f
:106d44000104200001007000004e8800a04b800068
:106d54000000e00004003200004e80000102200028
:106d640001007000004e8800b04b80000000e0007d
:106d740006003200604c8000e10f500003003a002e
:106d8400004e80000040a000004e8800904b800020
:106d94000000e00003003200004e80000030a0003c
:106da400004e8800c04b80000000e00003003a0061
:106db400004e80000020a000004e8800104180009a
:106dc400000040004108200080804000008b20002b
:106dd4000080400010007800e10f500003003200f2
:106de400004e80000010a000004e8800104180007a
:106df400000040004108200080804000008b2000fb
:106e04000080400010007800e10f500003003c00b7
:106e1400004e80000000a000004e8800004e80005c
:106e2400fa1f07000080fa00000006000200fa00c2
:106e3400889fbe0071003700d00020004620070064
:106e4400e0438800c000200043200700f04388008e
:106e5400e04380006104b900e04380006101b900af
:106e64000243b80003c0b9000702780000024200e0
:106e74000990b90000024200840378001644880097
:106e840027448800f04380006104b900f043800087
:106e94006101b9000243b80003c0b90007027800d9
:106ea400000242000990b900000242008403780005
:106eb40036448800474488001244800023448000fc
:106ec400304480004144800000005100818059001a
:106ed40050448800614488000040eb008f0907009b
:106ee40001ff0700f04f2a00460b0700464d8000c3
:106ef400574d800052448000634480000234b8003f
:106f040003b0b90009027800000242000790b900fa
:106f1400000242008404780040c8de00cf80de0016
:106f2400000f7800710720001e007800720c070023
:106f340000c4b30079090700a0512a00310b0700ef
:106f440080418000fa004000409920000080400009
:106f5400104078000004e00003003a000002200022
:106f6400fb0a070002003700d0022000f80a0700dd
:106f740080418000fa0040004099200000804000d9
:106f840010407800af0c070060522a001d0b070068
:106f940080418000fa0040004099200000804000b9
:106fa400104078000080fb00000f7800a000200053
:106fb400df1d07001e0f1000300020009e0f100080
:106fc4000200340030002000000f78001e00e000b2
:106fd40002003d000000eb00000f780081418000ba
:106fe4001e00780000417800fa804000409920009b
:106ff40000804000024878002eff0700cfc2bf0087
:107004000044b2000004e0008bff3a00e8fd0700f2
:10701400bd1d07004f04be000080fa0000000600fa
:107024000000fa00e04b8000ea160700f04b8000f5
:10703400504588000080fa00000006000000fa00b5
:107044000000eb00e31607000080fa0000000600d1
:107054000000fa00b04180000000e00002003200ad
:1070640072ff070043003700804380000000a20045
:1070740080438800804380000000e00004003a0060
:10708400614d8000c0f62100471707000300370058
:10709400614d8000108f2100431707002909070064
:1070a400004b2000406088002e0037000040eb00b9
:1070b4001a09070040608000c21220001100090074
:1070c4000280d800801f7800a0522a00801f780018
:1070d400008420009fe40700e48757000084200018
:1070e400c80a070000c4b3000c09070080438000ed
:1070f4000000e00003003200d0532a00c10a070058
:1071040002003700e0542a00be0a070040608000f5
:107114000000e00013003a00c8ff0700604d800043
:107124000000400080007800e05522001e17070090
:10713400604d8000000040006b1f070030fd070019
:107144008a160700f0552a00801f78009fe4070084
:107154008f87e90020002000631f0700cfa2a90049
:10716400ffff3700cfc2bf000044b2000004e000bc
:10717400ceff3a000080fa00000006000200fa0088
:10718400f0080700c0582a009e0a070000c4b30094
:10719400e2080700d0592a009a0a0700c819070014
:1071a4000000e00011003200d5190700004f7800fc
:1071b400a1002000904f2100fb1607001e4078001c
:1071c400b319070000c4b300d4080700e05a2a002a
:1071d4008c0a07001e80fb005d0a0700805b2a0002
:1071e400880a07001e4078005f0a0700cfc2bf006c
:1071f4000044b2000004e00001003a00e7ff370059
:107204000080fa00000006002600fa00889fbe00f5
:107214008a9fbe008c1f7800f0f32f0000168800b0
:107224000000eb001016880030e72f0030168800ad
:107234000000eb0040168800e0012400601688007e
:107244000000eb00701688000000eb009016880028
:107254000000eb00a016880080e12f00f0168800e3
:107264000000eb00001788000008210020178800a8
:107274000000eb0030178800cfa2a800404425008e
:10728400a00488000e160700c81e07006000b8009e
:10729400af1e07004079280051a82000ac1e07004b
:1072a4005055250051552500204088003140880064
:1072b4002003200010608800c0d4210040408800d2
:1072c4000000eb00704188000000eb00004e8800d5
:1072d400c01e0700004e8000cc1e0700a108070056
:1072e400e708070097080700d05b2a00450a070053
:1072f400e03b2a00430a070000c4b30087080700e4
:10730400805c2a003f0a070045190700c71d0700d3
:10731400905d2a00801f78002ce407008f87e90025
:10732400e03b2a00801f780028e407008f87e900eb
:10733400105f2a00801f780024e407008f87e9008b
:10734400503c2a00801f780020e407008f87e90062
:10735400a05f2a00801f78001ce407008f87e900e3
:1073640040408000801f780020622a00801f78003f
:1073740016e40700e4875700a0632a00d31d070022
:10738400e61e0700a0652a001e0a07000000eb00a5
:107394007043880080bb2000406088001d003700d7
:1073a400406080000000e0001a003a00e115070088
:1073b400c1122000e05522007b16070000c4b30070
:1073c4005608070030662a000e0a07001000200045
:1073d4007043880020c72100711c270020408800ca
:1073e40031408800cfc2bf000044b2000004e00076
:1073f400fcff3a000040eb004808070040672a0001
:10740400000a070000c4b3004408070050682a00bb
:10741400fc090700cfc2bf000044b2000004e00032
:10742400dfff3a0022fd0700200f9800b6fc07009a
:10743400100f980070458000801f78001e0890008f
:10744400801f7800ae089000811f780060692a00d0
:10745400801f7800dde30700e88757002e089000be
:107464000000e00003003a001e0890000000e00065
:107474000800320047110700d06d2a00801f7800f1
:10748400d2e307008f87e9009dfb0700c8fc0700d3
:107494005bfc0700d04b8000d4150700e04b800054
:1074a400cc150700911c07000000eb008043880006
:1074b4000000eb00404388000000eb0050438800cc
:1074c4000000eb00504388000000eb00b04188004e
:1074d4000000eb00a0418800804980001041880032
:1074e40010418000c200dd00008b200000804000bd
:1074f4001000be00d0408800e1408800d0408000e9
:10750400e1408000121e07005a0b0700007d200096
:10751400751e07000b080700c7170700851507002d
:1075240040012000701e0700604d800000004000f4
:1075340080007800904f21001b16070070438000e4
:107544000000e00012003200521307001000370060
:107554000040eb00f1070700e0702a00a9090700ca
:1075640000c4b300ed070700f0712a00a509070065
:10757400c3c2bf00704060000004e00004003a0091
:107584005ffb07008afc07001dfc070004003700ae
:10759400cec2bf00644060000004e000ecff320093
:1075a400804c80004300dd008000780000462a0003
:1075b40000804000814c8000801f7800811f78008b
:1075c40000732a00801f780080e30700e6875700d5
:1075d400804c80009f180700804c8000e30f50000f
:1075e4000c003200804c80004300dd0080007800f5
:1075f40000462a0000804000814c8000801f7800f3
:10760400811f7800b0752a00801f78006fe307009f
:10761400e6875700c3c2bf000042b2000004e00086
:1076240001003a00d5fe0700ae1807003d1d070013
:107634007bfe070000003700c8c2bf000044b20050
:107644000004e0000300320010002000c041880064
:10765400030037000000eb00c041880070fe070003
:10766400804980001041880090498000e20f50005a
:1076740029003a00c0418000e10f500006003a00a2
:1076840010418000e10f5000080034000000eb00be
:10769400104188000500370010418000e10f5000c0
:1076a400020034001000200010418800804980004e
:1076b400e20f500009003a00b0498000e20f500088
:1076c40003003a0010002000a04188002000370089
:1076d4000000eb00a04188001d003700104180002d
:1076e400000040004108200080804000008b200002
:1076f4000080400010007800e20f500003003a00c0
:1077040010002000a0418800110037000000eb00a9
:10771400a04188000e0037001041800000004000a6
:107724004108200080804000008b20000080400041
:1077340010007800e20f500003003a00100020000f
:10774400a0418800020037000000eb00a04188003f
:10775400104180000000400041082000808040006b
:10776400008b20000080400010007800e30f5000e0
:1077740011003a00c04180000000e0000a003a0015
:10778400ca62a800b04180000000e00010003a0086
:1077940010002000b0418800614d8000904f21000e
:1077a400811507000a003700ca62a9000000eb0037
:1077b400b041880006003700b04180000000e000be
:1077c400030032000000eb00b0418800ca62a90047
:1077d40040ccbf000004e00062003200404380005f
:1077e4000000e0005f003a000040eb0040ecb7000e
:1077f400804380000000e00059003a0008fe0700c2
:10780400504080000000e0001b003a001c41800052
:1078140010418000c200dd00008b20000080400089
:107824001005be00b81b07006104b9007049800050
:10783400c200dd00803e2a00008040001001be002e
:107844000243b80003c0b9000702780000024200f6
:107854000990b90000024200840378000a01430041
:107864008b814b00c260dd00008b20000080400053
:107874000288be001a0037001c41800010418000bd
:10788400c200dd00008b2000008040001005be0017
:107894009d1b07006104b90060408000c200dd0048
:1078a400003d2a00008040001001be000243b800e1
:1078b40003c0b90007027800000242000990b90031
:1078c40000024200840378000a0143008b814b00cc
:1078d400c260dd00008b2000008040000288be00f2
:1078e40010418000c200dd00008b200000804000b9
:1078f4001001be002040800031408000800f510004
:10790400818f59000700340010418000224080001c
:1079140033408000c200dd00008b20000080400066
:107924000288be0010418000c200dd00008b2000f0
:10793400008040001000be00e00f5000e08f5800af
:1079440008003d0010418000c200dd00008b2000d3
:10795400008140006000b8000089be0001003700cb
:10796400691b070010418000c200dd00008b20006d
:10797400008040001000be00d0408800e140880034
:1079840010418000c200dd00008b20000080400018
:107994001000be00f040880001418800804b800048
:1079a400e10f50002e003a00f00020006a1d07008d
:1079b400300f9800be08900010832000808f500084
:1079c400050034003e089000e17c2f0001004000d7
:1079d400300f98000b003700be089000e07c2000b8
:1079e400808f500005003c003e08900021832f004a
:1079f40001004000300f9800020037000000eb0047
:107a0400300f98003e0890006102b9008001200008
:107a14000023b8006020b90007017800000141008c
:107a24007828b900000141008203780026418800cb
:107a340037418800c0418000e10f500008003a003f
:107a4400d0408000e140800022418000334180002a
:107a54000000410081804900d0408800e140880056
:107a6400804b8000e20f50001b003a00f000200021
:107a7400391d0700300f98003e0890006101b900dd
:107a8400e00520000012b8006010b900050378007a
:107a940000034300e00520000098b9000003430000
:107aa400860278004441880055418800c041800026
:107ab4000000e00008003a00d0408000e14080006f
:107ac4004241800053418000000041008180490010
:107ad400d0408800e1408800104180000000400050
:107ae4004108200080804000008b2000008040007e
:107af40010007800e20f500013003a00c0418000eb
:107b04000000e00010003a00d2408000e340800012
:107b14004049800051498000000051008180590093
:107b2400d0408800e1408800f2408000034180009a
:107b34004049800051498000000051008180590073
:107b4400f040880001418800d0408000e14080007e
:107b54007f1c070057fc0700c04180000000e000c4
:107b64000f003a001041800000004000410820004e
:107b740080804000008b20000080400010007800ce
:107b8400e10f500003003c00304c80000314070058
:107b94000b00370020032000001407000800370002
:107ba400c04b800000004000010d20008080400098
:107bb400008b20000080400010007800f7130700bd
:107bc400c04180000000e0002d003a00d0002000f9
:107bd400e11c0700e0438800c0002000de1c070011
:107be400f0438800e04380006104b900e043800072
:107bf4006101b9000243b80003c0b900070278006c
:107c0400000242000990b900000242008403780097
:107c14001644880027448800f04380006104b900ba
:107c2400f04380006101b9000243b80003c0b90009
:107c340007027800000242000990b90000024200e5
:107c44008403780036448800474488001244800046
:107c540023448000304480004144800000005100ef
:107c6400818059005044880061448800f1438000b9
:107c7400e043800032fb0700e04488000200370044
:107c8400800c200000458800e0002000b21c0700a2
:107c9400204588002145800000002100010050009b
:107ca400300f98003e0890004015b000300f980047
:107cb4003e0890006104b9003e0890006101b900db
:107cc4000243b80003c0b900070278000002420072
:107cd4000990b90000024200840378001607980056
:107ce400270798001e009000ae0090004108de00b7
:107cf40001002000300f98003e08900074004000fe
:107d0400300f98003e09900012608800404c8000bb
:107d1400e0418800704c80000000e000190032004f
:107d2400c04180000000e00016003200d043800013
:107d34008080e800204580004680de00808f50006f
:107d440009003400904380000000e00006003a007f
:107d54008a130700401f2000304588000000eb0014
:107d6400404588000f003700304580000000e000e7
:107d74000c003a007d1307001000200040458800e5
:107d8400080037000000eb00404588009043800065
:107d94000000e00002003a007813070001003700f9
:107da40072130700c3c2bf000042b2000004e00027
:107db40055003a009afc0700803e2000406088008d
:107dc400404380000000e00007003a005043800078
:107dd400e40f500004003a00614d8000c0f6210019
:107de400f11307000d00370040438000e10f5000fd
:107df40007003a0060438000ec0f500004003a0092
:107e0400614d8000c0f62100e7130700030037002e
:107e1400614d8000108f2100e3130700400620000d
:107e2400311c070009003700406080000000e000ba
:107e340006003a00604d80006a00b90080007800b6
:107e4400c0f62100d813070004003700c3c2bf00e6
:107e54000042b2000004e000f3ff32004060800002
:107e64000000e0000f003a00404380000000e800fa
:107e74004043880040438000e10f5000020034007a
:107e84000000eb0040438800c3c2bf000042b200c0
:107e94000004e000fcff320040062000121c070032
:107ea40014003700404380000000e00009003a005d
:107eb400504380000000e800504388005043800095
:107ec400e40f50000b0034000000eb005043880026
:107ed40008003700604380000000e8006043880029
:107ee40060438000ec0f5000020034000000eb00ff
:107ef40060438800041a0700c3c2bf000042b200f6
:107f04000004e000fcff3200c3c2bf007040600008
:107f14000004e00035003a0041fc0700704980008d
:107f2400e20f500004003a00614d8000c0f62100c9
:107f34009d13070003003700614d8000108f21005e
:107f440099130700803e200040608800400620000e
:107f5400e51b070009003700406080000000e000d6
:107f640006003a00604d80006a00b9008000780085
:107f7400904f21008c13070004003700c3c2bf00d8
:107f8400704060000004e000f3ff320040608000b5
:107f94000000e00009003a00400020007049880019
:107fa400c3c2bf00704060000004e000fcff320068
:107fb40040062000cc1b07000800370070498000f1
:107fc400e20f500003003a001000200070498800be
:107fd400020037002000200070498800c3c2bf009f
:107fe400704060000004e000fcff3200cec2bf001d
:107ff400704060000004e00029003a0008fc07001b
:10800400803e200040608800804b80000000e0003b
:1080140006003200614d8000c0f6210062130700a3
:108024000000eb00804b880005003700614d8000a4
:10803400108f21005c13070010002000804b880083
:1080440040062000a81b07000b003700406080009a
:108054000000e00008003a00604d80006a00b900aa
:1080640080007800108f21004f13070020002000ab
:10807400804b880004003700cec2bf00704060000f
:108084000004e000f1ff3200cec2bf007040600087
:108094000004e000fcff320040062000921b0700b1
:1080a400cec2bf00684060000004e000ca003a008d
:1080b400c04180000000e000c7003200d8fb070088
:1080c40090498000e20f500049003a008049800046
:1080d400e20f500004003a00614d8000c0f6210018
:1080e4003113070003003700614d8000108f210019
:1080f4002d1307000000eb00c0498800803e2000db
:108104004060880040062000771b07000900370004
:10811400406080000000e00006003a00604d8000ee
:108124006a00b90080007800c0f621001e13070021
:1081340004003700cec2bf00684060000004e000c5
:10814400f3ff3200406080000000e0001f003a00ae
:10815400104180000000e0000b003a0080458000e0
:1081640091458000a0458800b1458800a049800061
:10817400b049880000c4b300e804070050782a001e
:10818400a00607000a003700a0458000b145800022
:108194008045880091458800b0498000a049880046
:1081a40000c4b300dd04070060792a0095060700c7
:1081b400cec2bf00684060000004e000fcff320053
:1081c40040062000481b07008300370080498000d8
:1081d4000000e8008049880080498000e20f5000d8
:1081e4007d0034000000eb00804988007a003700ed
:1081f40080498000914980008100e900810f50008e
:1082040004003a00614d8000c0f62100e612070028
:1082140003003700614d8000108f2100e212070037
:1082240039190700500f98000000eb00400f980028
:1082340055003700200120003d190700300f980039
:108244003e0890000000e0004f00320010002000c3
:10825400400f980081498000904980000000e900a7
:10826400808f500003003200804980000000e0004d
:1082740005003a00604d8000c280de00c0f6210097
:10828400c912070004003700604d8000c280de0080
:10829400108f2100c4120700814980003e0890001d
:1082a4000080400080498800814980009049800016
:1082b400808f500003003500904980000000e900e1
:1082c40080498800804980000000e00002003d00f1
:1082d4000000eb008049880000c4b3008f0407004d
:1082e40080498000c200dd00008b20000080400037
:1082f4001002be004fabde00cfb3de000400be00b0
:108304000601780086017800a84c8000b94c8000f2
:108314004fcdde00cfd5de000802be000a03780090
:108324008a037800a1eb070024812000009abe0094
:108334000292be00208120005001be004000be0019
:108344004110de004f1add0000007200c198de000b
:108354004f99de00cf99de0010079800210798009e
:108364001e009000ae00900021070700707a2a00da
:1083740024060700804980001004b000f4050700bb
:10838400c07a2a001f060700cec2bf006840600002
:108394000004e000a7ff32004e0890000000e00057
:1083a40009003a00804980000000e8008049880004
:1083b4008149800090498000808f50000200350080
:1083c4000000eb008049880040062000c61a070020
:1083d400cd180700500f9800cec2bf006440600063
:1083e4000004e00039003a00c04180000000e000d1
:1083f400360032000afb07001041800000004000f4
:108404004108200080804000008b20000080400054
:1084140010007800e30f500004003a00614d800022
:10842400c0f621006012070003003700614d800090
:10843400108f21005c120700114180000180400070
:108444004208200000014100008b20000000410090
:10845400100078000001e80001804000410820007d
:1084640080804000008b20000080400002087800db
:10847400104180000000400041082000808040003e
:10848400008b20000080400010007800e30f5000b3
:108494000800340010418000000040004108200022
:1084a40080804000008b2000808040000000eb00b2
:1084b40080087800400620008b1a0700cec2bf0057
:1084c400644060000004e000fcff3200cec2bf0044
:1084d400624060000004e00020003a00d0fa070087
:1084e400c04b80000000e00004003a00614d8000b1
:1084f400c0f621002c1207000a003700c04b800090
:10850400e20f500004003a00614d8000108f2100fa
:108514002512070003003700614d8000904f2100b1
:1085240021120700c04b80000000e900c04b880006
:10853400c04b80000000e00002003d00200020004d
:10854400c04b880040062000671a0700cec2bf0057
:10855400624060000004e000fcff320060458000df
:108564000000e000030032000000eb0060458800da
:10857400b2fa07000040eb00e80307004043800024
:10858400001798008e109000e18f500047013200d0
:108594000e119000e20f51006c03320052f90700f3
:1085a40053438000730f98007e0a9000e20f52003c
:1085b400570032007e089000e20f500004003c0097
:1085c400fe089000e18f50004f0032000600370093
:1085d4007e099000e30f51005f003200fe09900015
:1085e400e48f5100920032001041800000004000ee
:1085f4004108200080804000008b20000080400063
:10860400100078000000e00004003a0070c0b300dd
:10861400f4030700f07a2a007a050700104180006d
:10862400000040004108200080804000008b2000b2
:108634000080400010007800e10f500004003a0070
:1086440070c0b300e7030700307b2a006d05070004
:10865400104180000000400041082000808040005c
:10866400008b20000080400010007800e20f5000d2
:1086740004003a0070c0b300da030700707b2a00dc
:108684006005070010418000000040004108200000
:1086940080804000008b20000080400010007800a3
:1086a400e30f500002003a00b07b2a005505070092
:1086b400c04180000000e00003003a00007c2a0072
:1086c400500507005b003700c04b80000000e0004d
:1086d40002003a00507c2a004a050700c04b800083
:1086e400e10f500002003a00a07c2a004505070073
:1086f400c04b8000e20f50004e003a00f07c2a008c
:10870400400507004b00370000f907004900370017
:10871400c04180000000e0000c003a00407d2a00c7
:1087240038050700e04480000000e00003003a0040
:10873400807d2a00330507003e003700e0448000b6
:10874400210020006c0607003a003700e07d2a0073
:108754002c05070037003700a0002000fe19070091
:108764006101b900b0438000c143800002004000b1
:1087740083804800b0438800c1438800d0628000f1
:108784000000e800d0628800d0628000ef0f500043
:10879400280034000000eb00d0628800b043800061
:1087a400c1438000c48bde004c0add004403de00bc
:1087b40006037200e24c8000f34c80000234b800df
:1087c40003b0b90009027800000242000790b90022
:1087d40000024200840478001807980029079800d2
:1087e4006000b800b0438800c14388001e009000b8
:1087f400ae0090004809dd004800de000000710072
:10880400c808de00a043880070c0b30075030700e9
:10881400707e2a00fb040700a04380002100200092
:1088240035060700907e2a00f60407000100370091
:10883400e9f8070000c4b300380307007040800063
:108844000000e00021003a00f4408000054180006f
:108854004fabde00cfb3de000400be00060178009b
:1088640086017800a84c8000b94c80004fcdde0012
:10887400cfd5de000802be000a0378008a03780020
:108884004aea070024812000009abe000292be003a
:10889400208120005001be004000be004110de00d7
:1088a4004f1add0000007200c198de004f99de000f
:1088b400cf99de0010079800210798001e00900051
:1088c400ae009000ca0507000a003700f04080009f
:1088d40001418000809fbe00b07e2a00801f780086
:1088e400008420009bde0700e687570000842000f8
:1088f400c4040700804380000000e00068003a00e0
:10890400804b80000000e00047003200804b800074
:10891400e10f500020003a002441800035418000de
:108924004fabde00cfb3de000400be0006017800ca
:1089340086017800a84c8000b94c80004fcdde0041
:10894400cfd5de000802be000a0378008a0378004f
:1089540016ea070024812000009abe000292be009d
:10896400208120005001be004000be004110de0006
:108974004f1add0000007200c198de004f99de003e
:10898400cf99de00300f9800007f2a009d04070075
:108994003e0890009d050700804b8000e20f5000c8
:1089a4008c023a0044418000554180004fabde0008
:1089b400cfb3de000400be00060178008601780013
:1089c400a84c8000b94c80004fcdde00cfd5de002e
:1089d4000802be000a0378008a037800f3e907005e
:1089e40024812000009abe000292be002081200053
:1089f4005001be004000be004110de004f1add00f1
:108a040000007200c198de004f99de00cf99de00ad
:108a1400300f9800307f2a007a0407003e08900047
:108a24007a0507006b02370080498000e20f50008e
:108a340006003a0090498000e20f500003003a001b
:108a4400607f2a006f04070005003700707a2a004f
:108a54006c040700804980001004b0003c04070047
:108a640070498000e10f500002003a00c07f2a00e4
:108a74006404070070498000e20f500002003a00cd
:108a8400f07f2a005f04070070498000e40f500063
:108a940050023a0020802a005a0407004d02370091
:108aa40050802a00570407004a0237005cf9070087
:108ab4000040eb00990207000bf8070070c0b300f8
:108ac400c8020700d0802a004e04070000c4b30087
:108ad40092020700604380006101b9000080eb004e
:108ae4008080eb0002014000838148001217980047
:108af40023179800b0002000010020001e119000f0
:108b0400ae119000800f5100818f59000f003e007c
:108b14001e109000ae10900000600100200037008d
:108b2400890037009d003700b1003700d6003700b8
:108b3400290137003d013700580137007301370020
:108b440093013700b8013700d9013700ee1607004a
:108b5400500f98005e0890000000e000020034000e
:108b640010002000904b88005e0890000000e00098
:108b740002003d000000eb00904b8800904b800009
:108b84000000e0000300320050812a001d040700a9
:108b94001002370060822a001a0407000d02370011
:108ba400c94b8000c04b800000004000010d200034
:108bb40080804000008b200000804000100478007a
:108bc400a0002000da1607000001540009804400c8
:108bd400010d200080804000008b200000804000b8
:108be40002087800c04b800000004000010d200006
:108bf40080804000008b200000804000100178003d
:108c0400c04b800080004000004a2a0000804000e1
:108c140010007800800f51000c003d00c24b800012
:108c2400c04b800080004000004a2a0000804000c1
:108c34009001780002004100010d20008080400076
:108c4400008b20000080400003087800c04b8000a7
:108c540000004000010d200080804000008b2000b7
:108c64000080400010017800c04b8000800040006c
:108c7400604a2a000080400010007800800f5100f4
:108c84000c003400c24b8000c04b800080004000c8
:108c9400604a2a00008040009001780002004100f0
:108ca400010d200080804000008b200000804000e7
:108cb40003087800c04b80000000e00002003a0086
:108cc40070832a00cf030700c04b8000e10f5000df
:108cd40002003a00b0832a00ca030700c04b800098
:108ce400e20f500002003a00f0832a00c503070097
:108cf40030842a00c3030700c04b800000004000fa
:108d0400010d200080804000008b20000080400086
:108d1400100078006101b900804f2200110020008a
:108d240013e90700809fbe00a0842a00801f7800fa
:108d34000084200087dd0700e687570000842000b8
:108d4400b0030700a30137006f160700500f980007
:108d54005e0890000000e0000200340010002000d3
:108d6400b04b88005e0890000000e00002003d0067
:108d74000000eb00b04b8800b04b80000000e00026
:108d84000300320030852a009e030700910137005a
:108d940040862a009b0307008e0137005a160700fd
:108da400500f98005e0890000000e00002003400bc
:108db40010002000604c88005e0890000000e00075
:108dc40002003d000000eb00604c8800604c800015
:108dd4000000e00003003a0050872a0089030700de
:108de4007c01370060882a00860307007901370078
:108df400484c8000a00020004d16070000004400ed
:108e0400404c8800404c80000000e00002003d001f
:108e14000000eb00404c8800404c8000e30f500001
:108e24000200340030002000404c880070892a0081
:108e340074030700404c80000000e00002003a0088
:108e4400008a2a006f030700404c8000e10f5000a5
:108e540002003a00908a2a006a030700404c80000e
:108e6400e20f500002003a00208b2a00650307003d
:108e7400404c8000e30f500056013a00b08b2a00aa
:108e840060030700530137004a4980005b498000b2
:108e94001d1607006103b900421f8500531f85009a
:108ea4000234b80003b0b90009027800000242009d
:108eb4000790b90000024200840478000a004400cc
:108ec4008b804c0040498800514988004249800009
:108ed40053498000f0d02c0001002000800f510085
:108ee400818f590004003400f0d02c0001002000d0
:108ef4004049880051498800424980005349800014
:108f0400c07e230001002000800f5100818f590092
:108f140004003c00d07e230001002000404988006a
:108f24005149880044498000554980004fabde0018
:108f3400cfb3de000400be0006017800860178008d
:108f4400a84c8000b94c80004fcdde00cfd5de00a8
:108f54000802be000a0378008a03780093e8070039
:108f640024812000009abe000292be0020812000cd
:108f74005001be004000be004110de004f1add006b
:108f840000007200c198de004f99de00cf99de0028
:108f9400300f98003e089000000040006101b900c5
:108fa400000e270021072000aee807006049880072
:108fb4003e089000801f7800408c2a00801f7800b3
:108fc40000842000e3dc0700e487570000842000cd
:108fd4000c030700ff003700cb150700500f980063
:108fe4005e0890000000e000020034001000200041
:108ff400704c88005e0890000000e00002003d0014
:109004000000eb00704c8800704c80000000e00011
:1090140003003200508d2a00fa020700ed003700e9
:10902400608e2a00f7020700ea003700e84b800050
:10903400b51507006a00b90000004400e04b880041
:10904400e14b8000c0442000808f500002003400b7
:10905400c0442000e04b8800e04b80000000e000aa
:1090640002003d000000eb00e04b8800e04b800074
:10907400801f7800708f2a00801f780000842000f1
:10908400b4dc0700e487570000842000dd020700f9
:10909400e04b8000cf0e0700ce003700d84b800095
:1090a400991507006a00b90000004400d04b8800fd
:1090b400d14b8000c0da2000808f500002003400c1
:1090c400c0da2000d04b8800d04b80000000e000c4
:1090d40002003d000000eb00d04b8800d04b800024
:1090e400801f780090902a00801f78000084200060
:1090f40098dc0700e487570000842000c1020700c1
:10910400d04b8000b90e0700b2003700f84b800046
:109114007d15070000004400f04b8800f14b8000ef
:1091240000e12000808f50000200340000e12000a4
:10913400f04b8800f04b80000000e00002003d008e
:109144000000eb00f04b8800f04b80000000e000d2
:1091540005003a000184200092912a0010000900c1
:10916400b258780007003700f04b8000801f780069
:10917400a0922a00801f78000084200075dc07007c
:10918400e4875700008420009e0207009100370006
:10919400584c8000a0002000651507000000440022
:1091a400504c8800504c80000000e00002003d005c
:1091b4000000eb00504c8800504c8000e30f50003e
:1091c4000200340030002000504c8800c0932a0074
:1091d4008c020700504c80000000e00002003a00be
:1091e40050942a0087020700504c8000e10f500081
:1091f40002003a00e0942a0082020700504c8000ea
:10920400e20f500002003a0070952a007d02070028
:10921400504c8000e30f50006e003a0000962a0084
:10922400780207006b003700a000200040150700fb
:10923400000f78001e00e0000f003200804c800018
:109244001e004000804c8800804c80000000e0003c
:1092540002003d000000eb00804c8800804c800040
:10926400e70f50000200340070002000804c88009a
:10927400804c800077110700804c80004300dd00a3
:109284008000780000462a0000804000801f78009b
:1092940090962a00801f7800008420002ddc0700af
:1092a400e487570000842000560207004900370075
:1092b40098498000a00020001d150700000044000c
:1092c4009049880090498000e10f500002003c0062
:1092d400200020009049880090498000fa0f500037
:1092e40002003400a00120009049880081498000d8
:1092f40090498000808f5000020034009049800023
:109304008049880090498000e20f500005003a002f
:109314000384200064972a0010000900b4597800df
:109324000700370090498000801f780070982a0059
:10933400801f78000084200006dc0700e4875700c3
:10934400008420002f020700220037000040eb00b9
:1093540072000700104480002144800002ba2b00f0
:10936400d300200082e70700e1438000801f7800db
:10937400811f780090992a00801f780000842000c3
:10938400f4db0700e6875700008420001d02070075
:1093940000c4b300610007003044800041448000f1
:1093a40002ba2b00d300200071e70700f1438000cc
:1093b400801f7800811f7800409a2a00801f78005f
:1093c40000842000e3db0700e687570000842000c8
:1093d4000c020700504c8000600f9800ee089000cb
:1093e400e18f5000090032006e099000e20f510035
:1093f40008003200ee0990000300e0000100320092
:10940400060037009708070005003700ca04070064
:109414000300370085130700010037008d0907009a
:10942400e1140700cfc2bf000044b2000004e00012
:1094340081f83200faf6070005f707007ef83700d6
:109444000200fa00004f78000900fc00b116800009
:10945400f00f2000008160001e80fb004800dd004a
:109464008000780000f02f00008060000000710090
:10947400b01688001000200087160700d6a2a800a6
:109484001000200084160700d6a2a90010002000b6
:10949400811607000080fa00000006000200fa00ae
:1094a40000002800000f78000400fc0091168000e2
:1094b40000f02f000080700090168800d6c2a8002b
:1094c400d6e2a90009003700100020007216070038
:1094d400d6a2a800200020006f160700a116800065
:1094e40000f02f00008f6000d6a2a9001e007800b3
:1094f4000000e000f4ff3500d6c2a900d6e2a800bf
:109504000400fc0090168000f10f200001006000b0
:10951400901688000080fa00000006000200fa009d
:10952400004f7800ddff0700d6e2a90000c8b300b1
:109534001e407000c2ff0700d6e2a8000080fa00b7
:10954400000006000000fa00d4ff0700d6e2a900dc
:1095540010c0b300baff0700d6e2a8000080fa00ea
:10956400000006000000fa00d6e2a900d6c2a90055
:10957400f00020005c16070080c3b300b0ff0700b2
:10958400500020005816070080c3b300acff07004a
:10959400100020005416070080c3b300a8ff070082
:1095a4001000200050160700c0c0b300a4ff07003d
:1095b400100020004c16070010c0b300a0ff0700e5
:1095c400200020004816070060c0b3009cff07007d
:1095d4001000200044160700d6e2a8000080fa001c
:1095e400000006000200fa00004f7800abff0700fd
:1095f4001e40780092ff07000080fa000000060079
:109604000200fa00004f780011479800a3ff0700fa
:10961400d6e2a900f0c3b3001e4f600000c4b3003b
:109624001e40700086ff0700d6e2a8009bff0700db
:109634001e40900082ff0700c2ff07000080fa006e
:10964400000006000400fa00204798003147980003
:109654000040eb00004f7800040037008fff070044
:109664002e40900076ff07001e4fe8003e40900019
:109674009e4f1000f9ff35000080fa00000006003c
:109684000000fa0085ff0700d6e2a90000c4b30079
:109694006bff0700d6e2a80011c0b3000040eb0046
:1096a400e8ff070051c0b30000c1b300e5ff0700a5
:1096b40021c0b3000040eb00e2ff070011c0b3007b
:1096c4000040eb00dfff070051c0b30040c1b3000e
:1096d400dcff070021c0b3000040eb00d9ff070006
:1096e40011c0b3000040eb00d6ff070051c0b30027
:1096f40050c1b300d3ff070021c0b3000040eb000a
:10970400d0ff070011c0b3000040eb00cdff0700fd
:1097140051c0b30010c0b300caff070021c0b3009a
:109724000040eb00c7ff070011c0b3000040eb008e
:10973400c4ff070051c0b30050c0b300c1ff07000d
:1097440021c0b3000040eb00beff070021c0b300fe
:109754000040eb00bbff070011c0b30000c1b30021
:10976400b8ff070011c0b3000040eb00b5ff0700cd
:1097740011c0b30000c1b300b2ff070031c0b30091
:109784000040eb00afff070031c0b3000040eb0026
:10979400acff070011c0b30000c1b300a9ff07006c
:1097a40041c0b3000040eb00a6ff070021c0b30096
:1097b4000040eb00a3ff070031c0b30000c1b300b9
:1097c400a0ff070031c0b3000040eb009dff07007d
:1097d4005cff07000080fa00000006001200fa0097
:1097e400000f98008e08900000032000808f500026
:1097f4000200340000032000000f98000e089000bf
:1098040062002000110009000200d800200798001f
:109814000e08900062002000110009000200d80028
:109824008000fd00100798000000eb00000f780096
:109834000000eb00300798000c0037001e01780090
:10984400be009000a0162b000080400090407800dd
:109854006800470000004100014878001e0fe8003e
:109864003e0090000000e800300798003e009000a1
:10987400e70f5000f1ff34000000eb00000f780008
:10988400090037009e00780068004700808040008f
:1098940020c0b300804878001e0fe8002e0090001e
:1098a4000000e900200798002e0090000000e0006e
:1098b400f4ff3c001e0090000000e00008003400ab
:1098c4001e0178009e009000e0152b0000804000ef
:1098d400904078006800470000004100014878008b
:1098e4000000eb003007980008003700be0090002d
:1098f40068004700008040001040780039ff0700ee
:109904003e0090000000e800300798003e00900000
:10991400e70f5000f5ff34000080fa000000060055
:109924001600fa00100f9800210f98009e0890006e
:1099340000032000808f5000020034000003200048
:10994400100f980080002000100798001e08900057
:1099540062002000110009000200d80030079800be
:109964001e08900062002000110009000200d800c7
:109974008000fd00200798002e0890000000e00001
:1099840032003a000000eb00000f78000c003700b2
:109994009e0078006a0047008080400020c0b30029
:1099a400804878001e0fe8003e0090000000e900a7
:1099b400300798001e0090000000e900100798008e
:1099c4003e0090000000e000f1ff3c002e009000fb
:1099d4000000e0000c0034001e017800ae0090008e
:1099e400e0152b0000804000904078006a0047009a
:1099f40000004100014878001e0fe8001e0090009e
:109a04000000e900100798000000eb0040079800f0
:109a1400090037009e0078006a00470080804000fb
:109a240000c2b300804878001e0fe8004e0090008a
:109a34000000e80040079800ce0090001e0090004f
:109a4400808f5000f3ff3500310037007000200094
:109a5400000f78000c0037009e0078006a00470071
:109a64008080400020c0b300804878001e0fe900c9
:109a74003e0090000000e900300798001e009000ae
:109a84000000e900100798003e0090000000e0008c
:109a9400f1ff3c002e0090000000e0000c003400b8
:109aa4001e017800ae00900040162b00008040009c
:109ab400904078006a0047000000410001487800a7
:109ac4001e0fe9001e0090000000e9001007980036
:109ad4000000eb0040079800090037009e00780062
:109ae4006a0047008080400000c2b30080487800cc
:109af4001e0fe9004e0090000000e80040079800a7
:109b0400ce0090001e009000808f5000f3ff3500bf
:109b14000000eb004007980008003700ce009000da
:109b24006a0047000080400010407800adfe070046
:109b34004e0090000000e800400798004e0090009e
:109b4400e70f5000f5ff34000080fa000000060023
:109b54000200fa00004f78001e407800a1fe0700c2
:109b64000080fa00000006000400fa002047980074
:109b74002e409000004f78002e4090000080fb00a3
:109b84004400de00204798002e409000e94f50002a
:109b940004003e002e4090000043b000204798008f
:109ba400030037002e4090007043b0002047980017
:109bb4002e4090008bfe07001e407800204798003e
:109bc4002e4090006f406000204798002e40900087
:109bd400e94f500004003e002e4090000043b000c6
:109be40020479800030037002e4090007043b000d7
:109bf400204798002e4090007afe07000080fa006b
:109c0400000006000200fa00000f7800050037008b
:109c14009e0078001140780072fe07001e00780054
:109c2400610f40009e007800114078000004e000bd
:109c3400f7ff3a000080fa00000006000600fa0070
:109c4400008fbe00424798004e4090000004e000a0
:109c540030003a001e00be0002a02c00a3b923006d
:109c640043e507000043b0005efe07001e00be008f
:109c740002a02c00a3b923003de507000003be00a9
:109c840000a02c000032b800a0b9230000b0b90035
:109c9400050178000001410000a02c0000b8b900c3
:109ca40000014100820278001e1f12001e971a0054
:109cb400e0c2b3004bfe07001e00be0002102e00df
:109cc400535f20002ae507000043b00045fe07006b
:109cd4001e00be0002102e00535f200024e5070082
:109ce4000003be0000102e000032b800505f2000b8
:109cf40000b0b900050178000001410000102e00f9
:109d040000b8b90000014100820278001e1f120051
:109d14001e971a004e4090000004e0000e0032002e
:109d2400f0672900810920003e014000ae8148000f
:109d34000200be000001be00e0cf2200111320008b
:109d4400800f5100818f590003003e0000c2b30010
:109d540024fe0700060037001e00be00026829002a
:109d64008309200002e507000043b0001dfe070040
:109d74001e00be000268290083092000fce40700dd
:109d84000003be00006829000032b80080092000ea
:109d940000b0b90005017800000141000068290005
:109da40000b8b90000014100820278001e1f1200b1
:109db4001e971a001e00be0002242400f300200097
:109dc400ebe407000043b00006fe07001e00be00df
:109dd40002242400f3002000e5e407000001be0093
:109de400002424000012b8006f10b90005037800a5
:109df40000034300002424000098b900000343003a
:109e0400860278001e1f12001e971a00e0c2b300db
:109e1400f4fd07001e00be00026a280013002000a3
:109e2400d3e407000043b000eefd07001e00be00af
:109e3400026a280013002000cde407000001be00e0
:109e4400006a28000012b8006110b9000503780008
:109e540000034300006a28000098b900000343008f
:109e6400860278001e1f12001e971a001e00be00f4
:109e74000271220003002000bde407000043b0008b
:109e8400d8fd07001e00be0002712200030020005e
:109e9400b7e407000001be00007122000012b80000
:109ea4006010b9000503780000034300007122002c
:109eb4000098b90000034300860278001e1f1200b8
:109ec4001e971a001e00be00823e200003002000e0
:109ed400a7e407000043b000c2fd07001e00be0057
:109ee400823e200003002000a1e407000001be0020
:109ef400803e20000012b8006010b900050378000d
:109f040000034300803e20000098b9000003430092
:109f1400860278001e1f12001e971a00e0c2b300ca
:109f2400b0fd07001e00be00420620000300200012
:109f34008fe407000043b000aafd07001e00be0026
:109f4400420620000300200089e407000001be004f
:109f5400400620000012b8006010b9000503780024
:109f640000034300400620000098b90000034300aa
:109f7400860278001e1f12001e971a001e00be00e3
:109f8400a20020000300200079e407000043b00091
:109f940094fd07001e00be00a20020000300200064
:109fa40073e407000002be00a00020000023b800f4
:109fb4006020b90007017800000141006a28b90057
:109fc40000014100820378001e1f13001e971b002e
:109fd4004e4090000004e00003003a001e007800a8
:109fe4000043b0007ffd07000080fa000000060077
:109ff4000400fa00008fbe0012c0b3001e00be00b1
:10a004000eff07000080fa00000006000200fa00bc
:10a01400000f78001e00e00002003400b0c2b3005c
:10a0240070fd07001e00e00002003a0000c2b30009
:10a034006cfd07001e00e00003003d00d0c2b30029
:10a0440068fd07001e0fea001e007800823e200013
:10a05400110009000200d8000043b00061fd0700b0
:10a064001e007800823e2000110009000200d80082
:10a0740080007800803e20000088b9001e0f100088
:10a08400e0c2b30057fd07001e007800420620001e
:10a09400110009000200d8000043b00051fd070080
:10a0a4001e00780042062000110009000200d800ba
:10a0b40080007800400620000088b9001e0f1000c0
:10a0c4001e007800a2002000110009000200d80040
:10a0d4000043b00043fd07001e007800a2002000ea
:10a0e400110009000200d8006a00b9001e0f100018
:10a0f4000080fa00000006000400fa00000f780057
:10a1040011079800f07022009e0f10000200340026
:10a11400f0702200000f7800713e20001e80400085
:10a1240080007800e07c2000808f50000f00360013
:10a134001e007800823e2000110009000200d800b1
:10a144000043b00027fd07001e007800823e200077
:10a15400110009000200d80080007800803e200031
:10a164000088b9001e0f10000200370000c2b300bf
:10a174001cfd07001e0078004206200011000900a3
:10a184000200d8000043b00016fd07001e0078004e
:10a1940042062000110009000200d8008000780067
:10a1a400400620000088b9001e0f10001e00900019
:10a1b400e20f5000040032009e009000700720005f
:10a1c400808f500002003a00e0c2b30005fd070092
:10a1d4001e007800a2002000110009000200d8002f
:10a1e4000043b000fffc07001e007800a20020001e
:10a1f400110009000200d8006a00b9001e0f100007
:10a204001e009000e10f500002003a00e0c2b300cb
:10a21400f4fc07009e00900070072000808f50001f
:10a2240003003a0070c5b300eefc070003003700da
:10a234001e0078000043b000eafc07000080fa002a
:10a24400000006000200fa00004f780090c0b3003e
:10a254009e4f10000200340090c0b300004f7800fd
:10a2640001c3b3001ec04000defc07000080fa00fa
:10a27400000006000c00fa00a24c8000b34c8000e1
:10a2840000b0260051542f00020040008380480093
:10a294004007980051079800ce0090008095230055
:10a2a4000009b8004e0090000000d00003027800be
:10a2b40000024200de009000809523000088b9006f
:10a2c4000002420084017800028fbe004f98de0035
:10a2d400cf80de0020079800300798003e00be00c3
:10a2e4002e01be004800de00480add0000007200b6
:10a2f400c808de004812dd00810072004811de004b
:10a30400481add0002017200c899de00009fbe00f9
:10a314000297be0014ee2d0055c62d0076012000d4
:10a32400070020003e00be002e01be0000005200c7
:10a3340081805a0002015b0083815b0064c22000bb
:10a34400009abe000292be000080fa0000000600df
:10a354000c00fa000040eb003aecb70036ccbf002a
:10a364000080fb004400de000080fb0001002000b0
:10a374004007980051079800ce009000a0002000ec
:10a38400000ab8004e0090006000b9000501780092
:10a39400000141005e0090006a00b9000001410024
:10a3a4008202780036ccbf000080fb000100200050
:10a3b4006f0160006000b80003002000020070001c
:10a3c40083807000040040008580480040079800a6
:10a3d40051079800ce009000a0002000000ab800a9
:10a3e4004e0090006000b9000501780000014100b2
:10a3f4005e0090006a00b90000014100820278000a
:10a4040037ccbf000080fb004400de000080fb006e
:10a4140001002000040040008580480040079800a7
:10a4240051079800ce009000a0002000000ab80058
:10a434004e0090006000b900050178000001410061
:10a444005e0090006a00b9000001410082027800b9
:10a4540037ccbf000080fb00010020006f016000ca
:10a464006000b800030020000200700083807000c8
:10a474000400400085804800400798005107980078
:10a48400ce009000a0002000000ab8004e0090000a
:10a494006000b90005017800000141005e009000f1
:10a4a4006a00b900000141008202780038ccbf0084
:10a4b4000080fb004400de000080fb00010020005f
:10a4c4000400400085804800400798005107980028
:10a4d400ce009000a0002000000ab8004e009000ba
:10a4e4006000b90005017800000141005e009000a1
:10a4f4006a00b900000141008202780038ccbf0034
:10a504000080fb00010020006f0160006000b800c3
:10a5140003002000020070008380700004004000eb
:10a52400858048004007980051079800ce009000ad
:10a53400a0002000000ab8004e0090006000b9009e
:10a5440005017800000141005e0090006a00b90036
:10a55400000141008202780039ccbf000080fb007a
:10a564004400de000080fb000100200004004000e5
:10a57400858048004007980051079800ce0090005d
:10a58400a0002000000ab8004e0090006000b9004e
:10a5940005017800000141005e0090006a00b900e6
:10a5a400000141008202780039ccbf000080fb002a
:10a5b400010020006f0160006000b800030020006b
:10a5c4000200700083807000040040008580480011
:10a5d4004007980051079800ce009000a00020008a
:10a5e400000ab8004e0090006000b9000501780030
:10a5f400000141005e0090006a00b90000014100c2
:10a604008202780044079800550798004e00900095
:10a61400de00900065004000e0804800400798009c
:10a62400510798004e019000de01900000a0250023
:10a6340021262000800f5100818f5900040036002c
:10a6440000a025002126200040079800510798000b
:10a654004e009000de0090000001eb008001eb0052
:10a6640064c220005403be004402be00cfe20700cf
:10a67400009fbe000297be00144180003e00be0051
:10a684002e01be004f08de00c112dd000080720002
:10a69400cf10de00c11add00818072004f99de0008
:10a6a400cf99de000001be00c220dd00008b200037
:10a6b400008040000288be000080fa00000006000e
:10a6c4000200fa000000eb00000f780006003700db
:10a6d4009e007800e0c22000808040000040eb0033
:10a6e400804878001e0fe800400020009e0f1000f4
:10a6f400f7ff34000080fa00000006000200fa00b0
:10a704000000eb00000f7800060037009e00780080
:10a71400e0c2200000804000104078005c0c07007c
:10a724001e0fe800400020009e0f1000f7ff3400c9
:10a734000080fa00000006001400fa00889fbe00a2
:10a744008a9fbe003accbf000004e000040032003f
:10a7540020608000e10f400001003a00fcfe070089
:10a76400206080000000e00005003a000000eb00db
:10a77400a0618800d2ff07000080eb002060880001
:10a784004f0c07000000e000ea013200800c2000ba
:10a7940020608800a06180000000e00002003d000d
:10a7a4000000eb00a0618800a0618000e40f50006d
:10a7b4000200340040002000a0618800a8618000ed
:10a7c4004f0c070080407800e0c2200000004400e5
:10a7d40001487800a06180000000e800a0618800c2
:10a7e400a0618000e40f5000d20134000000eb00af
:10a7f400a061880032ccbf000080fb00100f9800dd
:10a80400000820009e089000808f5000c001320094
:10a81400000820001e0a9000800f520017003c0020
:10a824001e089000e20f50005e0132009e08900066
:10a83400e28f500007003c001e0a90000400e00074
:10a84400ae0132001e089000e10f50008a01320070
:10a85400270037009e089000e78f500074013200f3
:10a864001e0a9000e80f52009c0132001e0890005e
:10a87400e30f5000220032001d0037008008200042
:10a884009e089000808f50009801320080082000bc
:10a894001e0a9000800f520009003c00100820009e
:10a8a4009e089000808f5000530132002008200041
:10a8b4001e0a9000800f5200440132000c00370041
:10a8c400700e20009e089000808f5000f900320026
:10a8d400700f20001e0a9000800f52000e013200fb
:10a8e400b00b20009e089000808f50008d01320034
:10a8f40073ff070000cfb300e50b07008d0137009d
:10a904006fff0700d4408000e54080004fabde00bd
:10a91400cfb3de000400be00060178008601780093
:10a92400a84c8000b94c80004fcdde00cfd5de00ae
:10a934000802be000a0378008a0378001be20700bd
:10a9440010079800210798003207980043079800e1
:10a954001e009000ae0090003e019000ce019000d9
:10a964004110de004f1add0000007200c198de00c5
:10a974004f99de00cf99de005007980061079800d8
:10a984000040eb002eecb7002eccbf004404dd00e9
:10a994005e009000ee009000026829008309200008
:10a9a40030e20700004044002eecb7005e00900047
:10a9b400ee009000026829008309200029e20700c4
:10a9c4000002be00006829000023b80080092000ae
:10a9d40000a0b900070178000001410000682900c7
:10a9e40000a8b90000014100820378005e009000d5
:10a9f400ee00900006005000878058005007980031
:10aa0400610798005e009000ee009000022424008c
:10aa1400f300200013e207002fecb7005e00900063
:10aa2400ee00900002242400f30020000de2070051
:10aa34000001be00002424000013b8006f10b90008
:10aa44000702780000024200002424000098b900a4
:10aa540000024200840378005e009000ee00900043
:10aa6400060050008780580050079800610798003e
:10aa74002fccbf004404dd005e009000ee00900087
:10aa8400026a280013002000f6e107000040440099
:10aa94002fecb7005e009000ee009000026a2800e0
:10aaa40013002000efe107000001be00006a280047
:10aab4000013b8006110b9000702780000024200d8
:10aac400006a28000098b90000024200840378005c
:10aad4005e009000ee009000060050008780580051
:10aae40050079800610798005e009000ee00900007
:10aaf4000271220003002000dae1070030ecb70005
:10ab04005e009000ee00900002712200030020001d
:10ab1400d4e107000001be00007122000013b80058
:10ab24006010b900070278000002420000712200a0
:10ab34000098b90000024200840378005e0090008f
:10ab4400ee009000060050008780580050079800df
:10ab54006107980030ccbf004404dd005e00900023
:10ab6400ee009000823e200003002000bde10700bb
:10ab74000040440030ecb7005e009000ee0090000e
:10ab8400823e200003002000b6e107000001be0061
:10ab9400803e20000013b8006010b900070278005e
:10aba40000024200803e20000098b90000024200ea
:10abb400840378005e009000ee00900006005000d0
:10abc4008780580050079800610798005e00900045
:10abd400ee0090004206200003002000a1e10700df
:10abe40031ecb7005e009000ee00900042062000b9
:10abf400030020009be107000001be004006200086
:10ac04000013b8006010b900070278000002420087
:10ac1400400620000098b900000242008403780036
:10ac24005e009000ee0090000600500087805800ff
:10ac3400500798006107980031ccbf004404dd0040
:10ac44005e009000ee009000a200200003002000af
:10ac540084e107000040440031ecb700104180005b
:10ac6400000040004108200080804000008b20004c
:10ac74000080400010007800e20f500009003c0002
:10ac84001041800000004000410820008080400006
:10ac9400008b2000008040001000780032ecb700e8
:10aca400020037000040eb0032ecb70093fe0700cf
:10acb400a000370082fe0700c04180000000e000d1
:10acc40010003200d043800032002000110009003f
:10acd4000200d800004f7800f0c0b3009e4f10006f
:10ace40002003600f0c0b300004f780040458000f9
:10acf4000000e0000500320000c8b3001e4f7000e1
:10ad04000200370000c0eb00004f78001e407800be
:10ad1400df0a07008700370069fe0700c041800092
:10ad24000000e0001a003a001045800032002000c4
:10ad3400110009000200d800004f7800f1c0b300f0
:10ad44009ecf100002003600f0c0b300004f780020
:10ad540000c8b3001e4f7000f04480000000e00003
:10ad64000200320000c4b3001e4f7000804980000e
:10ad7400e20f500008003a0090498000e20f5000b2
:10ad840005003a0000c2b3001e4f700002003700f5
:10ad940000c0eb00004f78001e407800bc0a07009a
:10ada4006400370080498000206188009049800059
:10adb400e20f500002003a00200020008049880081
:10adc4000040eb00b20a07005a00370020618000ff
:10add400e10f500003003c0020618000804988009e
:10ade400020037000000eb00804988000040eb00bf
:10adf400a70a07004f00370090498000e20f500077
:10ae040008003a00804980000000e000030032009e
:10ae14000000eb0080498800020037001000200089
:10ae2400804988000040eb00990a07004100370080
:10ae34002eccbf00e24f50000c003e0011418000b8
:10ae44002eccbf000081fb0001804000410820009f
:10ae540080804000008b20000080400002087800c1
:10ae64000040eb008a0a07003200370000cfb3002d
:10ae7400870a07002f0037000000eb00000f98003e
:10ae8400100037000e0990008e089000e0c22000e8
:10ae9400008040009040780060c320000000410022
:10aea400014878008e089000e0c2200080804000b5
:10aeb4000040eb00804878000e0890000000e80095
:10aec400000f98000e089000e40f5000edff3400ce
:10aed4000040eb006e0a070016003700cae2a80023
:10aee4000040eb006a0a070012003700cae2a9001a
:10aef4000040eb00660a07000e0037001000200037
:10af0400804388000040eb00610a07000900370015
:10af14000000eb00804388000040eb005c0a07005f
:10af2400040037000040eb00590a07000040eb0022
:10af3400570a07004f05be004f04be000080fa0008
:10af4400000006000600fa00881f78001007980029
:10af54002107980070c0b300004f78000040eb0058
:10af640010479800160037001e04fb001e009000d6
:10af7400ae009000a200200003002000c9e00700fa
:10af840002c3b3008240400080c12000000044009e
:10af9400014878001e009000ae009000a20020003e
:10afa40003002000afe00700100798002107980075
:10afb4001e4fe9001e4090000040e8001047980032
:10afc4001e409000e74f5000e7ff34000040eb00c4
:10afd40020ecb7004f0478000080fa00000006005f
:10afe4000400fa00008fbe001e00be00d5ff07005b
:10aff40018ccbf00260a070019ccbf00240a07009a
:10b004001accbf00220a07001bccbf00200a07008d
:10b014001cccbf001e0a07001dccbf001c0a070081
:10b024001eccbf001a0a07001fccbf00180a070075
:10b034000080fa00000006000600fa00200020004c
:10b04400000f78006000b8001007980021079800ee
:10b054001b0037009e009000a0002000000ab800ea
:10b064001e0090006000b900050178000001410055
:10b074002e0090006a00b9000001410082027800ad
:10b084009e007800a0c0200000804000104078009e
:10b094000000fb00cf80de006f0160006000b8009c
:10b0a4000300200002007000838070000400400050
:10b0b4008580480010079800210798001e0fe800bb
:10b0c400b06080009e0f1000e2ff35001e0090006b
:10b0d400ae0090000080fa00000006000200fa00b2
:10b0e40080418000008fe9001e00e00002003d0066
:10b0f4000000eb00000f78001e007800801f78002d
:10b10400e00e2b00801f7800b0d40700e4875700be
:10b114000080fa00000006000000fa00c041800030
:10b124000000e00007003a0010458000801f78000e
:10b13400500f2b00801f7800a4d40700e487570029
:10b1440006003700d0438000801f7800500f2b008a
:10b15400801f78009dd40700e48757000080fa0020
:10b16400000006000000fa001041800000004000ca
:10b174004108200080804000008b200000804000b7
:10b1840010007800801f7800c00f2b00801f78000b
:10b194008ed40700e48757000080fa000000060000
:10b1a4000000fa0080498000801f780030102b00d6
:10b1b400801f780085d40700e48757000080fa00d8
:10b1c400000006000c00fa00889fbe008a9fbe00a3
:10b1d400f4408000054180004fabde00cfb3de00b9
:10b1e4000400be000601780086017800a84c8000a7
:10b1f400b94c80004fcdde00cfd5de000802be0082
:10b204000a0378008a037800e8df0700009fbe0085
:10b214000297be003e00be002e01be004110de00bb
:10b224004f1add0000007200c198de004f99de0065
:10b23400cf99de004007980051079800a0102b001a
:10b24400801f780061d407008f87e9004e009000ca
:10b25400de00900062ff0700d0102b00801f7800f2
:10b264005ad407008f87e9004f05be004f04be0083
:10b274000080fa00000006000000fa00c04b8000c5
:10b28400801f780000112b00801f78004fd4070026
:10b29400e48757000080fa00000006000000fa006e
:10b2a400c04b800000004000010d20008080400061
:10b2b400008b200000804000100078006101b9007c
:10b2c400804f220011002000a9df0700809fbe00ec
:10b2d40070112b00801f78003cd40700e6875700cc
:10b2e4000080fa00000006000000fa00804b800095
:10b2f400801f7800f0112b00801f780033d40700e2
:10b30400e48757000080fa00000006000000fa00fd
:10b31400c04180000000e00005003a0060122b00ec
:10b32400801f780029d407008f87e90004003700c4
:10b33400c0122b00801f780024d407008f87e900f7
:10b344000080fa00000006000c00fa003aff070033
:10b3540040079800510798004e009000de009000ce
:10b3640065004000e08048004007980051079800bd
:10b374004e019000de01900000a02500212620004f
:10b38400800f5100818f59000400360000a0250071
:10b394002126200040079800510798004e00900095
:10b3a400de0090000001eb008001eb0064c220008d
:10b3b4005403be004402be007cdf0700009fbe00b1
:10b3c4000297be00144180003e00be002e01be0064
:10b3d4004f08de00c112dd0000807200cf10de00d5
:10b3e400c11add00818072004f99de00cf99de0022
:10b3f4000001be00c220dd00008b20000080400060
:10b404000288be000080fa00000006000200fa0074
:10b414000cccbf000000fb006f0f60002000200078
:10b424009e0f10000200340020002000000f78005e
:10b434001e007800c04b88000080fa00000006005f
:10b444000200fa00881f7800fbfe0700000f780056
:10b45400c84b80001e0078006101b900804f2200b3
:10b464001100200042df07000001780008004400ba
:10b47400010d200080804000008b200000804000ef
:10b4840002087800c04b800000004000010d20003d
:10b4940080804000008b2000008040001001780074
:10b4a400c04b800080004000004a2a000080400019
:10b4b40010007800800f51000c003d00c24b80004a
:10b4c400c04b800080004000004a2a0000804000f9
:10b4d4009001780002004100010d200080804000ae
:10b4e400008b20000080400003087800c04b8000df
:10b4f40000004000010d200080804000008b2000ef
:10b504000080400010017800c04b800080004000a3
:10b51400604a2a000080400010007800800f51002b
:10b524000c003400c24b8000c04b800080004000ff
:10b53400604a2a0000804000900178000200410027
:10b54400010d200080804000008b2000008040001e
:10b55400030878004f0478000080fa000000060019
:10b564000200fa000cccbf000000fb006f0f60006b
:10b57400100020009e0f1000020034001000200074
:10b58400000f78001e007800804b88000080fa00cd
:10b59400000006000200fa00c1c0200091407800bb
:10b5a40010c3b30080cf500002003a00cae2a800e2
:10b5b40001003700cae2a9000080fa00000006007a
:10b5c4000200fa000000eb00000f780006003700cc
:10b5d4009e007800a0c02000808040000040eb0066
:10b5e400804878001e0fe800b00020009e0f100075
:10b5f400f7ff34000000eb00b06088000080fa0020
:10b60400000006000400fa00004f78001e04e00069
:10b614000c003200a0c0b3009e4f1000090032009d
:10b6240000c2b3009e4f100006003200c0c2b30037
:10b634009e4f100003003200e0c2b3009e4f100082
:10b6440003003a00100020001007980002003700a1
:10b654000000eb00100798001e0090000080fa0024
:10b66400000006000a00fa00814180001061800099
:10b67400808f500008003200306080000000e0003d
:10b6840005003a00400620003060880080418000b8
:10b694001061880091fe0700890807000000e0009f
:10b6a400ba00320096080700204798002e40900008
:10b6b400d4ff07000000e000b4003a00ae40900060
:10b6c400d0c3b30080cf500004003200ae409000dd
:10b6d400f0c3b30080cf500001003a00b8ff070068
:10b6e4002e409000ed4f50009d003a000accbf0060
:10b6f4000000fb0040079800d0032000ce0090001b
:10b70400808f50004a003200f0032000ce009000e9
:10b71400808f5000010032008f0037000bccbf0037
:10b724000000fb003007980020052000be009000b8
:10b73400808f50003900320020052000be009000a8
:10b74400808f500016003c0020042000be009000b2
:10b75400808f50002300320020042000be0090009f
:10b76400808f500005003c0010042000be009000b3
:10b77400808f5000250032002b0037006004200029
:10b78400be009000808f50001e003200d0042000c4
:10b79400be009000808f5000160032002200370057
:10b7a40040052000be009000808f50001d00320034
:10b7b40040052000be009000808f50000b00350033
:10b7c40060052000be009000808f50000b00320006
:10b7d40070052000be009000808f50000d003200e4
:10b7e400110037003dfe07000f0037004afe070036
:10b7f4000d0037005bfe07000b00370068fe0700f2
:10b80400090037006ffe0700070037009afe0700a3
:10b8140005003700a1fe070003003700b2fe070051
:10b8240001003700b9fe070065ff07005700370025
:10b834000bccbf000000fb0020079800200520006f
:10b84400ae009000808f50003e00320020052000a2
:10b85400ae009000808f50000d003c00600420007a
:10b86400ae009000808f500030003200d0042000e1
:10b87400ae009000808f50001200320010042000af
:10b88400ae009000808f50002a0032003000370054
:10b8940060052000ae009000808f50001900320037
:10b8a40070052000ae009000808f5000230032000d
:10b8b40040052000ae009000808f5000230032002d
:10b8c400230037000cccbf000000fb006f0f6000aa
:10b8d400300020009e0f10000200340030002000d1
:10b8e400000f780010418000000040004108200053
:10b8f40080804000008b2000008040001e087800fb
:10b9040013003700ccfd0700000f780091012000e0
:10b914009e8f10000200340090012000000f780078
:10b924001e007800804988000900370086fe070061
:10b9340007003700b5fe070005003700c0fe07000a
:10b944000300370006ff07000100370011ff07005e
:10b954001bff07000d00370019ff07000b0037001d
:10b96400b1608000a0c0200000804000ae40900084
:10b9740001487800b0608000ea0f500003003c00ea
:10b98400b06080000000e800b06088000080fa0029
:10b99400000006000600fa00009b2a00801f7800c1
:10b9a4008ad207008f87e9000000eb001007980097
:10b9b4001c0037009e00900000002f000080400013
:10b9c400800078006401470013002000f007200085
:10b9d400750c0700000f78001e0090006f006000d7
:10b9e4000000e00006003a001e009000801f78006e
:10b9f400709c2a00801f780074d20700e4875700e7
:10ba04002e009000801f7800f09c2a00801f780090
:10ba14006ed20700e48757001e0090000080e80003
:10ba2400100798009e009000f01f2000808f5000a7
:10ba3400e0ff34001e007800801f7800409d2a003b
:10ba4400801f780061d20700e48757000080fa0065
:10ba5400000006001000fa00990707000000e0004b
:10ba64000a023200a6070700004f78001e80fb0080
:10ba74006101b900f0fd2f00f1ff2f000201400029
:10ba840083814800620798007307980030052000fe
:10ba9400010020006e019000fe019000800f510013
:10baa400818f5900ef013e006e009000fe0090006f
:10bab4000060010011013700ea013700e901370095
:10bac400e8013700e7013700e6013700e5013700f8
:10bad400e4013700e3013700e20137005701370082
:10bae400e001370076013700de013700dd01370061
:10baf4009d013700be013700bd013700bc0137008e
:10bb0400bb013700ba013700b9013700d50137004e
:10bb1400d4013700a5013700d2013700d101370025
:10bb2400d0013700cf013700ce013700cd013700f7
:10bb3400cc01370044003700ca01370057003700f2
:10bb4400fb00370053003700c6013700c50137003a
:10bb5400c40137002b003700c2013700c101370090
:10bb6400c0013700bf013700be013700bd013700f7
:10bb7400bc013700bb013700ba0137009e00370013
:10bb8400b8013700b7013700b60137005400370059
:10bb9400b4013700b3013700a6013700b101370003
:10bba400b0013700af013700ae013700ad013700f7
:10bbb400ac013700ab0137005f00370010013700dc
:10bbc4009d003700a70137005e013700a50137004b
:10bbd400a4013700a3013700a2013700a1013700f7
:10bbe400a0013700f80037009e013700ee0037004f
:10bbf400880037009b0137009a013700770037002f
:10bc0400f8003700e09e2a00801f7800efd107007b
:10bc14008f87e90050a12a00801f7800ebd107002c
:10bc24008f87e900e03b2a00801f7800e7d10700f6
:10bc34008f87e90090a22a00801f7800e3d10700d3
:10bc44008f87e90091013700900020004007980099
:10bc54000c0037004e009000bf0c0700801f7800d6
:10bc6400ce009000811f7800e0a42a00801f780095
:10bc7400d6d10700e68757004e0090000000e80088
:10bc8400400798004e009000ef0f5000f1ff340081
:10bc94007e0137003fff07007c013700c0a52a0062
:10bca400801f7800c9d107008f87e9000000eb00ee
:10bcb4005007980012002000e11f2f00f007200019
:10bcc400c60b07006a00470013002000e21f2f0084
:10bcd400f1072000e20b07002eff07006b0137007d
:10bce400b0a72a00801f7800b8d107008f87e90029
:10bcf4000d003700f20607000000e000fdff3200ef
:10bd0400ff060700004f78001e80fb00801f7800ac
:10bd140070a82a00801f7800acd10700e487570080
:10bd24001e80fb008af70700b2c1b3009e4f1100ca
:10bd3400f0ff3a005501370030a92a00801f78002f
:10bd4400a2d107008f87e9000040eb00004f780084
:10bd5400fcf507000000eb004007980009003700dd
:10bd64000040eb00edf507004e0090009bf6070045
:10bd7400200320005c0c07004e0090000000e80047
:10bd840040079800ce009000f0052000808f5000fe
:10bd9400f3ff340000c4b300e0f507001e80fb008d
:10bda4009e80fb00801f7800811f780040ab2a0032
:10bdb400801f78000084200066d10700e6875700c2
:10bdc400008420008ff707001e4fe800bc06070020
:10bdd4000000e0002d013a00deff370000ac2a002d
:10bde400801f780079d107008f87e90010002000b8
:10bdf400904388002501370070ac2a00801f78002a
:10be040072d107008f87e9000000eb00904388009f
:10be14001e01370020458000d1438000801f780038
:10be2400811f780020ad2a00801f780067d10700a9
:10be3400e68757001501370080498000801f78008d
:10be4400c0ae2a00801f780060d10700e487570045
:10be540010418000801f7800a0b02a00801f780065
:10be64005ad10700e48757001041800000004000c9
:10be74004108200080804000008b200000804000aa
:10be840010007800801f7800a0b12a00801f78007d
:10be94004ed10700e4875700c0498000801f780016
:10bea400e0b32a00801f780048d10700e4875700d8
:10beb400a0418000801f7800c0b52a00801f780050
:10bec40042d10700e4875700b0418000801f78000a
:10bed400e0b62a00801f78003cd10700e4875700b1
:10bee400c0418000801f7800e0b72a00801f7800de
:10bef40036d10700e4875700e4003700d0b82a00a1
:10bf0400801f780031d107008f87e9007c06070085
:10bf1400004f78001e4078005d0607009e80fb00fd
:10bf240000fd2f0000804000c0498800d700370082
:10bf340084f507000040eb00004f7800160037003e
:10bf44005f0607000000e000080032006c060700ee
:10bf5400004f78001e407800d00a07000040eb0034
:10bf64006ef507001e80fb00f9f60700e40a0700df
:10bf74000000e00008003200f10a0700004f7800da
:10bf84001e4078004206070000c4b30063f50700b2
:10bf94001e80fb00eef60700b3c1b3009ecf110074
:10bfa400e7ff3a00b9003700a04c8000b14c800094
:10bfb400809fbe00d0ba2a00801f780003d10700fa
:10bfc400e6875700b1003700f0020700801f7800b1
:10bfd40030bc2a00801f7800fcd00700e48757009b
:10bfe400aa00370070bd2a00801f7800f7d0070030
:10bff4008f87e90010502500840b0700a300370049
:10c0040000be2a00801f7800f0d007008f87e90067
:10c014001e0090000000e800100798001e00900029
:10c024007a0b0700a0002000af0b070024060700ce
:10c034000000e00095003a00f5ff370082418000df
:10c04400fa00410040992000008040001040780030
:10c054008041e800fa00410040992000008040003f
:10c06400034878008341800080418000fa0040004a
:10c074004099200000804000104078006341600037
:10c08400fa80410040992000008040000248780076
:10c0940080418000fa004000409920000080400068
:10c0a400104078000080fb00801f7800e0be2a006a
:10c0b400801f7800c5d00700e4875700730037005d
:10c0c40082418000fa004100409920000080400035
:10c0d400104078008041e900fa00410040992000b6
:10c0e4000080400003487800834180008041800044
:10c0f400fa00400040992000008040001040780081
:10c1040063416000fa8041004099200000804000b3
:10c114000248780080418000fa00400040992000e5
:10c1240000804000104078000080fb00801f7800f1
:10c13400e0be2a00801f7800a4d00700e4875700df
:10c1440052003700004e800081418000801f78003b
:10c15400811f780050c02a00801f78009bd0070000
:10c16400e687570049003700504080000000e00097
:10c1740007003a0020c32a00801f780093d00700ec
:10c184008f87e90010002000504088003f003700ee
:10c1940050c42a00801f78008cd007008f87e900e4
:10c1a4000000eb00504088003800370070408000e9
:10c1b4000000e00007003a0090c52a00801f7800c4
:10c1c40082d007008f87e9001000200070408800ab
:10c1d4002e00370030c72a00801f78007bd007006c
:10c1e4008f87e9000000eb007040880027003700cb
:10c1f4001e80fb006f0060000000e90060408800c2
:10c2040060408000c200dd00003d2a000080400044
:10c214001000be0062408000809fbe00821f780034
:10c22400e0c82a00801f780068d00700e88757001c
:10c2340016003700b0ca2a00801f780063d00700b8
:10c244008f87e9000000eb00400798002e00900063
:10c254004e019000110009000200d8002007980048
:10c264000a0037001e80fb00801f780090cb2a0054
:10c27400801f780055d00700e487570060cc2a005f
:10c28400801f780051d007008f87e9000080fa00f2
:10c29400000006004000fa00889fbe008a9fbe008e
:10c2a40080498000c200dd00008b20000080400037
:10c2b4001001be0062079800730798006e0090009a
:10c2c400fe009000a20a07006e009000fe0090009d
:10c2d4004f8ade00cfa2de006e009000fe009000c8
:10c2e4000401780084017800a84c8000b94c8000d7
:10c2f4004fcdde00cfd5de000802be000a03780071
:10c304008a037800a9db070020079800310798000a
:10c3140042079800530798002e009000be0090003a
:10c324004e019000de0190004110de004f1add0046
:10c3340000007200c198de004f99de00cf99de0044
:10c34400000f9800110f98000000eb00400f9800b8
:10c354007cf407006e009000fe009000809fbe00f9
:10c364000e0990009e099000829fbe00c0cd2a0055
:10c37400801f780015d00700ea87570040d12a00b3
:10c38400801f780011d007008f87e9000000370074
:10c39400c8c2bf000044b2000004e0000400320040
:10c3a40010002000c0418800ca62a90003003700c1
:10c3b4000000eb00c0418800ca62a800d000200041
:10c3c400e50a0700e0438800c0002000e20a0700f5
:10c3d400f0438800e04380006104b900e04380003a
:10c3e4006101b9000243b80003c0b9000702780034
:10c3f400000242000990b900000242008403780060
:10c404001644880027448800f04380006104b90082
:10c41400f04380006101b9000243b80003c0b900d1
:10c4240007027800000242000990b90000024200ad
:10c43400840378003644880047448800124480000e
:10c4440023448000304480004144800000005100b7
:10c4540081805900504488006144880015ea07002f
:10c46400c3c2bf000042b2000004e00012003a0060
:10c474004e0890000000e800400f98004e0890001d
:10c48400e60f5000020034000000eb00400f98005b
:10c4940021032000e055220043020700c3c2bf006d
:10c4a4000042b2000004e000fcff3200400620001d
:10c4b4008d0a070094080700ce099000731f9800a6
:10c4c4007e1a9000e30f5200d90032007e189000cb
:10c4d400e30f500007003c00fe189000e18f50006d
:10c4e400600032007e199000e20f5100a900320072
:10c4f40009003700fe199000e58f51000301320056
:10c504007e1a9000e50f5200e40035007e1890007a
:10c51400e60f5000180132000040eb00fff3070063
:10c52400b0d42a00b7f5070000c4b300fbf307003a
:10c5340075080700500f98005e0890000000e000a6
:10c544003c003200a24c8000b34c80005e08900096
:10c55400cf80de000200400083804800a04c8800a9
:10c56400b14c8800a04c8000b14c800050db070027
:10c574000001be00000020000100250077db070059
:10c58400008fbe000e0890009e089000e00f50003f
:10c59400e08f5800060035000e0890009e089000b9
:10c5a40043db0700501f9800611f980017003700f5
:10c5b4000e0890009e089000610160006000b800c1
:10c5c4000300200002007000838070000e099000b8
:10c5d4009e0990008301d1000281d3000200700003
:10c5e4008380700032db0700501f9800611f9800a1
:10c5f4005e199000ee1990005e189000ee189000fd
:10c6040099db0700501f9800611f98001e01be00af
:10c614005e189000ee189000f0db070023dc0700a2
:10c6240060079800710798006e009000fe0090006b
:10c63400c7090700a04c8000b14c80007c01470072
:10c64400809fbe00c0d52a00801f780002007800b9
:10c6540040cf0700e68757007c00470069f50700d4
:10c66400cd0037000040eb00acf30700a000200031
:10c67400390a07006104b900e04c8000f14c8000e5
:10c684000001be000243b80003c0b90007027800ed
:10c69400000242000990b9000002420084037800bd
:10c6a400260f9800370f98002e089000be089000bf
:10c6b4004809dd004800de0000007100c808de0003
:10c6c400a043880070d62a004ef50700a0438000de
:10c6d4002100200088f6070000d72a0049f507004a
:10c6e40000c4b3008df30700e84c8000f94c8000cf
:10c6f400500020000e080700cf80de000800400034
:10c7040089804800e04c8800f14c8800e24c8000ad
:10c71400f34c80003006200001002000800f5100ff
:10c72400818f590004003c004006200001002000d5
:10c73400e04c8800f14c8800e24c8000f34c80000f
:10c74400800c200001002000800f5100818f5900cf
:10c7540004003400800c200001002000e04c88001c
:10c76400f14c8800e04c8000f14c80007c014700d3
:10c77400809fbe0040d72a00801f78000200780006
:10c78400f4ce0700e68757007c0047001df507003c
:10c79400810037000040eb0060f307007c00470095
:10c7a40073d82a0010000900335878001001b10032
:10c7b4007c00470013f5070000c4b30057f30700db
:10c7c400684d800050002000d90707006500b900bb
:10c7d40000004400604d8800604d80000000e000cf
:10c7e40002003d000000eb00604d8800614d8000b8
:10c7f40040062000808f50000200340040062000d4
:10c80400604d8800604d8000fc004700801f780068
:10c8140080d92a00801f780001007800cdce07005f
:10c82400e48757007c004700f6f407005a003700fd
:10c834000040eb0039f307007fe8070090da2a0094
:10c84400f0f4070000c4b30034f30700084d80007f
:10c85400194d8000ac070700cf80de0008004000bf
:10c8640089804800004d8800114d8800004d8000eb
:10c87400114d80007c014700809fbe0010db2a0020
:10c88400801f780002007800b2ce0700e6875700c8
:10c894007c004700dbf407003f0037000040eb005a
:10c8a4001ef3070020dc2a00d6f4070097e80700ef
:10c8b40000c4b30019f30700484d8000594d8000af
:10c8c400500020009a070700cf80de0008004000d7
:10c8d40089804800404d8800514d8800404d8000bb
:10c8e400514d80007c014700809fbe0040d72a0044
:10c8f400801f78000200780096ce0700e687570074
:10c904007c004700bff40700230037000040eb0021
:10c9140002f30700b0dc2a00baf40700aee807000f
:10c9240000c4b300fdf20700c84c8000d94c80005d
:10c9340075070700cf80de000800400089804800aa
:10c94400c04c8800d14c8800c04c8000d14c800081
:10c954007c014700809fbe0010db2a00801f780006
:10c96400020078007bce0700e68757007c00470072
:10c97400a4f40700080037000040eb00e7f20700ca
:10c9840040dd2a009ff4070000c4b300e3f207006f
:10c9940050de2a009bf407004e089000e60f50007a
:10c9a40027003a00c3c2bf00704060000004e000ea
:10c9b40039003a00803e2000406088001b003700a8
:10c9c400406080000000e00018003a004ce60700d8
:10c9d40077e707000ae70700604d80006a00b900a6
:10c9e40080007800c0f62100ef0007000000eb0093
:10c9f40070438800d3f2070060df2a0081f4070047
:10ca040070e02a00801f780070ce07008f87e9004d
:10ca1400c05d200034090700c3c2bf00704060003d
:10ca24000004e000fcff320021003700c3c2bf0055
:10ca3400704060000004e000e1ff3200160037009f
:10ca4400c3c2bf00704060000004e00012003a005e
:10ca540057e70700614d8000c0f62100d2000700af
:10ca64000000eb0070438800b6f2070030e22a00b1
:10ca740064f4070010e32a00801f780053ce0700f7
:10ca84008f87e900c3c2bf00704060000004e0006b
:10ca9400fcff320006003700cfc2bf000044b200e2
:10caa4000004e0003afe320069e9070038fe37006e
:10cab4004f05be004f04be000080fa0000000600cf
:10cac4000000fa0010002000e05f88001000200041
:10cad400f05f8800803e2000805f88000000eb004b
:10cae400800c88000000eb00b00c88004006200099
:10caf400600c880040062000700c8800e0002000d4
:10cb0400800c8800007d2000900c8800007d2000af
:10cb1400a00c8800e0002000b00c8800b0d42100f4
:10cb24007008880013e1a8008ce0a8000080fa00d7
:10cb3400000006000000fa000000eb00200c880052
:10cb4400f0002000000c8800f0002000100c880089
:10cb540060002000200c8800e001200060088800ac
:10cb640011e1a8000080fa00000006000000fa00ad
:10cb740011e1a9000080fa00000006000000fa009c
:10cb840011e1a8000080fa00000006000000fa008d
:10cb9400805f80000080fa00000006000200fa00b6
:10cba400000f7800100020009e0f100002003e00cd
:10cbb40020002000000f78001e0078000000d10043
:10cbc400000c88001e00e900600888000080fa005c
:10cbd400000006000200fa00000f78001e00780032
:10cbe400600c88000080fa00000006000200fa00d1
:10cbf400000f78001e007800900c88000080fa0076
:10cc040000000600809fbe00821f78003400f800f8
:10cc140000002000a00188000200fa00c05f80002c
:10cc2400000f78001e007800e20f50001e00320052
:10cc34001e007800e30f5000310032001e0078001f
:10cc4400e10f500003003200d222a8008c60a9003a
:10cc54003a003700d6c2bf000080fb000000d100bc
:10cc64000004a20061406000614060006140600017
:10cc74006140600000414000612d20009140780037
:10cc8400d0cfb30000c0600002407000d6e2b7000d
:10cc9400100880000000d100100888000000eb009c
:10cca400c05f880025003700d6c2bf000080fb00ab
:10ccb4000000d1000004a2006140600061406000f7
:10ccc400614060006140600000414000612d20002f
:10ccd40091407800d0cfb30000c0600002407000e3
:10cce400d6e2b700d6c2bf00624060000004e00094
:10ccf4001200320010002000c05f88000f003700cf
:10cd0400d6c2bf000080fb000000d1000004a200d6
:10cd1400614060006140600061406000614060000b
:10cd240000414000612d200091407800d0cfb30035
:10cd340000c0600002407000d6e2b7008460a90021
:10cd44000080fa003400f9004f0178004f00be0063
:10cd5400004006000200fa00000f780030002000b6
:10cd6400c05f88001e00e9001008880010088000d9
:10cd74000000d10000088800d622a900d222a90010
:10cd840005e1a8008460a9008c60a8000080fa0076
:10cd9400000006000000fa0020002000c05f8800a8
:10cda4000080fa00000006000400fa00000f78007a
:10cdb40011079800a05f80000000e0000d003a0019
:10cdc4001e0090000000e0000a003400b05f800004
:10cdd4000000e00007003a0068ff0700401f200041
:10cde400304588001e009000905f88001e00780087
:10cdf400d8ff07000080fa00000006000000fa00d7
:10ce04000000eb00d05f8800a04180000000e0003b
:10ce140005003200cae2a800106080006700b90073
:10ce240000608800ca62a800116080006049800028
:10ce3400ddff07001060800000004000a05f880054
:10ce44000080fa00000006000000fa001000200034
:10ce5400d05f8800a04180000000e000050032009f
:10ce6400cae2a800106080006700b9000060880072
:10ce7400ca62a800106080006300b90080007800d6
:10ce840060498000c8ff0700106080004200dd0098
:10ce9400a05f88000080fa00000006003600f80059
:10cea400809fbe00829fbe00849fbe00869fbe00fe
:10ceb4003400f80000002000a00188000200fa00fd
:10cec40084e0a900905f80000000e00011003200bf
:10ced400905f80000000e900905f8800905f800010
:10cee4000000e0000b003a00aaff07008049800020
:10cef400000040004108200080804000008b20009a
:10cf04000080400010007800e30f50000100320060
:10cf1400ca62a900006080000000e000070032003f
:10cf2400006080000000e90000608800006080006c
:10cf34000000e00001003a00cae2a900a05f8000fe
:10cf44000000e0000e003200a05f80000000e90055
:10cf5400a05f8800a05f80000000e00008003a00a5
:10cf6400d05f80000000e00003003a0010002000c1
:10cf7400e05f88000200370010002000f05f8800a6
:10cf8400406080000000e000030032004060800048
:10cf94000000e90040608800e0418000e20f50009a
:10cfa4000d003a00c8c2bf000042b2000004e00015
:10cfb40002003a000000eb00e05f8800c8c2bf0036
:10cfc400704060000004e00015003a000000eb002f
:10cfd400f05f880012003700c8c2bf000042b200f0
:10cfe4000004e00003003a000000eb00e05f88006a
:10cff4000200370010002000e05f8800c8c2bf00b4
:10d00400704060000004e00003003a000000eb0000
:10d01400f05f88000200370010002000f05f8800f5
:10d02400e0418000000f78001e007800e10f5000fe
:10d03400060035001e007800e20f50001500340091
:10d044001e007800e30f500035003200c8c2bf0054
:10d054000042b2000004e00005003a00a05f800036
:10d064000000e00002003a0064ff07004a003700b5
:10d07400c8c2bf00704060000004e00046003a00ef
:10d08400a05f80000000e00043003a006eff07004c
:10d0940041003700d05f80000000e0001000320043
:10d0a400e05f80000000e00005003a00a05f80001f
:10d0b4000000e00002003a0050ff0700360037008d
:10d0c400f05f80000000e00033003a00a05f8000c1
:10d0d4000000e00030003a005bff07002e0037003c
:10d0e400f05f80000000e00005003a00a05f8000cf
:10d0f4000000e00002003a0053ff0700260037005a
:10d10400e05f80000000e00023003a00a05f8000a0
:10d114000000e00020003a0038ff07001e0037003e
:10d12400c8c2bf000042b2000004e0000f003a0091
:10d13400b05f80000000e00004003a00100020000e
:10d14400b05f88006049800002ff0700a0418000b2
:10d154000000e00005003200cae2a8001060800070
:10d164006700b90000608800ca62a800c8c2bf0096
:10d174000042b2000004e00007003200b05f80000b
:10d184000000e00004003200ca62a90001ff0700a9
:10d194000000eb00b05f8800805f80000000e900c1
:10d1a400805f8800805f80000000e00010003a008b
:10d1b400803e2000805f8800d04180000000e800ad
:10d1c400d0418800504580000000e0000800320093
:10d1d400504580000000e90050458800504580001b
:10d1e4000000e00002003a001000200060458800c2
:10d1f400304580000000e00003003200304580002c
:10d204000000e90030458800206080000000e00054
:10d2140003003400206080000000e90020608800e2
:10d22400306080000000e0000300320030608000c5
:10d234000000e900306088000080fa003400f90042
:10d244004f03be004f02be004f01be004f00be00a0
:10d254003600f900004006000200fa000000eb006e
:10d26400000f7800504c8000e20f500005003a0097
:10d27400930107000000e0000200320010002000cb
:10d28400000f78001e0607000000e00002003200d4
:10d2940010002000000f78001e0078000080fa00c3
:10d2a400000006000000fa00e922a800e8c2a80075
:10d2b400e902a9000080fa00000006000600fa0056
:10d2c400200798000000eb00100798001a003700b0
:10d2d400e8c2a9002e009000610060000004e00094
:10d2e40002003200e902a80001003700e902a900a7
:10d2f4002e0090000000d100200798001e00780046
:10d304000000d100000f7800612e200091407800c9
:10d3140000c8b30000c060000004e0000200320056
:10d32400000028001e0f7000e8c2a8001e00900034
:10d334000000e800100798001e009000ef0f500056
:10d34400e3ff34001e0078000080fa0000000600ad
:10d354000400fa0010079800e922a9001e009000ba
:10d36400d6ff0700000f7800e922a800e902a9000f
:10d374001e0078000080fa00000006000600fa0093
:10d384001007980021079800e922a9001e009000c8
:10d39400caff07002e009000c8ff0700000f7800a6
:10d3a400e922a800e902a9001e0078000080fa0022
:10d3b400000006000a00fa002007980031079800d0
:10d3c40042079800e922a9002e009000bbff070045
:10d3d400100798003e009000b8ff0700100798005f
:10d3e4004e009000b5ff070010079800e902a9005d
:10d3f4000000eb00000f780007003700e8c2a90026
:10d404000000000000000000e8c2a80000000000c6
:10d41400000000001e0fe800700020009e0f1000a6
:10d42400f6ff3400e922a800e902a9001e009000da
:10d434000080fa00000006000200fa00e9c2a80019
:10d4440098ff070010002000c1ff0700d100200052
:10d4540050862800c9ff07008000eb0090002000e0
:10d46400c6ff070080007800f00f2000008f6000e6
:10d474000000eb00f0418800000e20009e0f100019
:10d4840009003a00d100200050862800bbff0700a5
:10d4940020072b00801f7800cccb07008f87e90082
:10d4a40010002000f04188000080fa00000006000f
:10d4b4000200fa00000f78001e007800c200dd00b0
:10d4c400a0042b00008040001000780070628800e7
:10d4d4001e0078004200dd008080e800a0042b00dc
:10d4e4000080400010007800806288000080fa000c
:10d4f400000006000400fa00000f780011079800ed
:10d504000000eb00d04188000ef007001e009000e0
:10d514000000e00008003a001e007800801f780038
:10d52400600a2b00801f78000084200089cb07004c
:10d53400e48757000a00370090fd0700401f2000d1
:10d54400304588001e007800801f7800600b2b0097
:10d55400801f7800008420007ecb0700e4875700fa
:10d5640000842000a7f10700d100200050862c0081
:10d5740082ff07001e007800cdff07004000200056
:10d5840073ff0700806280000001780070628000f1
:10d59400800078000009200086ff07001a00370089
:10d5a4001e0090000000e0000600320080c0b300be
:10d5b400daef0700d000200067060700e043880088
:10d5c40049e5070000c4b300d4ef0700d041800050
:10d5d400801f7800000c2b00801f7800008420003e
:10d5e4005ccb0700e48757000084200085f1070026
:10d5f40019ff07000000e0000300320020012000b2
:10d6040053ff070004003700e7c2bf00704060000a
:10d614000004e000e2ff3a00d10020005086280018
:10d6240056ff07000080fa00000006000400fa001c
:10d63400000f7800110798000000eb00d04188002b
:10d64400c0ef07001e0090000000e0000b003a004d
:10d654001e007800801f7800000d2b00801f7800ca
:10d66400008420003bcb0700e4875700d100200052
:10d6740050062c0041ff07000d0037003ffd070056
:10d68400401f2000304588001e007800801f78006d
:10d69400300e2b00801f7800008420002dcb070063
:10d6a400e4875700d10020005086280033ff07008c
:10d6b4000084200053f1070000c4b30097ef070073
:10d6c4001e0078007aff07004000200020ff0700ba
:10d6d4008062800000017800706280008000780021
:10d6e4002009200033ff0700e7c2bf00704060003c
:10d6f4000004e000fcff3a004000200014ff070093
:10d7040080628000000178007062800080007800f0
:10d714001009200027ff0700170037001e009000a3
:10d724000000e0000300320080c0b3007bef07007c
:10d73400ede4070000c4b30078ef0700d041800097
:10d74400801f7800000c2b00801f780000842000cc
:10d7540000cb0700e48757000084200029f107006c
:10d76400bdfe07000000e00003003200200120009d
:10d77400f7fe070004003700e7c2bf0070406000f6
:10d784000004e000e5ff3a0040002000f0fe07003e
:10d79400d100200050862800f8fe07000080fa001f
:10d7a40000000600809fbe003400f8000000200046
:10d7b400a00188000200fa0090108000004f780059
:10d7c4005cccbf000040e80080407800c2c9bf00c4
:10d7d40080cf5000080032005cccbf008080fb008a
:10d7e400309c2000008040001e4878005cccbf00c4
:10d7f4000040e8005cecb7000ec2bf00624060006d
:10d804000004e000010032000e22a9008520a900d6
:10d814000080fa003400f9004f00be00004006000a
:10d824000000fa00c0898500a01088000000eb0009
:10d83400601088000000eb00701088008520a900ab
:10d844008d20a8000de2a8000f42a8000080fa0075
:10d85400000006000200fa00000f780070002000ab
:10d864009e0f10000200340070002000000f7800aa
:10d874001e0078008000400020132b000080400030
:10d8840010007800a01088000080fa000000060054
:10d894000200fa00004f78000fc2bf00624060002f
:10d8a4000004e000fcff3a001e00fb00f10f200022
:10d8b40001006000801088000080fa00000006006b
:10d8c4000200fa00c1c5200091407800c2c9bf001f
:10d8d40000c05000004fe9001e80fb000080fa00e9
:10d8e400000006000000fa000040eb00c2e9b700a7
:10d8f40010c0b3005cecb7000080fa000000060022
:10d904000000fa00c2c9bf000040e800804078006f
:10d914005cccbf0080cf5000faff3200c2c9bf0008
:10d924000040e800c2e9b700c2c9bf008080fb0024
:10d93400309c200000804000104078000080fb00f4
:10d944000080fa00000006000200fa00ecff070065
:10d95400004f78001e407800cdff07001e80fb00ba
:10d964000080fa00000006000600fa006000b8001b
:10d974001007980021079800e1ff07008040780015
:10d984000174a100014f78001e407800c0ff070019
:10d99400f0c2b3009e4f10001600340090c3b300d1
:10d9a4009e4f100013003c009e009000a000200039
:10d9b400000ab8001e0090006000b900050178005c
:10d9c400000141002e0090006a00b90000014100ee
:10d9d400820278009e00fb0000fd2f0000804000c2
:10d9e400cf80de00040040008580480010079800c6
:10d9f40021079800d0c0b3009e4f1000deff3a000c
:10da04001e009000ae0090000080fa0000000600a6
:10da14000600fa00881f7800100798002107980074
:10da240090c0b300004f78000040eb00104798000e
:10da3400160037001e04fb001e009000ae0090008c
:10da4400a20020000300200016d6070002c3b30082
:10da54008240400030ac20000000440001487800bf
:10da64001e009000ae009000a200200003002000e1
:10da7400fcd5070010079800210798001e4fe90005
:10da84001e4090000040e800104798001e4090009f
:10da9400e94f5000e7ff34000040eb00cdeab70047
:10daa4004f0478000080fa00000006000400fa0029
:10dab400008fbe001e00be00d5ff0700c3cabf0012
:10dac40073ff0700c4cabf0071ff0700c5cabf00c7
:10dad4006fff0700c6cabf006dff0700c7cabf00bb
:10dae4006bff0700c8cabf0069ff0700c9cabf00af
:10daf40067ff0700cacabf0065ff0700cbcabf00a3
:10db040063ff0700cccabf0061ff07000080fa0072
:10db1400000006000200fa005cccbf008080fb001d
:10db2400c2c9bf000080fb00811f7800801f7800fd
:10db340020142b00801f780024ca0700e6875700b2
:10db44000000eb00000f7800060037009e0078000c
:10db5400309c200000804000104078004cff0700fb
:10db64001e0fe800e00f20009e0f1000f7ff3400a6
:10db74000080fa00000006003600f800809fbe0016
:10db8400829fbe00849fbe00869fbe003400f800c2
:10db940000002000a00188000200fa0030032000e9
:10dba400a01088000000eb00000f7800020037008e
:10dbb400000000001e0fe800f0cf27009e0f1000a9
:10dbc400fbff340080e52a00801f7800ffc90700ae
:10dbd4008f87e900103a8000801f780020e72a0030
:10dbe400801f7800f9c90700e4875700b7000700d1
:10dbf400ffff37003600f800809fbe00829fbe0002
:10dc0400849fbe00869fbe003400f8000000200000
:10dc1400a00188000000fa00805e8800915e880000
:10dc2400a25e8800b35e8800c45e8800d55e88006a
:10dc3400e65e8800f75e8800085f8800195f880048
:10dc44002a5f88003b5f88004c5f88005d5f880026
:10dc54006e5f88007f5f880000e82a00801f7800dc
:10dc6400dac907008f87e900805e8000801f780092
:10dc740080e92a00801f7800d4c90700e487570090
:10dc8400905e8000801f780020ea2a00801f7800c0
:10dc9400cec90700e4875700a05e8000801f78008b
:10dca400c0ea2a00801f7800c8c90700e48757002b
:10dcb400b05e8000801f780060eb2a00801f78002f
:10dcc400c2c90700e4875700c05e8000801f780047
:10dcd40000ec2a00801f7800bcc90700e4875700c5
:10dce400d05e8000801f7800a0ec2a00801f78009e
:10dcf400b6c90700e4875700e05e8000801f780003
:10dd040040ed2a00801f7800b0c90700e48757005f
:10dd1400f05e8000801f7800e0ed2a00801f78000c
:10dd2400aac90700e4875700005f8000801f7800bd
:10dd340080ee2a00801f7800a4c90700e4875700fa
:10dd4400105f8000801f780020ef2a00801f780079
:10dd54009ec90700e4875700205f8000801f780079
:10dd6400c0ef2a00801f780098c90700e487570095
:10dd7400305f8000801f780070f02a00801f7800d8
:10dd840092c90700e4875700405f8000801f780035
:10dd940020f12a00801f78008cc90700e48757000f
:10dda400505f8000801f7800d0f12a00801f780027
:10ddb40086c90700e4875700605f8000801f7800f1
:10ddc40080f22a00801f780080c90700e48757008a
:10ddd400705f8000801f780030f32a00801f780075
:10dde4007ac90700e487570038000700ffff3700af
:10ddf4003600f800809fbe00829fbe00849fbe0054
:10de0400869fbe003400f80000002000a0018800b6
:10de14000000fa007f5f88000f902000e0f32a00e2
:10de2400801f780069c907008f87e900705f800050
:10de3400801f780030f32a00801f780063c9070030
:10de4400e487570021000700ffff37003600f80081
:10de5400809fbe00829fbe00849fbe00869fbe003e
:10de64003400f80000002000a00188000000fa003f
:10de740040f52a00801f780054c907008f87e90005
:10de840012000700ffff37003600f800809fbe0035
:10de9400829fbe00849fbe00869fbe003400f800af
:10dea40000002000a00188000000fa0090a0a90052
:10deb4009120a90090f62a00801f780043c907002a
:10dec4008f87e90001000700ffff37000000fa0018
:10ded4009ced070060f82a004aef070000003700b5
:10dee400cfc2bf000044b2000004e000fcff3200d7
:08def400cfa2a900faff3700dc
:020000040000fa
:10defc005a0c0000020000000200000000000000ac
:10df0c0000080000c201000000000000c20900006f
:10df1c000c010000000000005c0c0000020000007e
:10df2c0002000000010000003c0c00000600000094
:10df3c0000000000420c0000060000000000000081
:10df4c00d00b00002000000000000000f00b0000cf
:10df5c001a00000000000000480c00000600000041
:10df6c0000000000240c000018000000000000005d
:10df7c004e0c00000400000000000000520c0000d9
:10df8c000400000000000000ce0a000002010000a6
:10df9c00000000005e0c0000020000000200000007
:10dfac0001000000560c00000400000000000000fe
:10dfbc000a0c00001a00000000000000600c0000b9
:10dfcc008800000002000000c00c98000c700c00cf
:10dfdc00000000000000000000000000000208002b
:10dfec00020296000c970c00960c96000c960c00f6
:10dffc00960c86000c0000000000000000000000e1
:10e00c000000000000000000000000000000000004
:10e01c000000020008010100be0cbf000cbe0c0089
:10e02c00be0cbe000cbe0c00ae0c000000000000cc
:10e03c0000000000000000000000000000000000d4
:10e04c0000000000000000000100000000e60c00d1
:10e05c00e70ce6000ce60c00e60ce6000cd60c0017
:10e06c0000000000000000000000000000000000a4
:10e07c000000000000000000000000000000000094
:10e08c00840d0000120000000200000001000200dc
:10e09c00000400000800100000000000202b2d00e0
:10e0ac0023300000960d0000080000000200000064
:10e0bc00686a6c00747a4c00000000009e0d000031
:10e0cc000600000002000000040000000000000038
:10e0dc00a40d00000200000000000000620d000012
:10e0ec0022000000020000003031320033343500d1
:10e0fc0036373800396162006364650066003000b1
:10e10c003132330034353600373839004142430060
:10e11c004445460000000000e80c000048000000e8
:10e12c00020000000000000000000000244000007d
:10e13c00000000000000590040000000000000003a
:10e14c0088c34000000000000084d7009741000005
:10e15c0080e0370079c3410043176e0005b5b50068
:10e16c00b8934600f5f93f00e9034f00384d3200f3
:10e17c001d30f900487782005a3cbf00737fdd00e8
:10e18c004f157500300d0000320000000200000039
:10e19c004e414e00006e61006e0049004e4600007c
:10e1ac00696e66000030310032333400353637008a
:10e1bc0038396100626364006566000030313200fa
:10e1cc00333435003637380039414200434445007a
:10e1dc0046000000a60d0000020000000200000036
:10e1ec0000000000a80d000002000000020000006a
:10e1fc0030000000aa0d0000020000000200000028
:10e20c0000000000ac0d0000020000000200000045
:10e21c0001000000ae0d0000020000000000000034
:04e22c0000000000ee
:020000040000fa
:10e230000800fa00a3fd07000000e000ae00320075
:10e24000b0fd0700004f7800f04180000000e000c2
:10e2500002003a000040eb00004f78001e80fb00f7
:10e2600030079800d0042000be009000808f50003e
:10e270002b003200d0042000be009000808f5000a0
:10e2800011003c0090032000be009000808f5000e1
:10e2900008003c0000032000be009000808f50006a
:10e2a00043003d003e0090000000e0008900320085
:10e2b0008d00370050042000be009000808f500079
:10e2c0002d0032008800370020052000be0090009d
:10e2d000808f50001200320020052000be00900008
:10e2e000808f500005003c0000052000be0090001b
:10e2f000808f50000a0032007b003700300520007c
:10e30000be009000808f50001100320040052000b8
:10e31000be009000808f5000010032007200370074
:10e320001e40780054ecb700614d8000108f210032
:10e330009efa070080f92a00801f780024c8070091
:10e340008f87e9001e40780052fd07006a00370001
:10e35000b0fa2a00801f78001dc807008f87e900e7
:10e3600020012000fbfb0700614d8000108f210081
:10e370008efa07006000370060fc2a00801f7800da
:10e3800013c807008f87e900604d80006a00b9005c
:10e3900080007800108f210084fa070030052000eb
:10e3a000ecfb07000040eb0054ecb70052003700d4
:10e3b0009e80fb0000fd2f000080400090628800de
:10e3c00090628000801f7800f0fd2a00801f780096
:10e3d000ffc70700e48757009062800035fc070004
:10e3e00054ccbf000080fb002007980000052000ef
:10e3f000ae009000808f5000120032000005200017
:10e40000ae009000808f500005003c00d00420003a
:10e41000ae009000808f500026003200360037009a
:10e4200020052000ae009000808f500019003200bf
:10e4300040052000ae009000808f5000090032009f
:10e440002d003700a0fe2a00801f7800e0c70700db
:10e450008f87e900906280008000eb0026fc0700b7
:10e4600025003700c0ff2a00801f7800d8c70700aa
:10e470008f87e900e9e2a800cae2a8009062800064
:10e48000110020001cfc0700cae2a900e9e2a90073
:10e490001900370050002b00801f7800ccc7070000
:10e4a0008f87e900906280001100200060fc070067
:10e4b00011003700d0002b00801f7800c4c7070070
:10e4c0008f87e900906280008000eb0058fc070015
:10e4d0000900370030022b00801f7800bcc70700fe
:10e4e0008f87e9000400370070042b00801f78003c
:10e4f000b7c707008f87e9000080fa000000060018
:10e50000809fbe00821f78003400f80000002000c9
:10e51000a00188000000fa0082c0bf000080fb005c
:10e520004400de000004a200614060006140600021
:10e5300061406000614060004401dd00210820006e
:10e5400091407800f0ceb30000c06000024070003f
:10e5500082e0b70088a0a90010c0b30040ecb7006b
:10e56000e06180000000e0001b00320082c0bf00bc
:10e57000704060000004e0000c003a00c3c2bf001d
:10e580000044b2000004e00004003200f0618000aa
:10e590000000e800f06188000f003700f0618000a3
:10e5a0000000e900f06188000b003700c3c2bf0023
:10e5b0000044b2000004e00004003200f06180007a
:10e5c0000000e900f061880003003700f06180007e
:10e5d0000000e800f06188000000eb00e0618800c6
:10e5e0000080fa003400f9004f0178004f00be00af
:10e5f00000400600809fbe00821f78003400f800b3
:10e6000000002000a00188000000fa0082c0bf00c6
:10e610000080fb004300de000004a20061406000b7
:10e620006140600061406000614060004301dd00c6
:10e63000210820009140780070cfb30000c0600036
:10e640000240700082e0b7008880a90010c0b300cb
:10e6500040ecb700e06180000000e0001d003a00df
:10e6600082c0bf00684060000004e0000d003a0076
:10e67000c3c2bf0001c8b300014060000004e00055
:10e6800004003200f06180000000e900f0618800c1
:10e6900010003700f06180000000e800f0618800a1
:10e6a0000c003700c3c2bf0001c8b30001406000c6
:10e6b0000004e00004003200f06180000000e80087
:10e6c000f061880003003700f06180000000e9007d
:10e6d000f061880010002000e06188000080fa00ee
:10e6e0003400f9004f0178004f00be0000400600e2
:10e6f0000000fa0088a0a90090a0a8008880a900c6
:10e700009080a8000080fa00000006000200fa00d5
:10e71000f0618000000f78000000eb00f0618800dd
:10e720000040eb0040ecb7001e0078000080fa00cb
:10e73000000006000600fa0010079800f161800052
:10e740001e009000808f5000070034000000eb0096
:10e75000f06188000040eb0040ecb70010002000a2
:10e76000200798000e0037001e0090008000ea008d
:10e77000f0618000808f5000070034000000eb0043
:10e78000f06188000040eb0040ecb7000080eb0037
:10e7900020079800020037000000eb0020079800d7
:10e7a0002e0090000080fa00000006000800fa0029
:10e7b000d40007000000e0007c003200e100070008
:10e7c000004f7800f04180000000e0007700320048
:10e7d0001e80fb0030079800d0042000be0090008f
:10e7e000808f500027003200d0042000be0090002f
:10e7f000808f50000d003c0000032000be00900000
:10e80000808f50006900350090032000be0090000a
:10e81000808f50003300340050042000be00900070
:10e82000808f500025003200600037002005200056
:10e83000be009000808f50001200320020052000a2
:10e84000be009000808f500005003c0000052000b5
:10e85000be009000808f50000a0032005300370045
:10e8600030052000be009000808f50000b00320069
:10e8700040052000be009000808f50000100320053
:10e880004a0037001e40780058ecb700614d800008
:10e89000108f210045f907004400370020012000b7
:10e8a000acfa0700614d8000108f21003ff907008e
:10e8b0000040eb0058ecb7003c003700604d800092
:10e8c0006a00b90080007800108f210037f9070036
:10e8d000300520009ffa07000040eb0058ecb7001d
:10e8e000320037009e80fb0000fd2f0000804000ba
:10e8f000b0628800b0628000eefa070058ccbf001a
:10e900000080fb002007980000052000ae0090006a
:10e91000808f50001200320000052000ae009000f1
:10e92000808f500005003c00d0042000ae00900015
:10e93000808f50001a0032001c0037002005200094
:10e94000ae009000808f5000110032004005200082
:10e95000ae009000808f5000050032001300370099
:10e96000b06280008000eb00e3fa07000f00370080
:10e97000e9e2a800cae2a800b0628000110020000d
:10e98000ddfa0700cae2a900e9e2a90007003700a2
:10e99000b06280001100200025fb07000300370053
:10e9a000b06280008000eb0021fb07000080fa00cd
:10e9b00000000600809fbe003400f8000000200028
:10e9c000a00188000200fa00e0108000004f7800eb
:10e9d0005eccbf000040e80080407800cecabf0097
:10e9e00080cf5000080032005eccbf008080fb006a
:10e9f000f0ac2000008040001e4878005eccbf00d4
:10ea00000040e8005eecb70018c2bf006240600042
:10ea10000004e000010032001822a9008700a900cc
:10ea20000080fa003400f9004f00be0000400600ec
:10ea30000000fa00c08b8500f01088000000eb0099
:10ea4000b010880000402000c01088008700a90096
:10ea50008f00a80017e2a8001942a8000080fa0061
:10ea6000000006000200fa00000f7800700020008d
:10ea70009e0f10000200340070002000000f78008c
:10ea80001e0078008000400020172b00008040000e
:10ea900010007800f01088000080fa0000000600e6
:10eaa0000200fa00004f780019c2bf006240600007
:10eab0000004e000fcff3a001e00fb00f10f200004
:10eac00001006000d01088000080fa0000000600fd
:10ead0000200fa00000f7800040037001e007800e2
:10eae00010407800eeff07001e0fe8001e007800bf
:10eaf000104078000004e000f8ff3a000080fa00bf
:10eb0000000006000200fa00e1c5200091407800f4
:10eb1000cecabf0000c05000004fe9001e80fb00bd
:10eb20000080fa00000006000000fa000040eb0040
:10eb3000ceeab70010c0b3005eecb7000080fa0068
:10eb4000000006000000fa00cecabf000040e80046
:10eb5000804078005eccbf0080cf5000faff3200ca
:10eb6000cecabf000040e800ceeab700cecabf0060
:10eb70008080fb00f0ac2000008040001040780056
:10eb80000080fb000080fa00000006000200fa008e
:10eb9000ecff0700004f78001e407800c0ff070020
:10eba0001e80fb000080fa00000006003200f80022
:10ebb000900188006118e100040032007018e10043
:10ebc00002003200f0ff2f00030037003119ba00b5
:10ebd0008301e900fdff3a003200f9000000060061
:10ebe000849fbe004220a900440424006110e1007b
:10ebf0000a003200540424007010e10007003200c3
:10ec000064042400f5ff2f000510e100030032002a
:10ec1000f0ff2f004f02be00000006003200f80097
:10ec2000203b8800113b8800043b88000500fc0065
:10ec300050052000303b8800a00a2000303b8800af
:10ec400061e7a800000000000000000061e7af00dd
:10ec5000feff37000000eb003200f9004f02be005b
:10ec600000000600841f78004220a9004400240010
:10ec70006118e10006003200540024007018e10021
:10ec8000030032004f027800f0ff2f000000060062
:10ec90003200f80091018800821f78003019bb0013
:10eca0008301e900fdff3a00213b88004f01780015
:10ecb000123b8800043b88000500fc005005200042
:10ecc000303b8800a00a2000303b880061e7a800a4
:10ecd000000000000000000061e7af00feff370009
:10ece0000000eb003200f9004f027800000006003f
:10ecf0000400fa00204798000040eb00004f780025
:10ed00000f0037002e4090000080fb006100600083
:10ed10000004e00002003200e202a8000100370017
:10ed2000e202a900e222a8002e4090000080fb0031
:10ed30000000d10020479800e222a9001e4fe80001
:10ed400070c0b3009e4f1000eeff34000080fa0048
:10ed5000000006000600fa0010079800210798003e
:10ed60001e009000ae0090001062880021628800b2
:10ed70000040eb00004f7800060037009e00fb00cb
:10ed800020c420000080400010407800d8ff070019
:10ed90001e4fe80041c0b3009ecf1000f7ff3400c3
:10eda000e822a800e822a9000080fa00000006007e
:10edb0000000fa00e802a800e202a900e802a900a7
:10edc000e822a800e822a90010c0b30046ecb70072
:10edd0000080fa00000006000000fa00ca42a90004
:10ede0000000eb00606288000000eb0040628800d9
:10edf00090432000101188000000280000118800b6
:10ee00008500a9008d00a8000080fa00000006001f
:10ee10000200fa00000f7800406280009e0f100090
:10ee20000800320020c2bf00624060000004e00021
:10ee3000fcff3a001e007800201188001e007800b8
:10ee4000406288000080fa0000000600801f780001
:10ee50003400f80000002000a00188000200fa0041
:10ee6000ca42a8008500a90020c2bf00614060001e
:10ee70000004e0000400320020118000506288008d
:10ee80001000200060628800ca42a9000080fa00d9
:10ee90003400f9004f007800004006000200fa003c
:10eea000000f78000000eb00c00888001e0078000a
:10eeb000010020004309dd00cd00de00810071006b
:10eec0004300dd00e008880086c0a90021e1a80019
:10eed00086c0bf000044b2000004e000fcff320026
:10eee00021e1a9000080fa00000006000400fa00f9
:10eef000100798000000eb00000f780003003700b7
:10ef0000803e2000e5ff07001e0fe8001e00900075
:10ef10009e0f1000faff39000080fa000000060082
:10ef20000000fa000000eb0050158800f01f2000e0
:10ef300040158800f00020003015880000082000ef
:10ef4000201588000000eb00101588000000280044
:10ef5000001588000080fa00000006000200fa0098
:10ef6000000f78009e0078006f80600030158800e8
:10ef7000a022a800401f2000c8ff0700a022a9006f
:10ef8000a0c2bf00614060000004e000fcff32004e
:0cef9000001480000080fa000000060061
:00000001FF
